:020000040800F2
:10000000D8FF0120612E0008251B00082B1B0008CB
:10001000311B0008371B00083D1B000800000000D2
:10002000000000000000000000000000431B00086A
:10003000511B0008000000005F1B00086D1B00083A
:10004000B12E0008B12E0008B12E0008B12E000814
:10005000B12E0008B12E00087B1B0008B12E00084D
:10006000B12E0008B12E0008B12E0008B12E0008F4
:10007000B12E0008B12E0008B12E0008B12E0008E4
:10008000891B00089D1B0008B11B0008B12E000849
:10009000B12E0008B12E0008B12E0008B12E0008C4
:1000A000B12E0008C51B0008B12E0008B12E0008B3
:1000B000D91B0008ED1B0008011C0008B12E000828
:1000C000B12E0008B12E0008B12E0008B12E000894
:1000D000B12E0008B12E0008151C0008B12E000832
:1000E000291C0008B12E0008B12E0008611C000870
:1000F000751C0008891C00089D1C0008B12E000812
:10010000B12E0008B12E0008B11C0008B12E000865
:10011000B12E0008B12E0008B12E0008B12E000843
:10012000C51C0008B12E0008B12E0008B12E000831
:10013000B12E00080000000000000000B12E0008F1
:10014000B12E0008B12E0008B12E0008D91C0008FD
:10015000B12E0008B12E0008B12E0008B12E000803
:10016000B12E0008B12E0008B12E0008B12E0008F3
:10017000B12E0008B12E0008B12E000800000000CA
:1001800000000000B12E0008000000000000000088
:10019000B12E00080000000000000000B12E000891
:1001A000000000000000000000000000B12E000868
:1001B000B12E0008B12E0008B12E0008B12E0008A3
:0401C000B12E000854
:1001C40010B5054C237833B9044B13B10448AFF38D
:1001D40000800123237010BD1801002000000000DE
:1001E400D0F2000808B5034B1BB103490348AFF331
:1001F400008008BD000000001C010020D0F20008AF
:10020400034613F8012B002AFBD1181A0138704752
:1002140053B94AB9002908BF00281CBF4FF0FF3169
:100224004FF0FF3000F074B9ADF1080C6DE904CE65
:1002340000F006F8DDF804E0DDE9022304B07047BD
:100244002DE9F047089D04468E46002B4DD18A4285
:10025400944669D9B2FA82F252B101FA02F3C2F1B8
:10026400200120FA01F10CFA02FC41EA030E944049
:100274004FEA1C48210CBEFBF8F61FFA8CF708FB6A
:1002840016E341EA034306FB07F199420AD91CEB42
:10029400030306F1FF3080F01F81994240F21C8174
:1002A400023E63445B1AA4B2B3FBF8F008FB1033BC
:1002B40044EA034400FB07F7A7420AD91CEB0404F1
:1002C40000F1FF3380F00A81A74240F207816444C1
:1002D400023840EA0640E41B00261DB1D440002346
:1002E400C5E900433146BDE8F0878B4209D9002DAA
:1002F40000F0EF800026C5E9000130463146BDE834
:10030400F087B3FA83F6002E4AD18B4202D382429D
:1003140000F2F980841A61EB030301209E46002D4C
:10032400E0D0C5E9004EDDE702B9FFDEB2FA82F2A1
:10033400002A40F09280A1EB0C014FEA1C471FFAFF
:100344008CFE0126200CB1FBF7F307FB131140EAE6
:1003540001410EFB03F0884208D91CEB010103F1B3
:10036400FF3802D2884200F2CB804346091AA4B275
:10037400B1FBF7F007FB101144EA01440EFB00FE49
:10038400A64508D91CEB040400F1FF3102D2A645AE
:1003940000F2BB800846A4EB0E0440EA03409CE74D
:1003A400C6F12007B34022FA07FC4CEA030C20FAFA
:1003B40007F401FA06F31C43F9404FEA1C4900FA1A
:1003C40006F3B1FBF9F8200C1FFA8CFE09FB181197
:1003D40040EA014108FB0EF0884202FA06F20BD90A
:1003E4001CEB010108F1FF3A80F08880884240F25A
:1003F4008580A8F102086144091AA4B2B1FBF9F09E
:1004040009FB101144EA014100FB0EFE8E4508D998
:100414001CEB010100F1FF346CD28E456AD902381D
:10042400614440EA0840A0FB0294A1EB0E01A14202
:10043400C846A64656D353D05DB1B3EB080261EB70
:100444000E0101FA07F722FA06F3F1401F43C5E94A
:10045400007100263146BDE8F087C2F12003D84080
:100464000CFA02FC21FA03F3914001434FEA1C47C2
:100474001FFA8CFEB3FBF7F007FB10360B0C43EAB4
:10048400064300FB0EF69E4204FA02F408D91CEB64
:10049400030300F1FF382FD29E422DD90238634462
:1004A4009B1B89B2B3FBF7F607FB163341EA034102
:1004B40006FB0EF38B4208D91CEB010106F1FF3851
:1004C40016D28B4214D9023E6144C91A46EA004648
:1004D40038E72E46284605E70646E3E61846F8E6DA
:1004E4004B45A9D2B9EB020864EB0C0E0138A3E723
:1004F4004646EAE7204694E74046D1E7D0467BE704
:10050400023B614432E7304609E76444023842E77B
:10051400704700BF80B584B004AF4FF4805302939A
:1005240005230193164B009310231022A021154894
:1005340004F0F6FA0346002B1ED1322002F0FAFC36
:100544004FF480530293052301930F4B0093102320
:100554001022A0210B4804F0DDFB0346002B09D137
:10056400094B9A78064B9B789A4201D1002304E008
:10057400012302E0012300E001231846BD4680BDAB
:1005840000000020780200203401002080B582B0F1
:1005940000AF222002F0D6FB02F0C4FB0346FB713D
:1005A40002F0F6FBFB7918460837BD4680BD000013
:1005B40080B582B000AF00237B600BE002F0F4FB57
:1005C4000346002B03D0FFF7E1FF034607E07B68F7
:1005D40001337B607B68044A9342EFD9FA231846BF
:1005E4000837BD4680BD00BF3F4B4C0080B582B08C
:1005F40000AF0346FB71FB79184602F0A3FB02F03F
:10060400C7FBFFF7D5FF034618460837BD4680BD34
:1006140080B500AF02F0C8FB0346002B01D0FFF702
:10062400B5FF3020FFF7E2FF0346184680BD000007
:1006340080B584B000AF3B4600221A605A609A60CD
:10064400DA604B4B4B4A1A60494B00225A60484BC4
:1006540000229A60464B01221A61454B01221A7608
:10066400434B002283F82020414B0022DA62404BA6
:10067400414A9A623E4B0022DA603D4B0722DA611E
:100684003B4B012283F83020394B00225A61384811
:1006940002F074FC0346002B01D001F04BF8082350
:1006A4003B6001237B600723BB603B46194630480F
:1006B40002F040FF0346002B01D001F03BF8092370
:1006C4003B6002237B603B461946294802F032FF17
:1006D4000346002B01D001F02DF80A233B600323CD
:1006E4007B603B461946224802F024FF0346002B58
:1006F40001D001F01FF80B233B6004237B603B46D1
:1007040019461B4802F016FF0346002B01D001F0E6
:1007140011F80C233B6005237B603B4619461448C3
:1007240002F008FF0346002B01D001F003F80D236B
:100734003B6006237B603B4619460D4802F0FAFEF7
:100744000346002B01D000F0F5FF0F233B60072385
:100754007B603B461946064802F0ECFE0346002B3C
:1007640001D000F0E7FF00BF1037BD4680BD00BFD9
:100774003C010020002001400100000F80B58AB038
:1007840000AF786007F1140300221A605A609A607F
:10079400DA601A617B681B683F4A934278D1002370
:1007A4003B613E4B5B6C3D4A43F4807353643B4B6B
:1007B4005B6C03F480733B613B690023FB60374B44
:1007C4001B6B364A43F004031363344B1B6B03F077
:1007D4000403FB60FB680023BB60304B1B6B2F4A98
:1007E40043F0020313632D4B1B6B03F00203BB6046
:1007F400BB682F237B610323BB610023FB6107F1EB
:1008040014031946264803F04FFE03237B61032398
:10081400BB610023FB6107F114031946214803F06F
:1008240043FE214B214A1A601F4B00225A601E4B83
:1008340000229A601C4B0022DA601B4B4FF480624A
:100844001A61194B4FF480525A61174B4FF480428E
:100854009A61154B0022DA61134B00221A62124B83
:1008640000225A62104803F01DFA0346002B01D0FF
:1008740000F060FF7B680C4A9A630B4A7B689363C1
:1008840000220021122003F0DEF9122003F0F7F910
:1008940000BF2837BD4680BD00200140003802401B
:1008A4000008024000040240840100201064024059
:1008B40080B582B000AF78607B681B68064A9342BB
:1008C40005D1064B01221A70054802F0BBFD00BF9A
:1008D4000837BD4680BD00BF00200140E401002070
:1008E4003C01002080B485B000AF0346FB80FB8848
:1008F4001B0AFB81FB881B02FB80FA89FB881344DB
:10090400FB81FB8918461437BD465DF8047B7047AC
:1009140080B485B000AF78607B68A82202FB03F343
:100924009B08FB6000BFFB685A1EFA60002BF9D1DC
:1009340000BF00BF1437BD465DF8047B704700005C
:1009440080B400AF104B4AF25A521A800E4B152253
:100954009A700D4B8222DA700B4B52229A800B4B09
:100964004AF25A521A80094B04229A70074B832286
:10097400DA70064B51229A80044B10229A7100BF00
:10098400BD465DF8047B70472C0200204402002021
:10099400B0B586B000AF00233B603B1D00221A6057
:1009A4005A609A60DA601A610A4B3C461D460FCDC4
:1009B4000FC495E8030084E803003B461822194657
:1009C400054809F033F9052002F0B4FA00BF1837DE
:1009D400BD46B0BD2C0200209805002080B582B031
:1009E40000AF0B4A3B4692E80300186004331980B9
:1009F40002330A0C1A703B4607221946054809F0CF
:100A040015F9052002F096FA00BF0837BD4680BDEF
:100A1400440200209805002080B400AF1B4B9A8A42
:100A24001B4B1B685A63194BDA8A194B1B689A6370
:100A3400164B1A8B164B1B68DA63144B5A8B144BE8
:100A44001B681A64114B1A89124B1B685A630F4BAB
:100A54005A89104B1B689A630C4B9A890D4B1B687F
:100A6400DA630A4BDA890B4B1B681A64074B1A8A40
:100A7400094B1B689A63054B5A8A074B1B68DA6358
:100A840000BFBD465DF8047B704700BF4C020020E8
:100A940064040020AC0400203C05002080B500AFB5
:100AA400FFF74EFF02F096F9FFF734FD03469BB2C1
:100AB4001846FFF717FF03461A46034BDA8201F084
:100AC40085FE00BF80BD00BF2C02002080B500AFB2
:100AD4008A4B1B78012B04D1884B00221A70FFF734
:100AE4007DFF874B1B78012B40F00B82854B1B78D5
:100AF4005A2B40F0FB81834B9B78242B40F0F681EA
:100B04002822002180480EF0C3FB7F4B1A897D4BBD
:100B1400DB799BB213439AB27B4B1A817A4B1B89C4
:100B24001B029AB2784B1A81774B1A89754B1B7A40
:100B34009BB213439AB2744B1A81734B5A89714B0B
:100B44005B7A9BB213439AB26F4B5A816E4B5B89AB
:100B54001B029AB26C4B5A816B4B5A89694B9B7A34
:100B64009BB213439AB2684B5A81674B9A89654B7F
:100B7400DB7A9BB213439AB2634B9A81624B9B8993
:100B84001B029AB2604B9A815F4B9A895D4B1B7B27
:100B94009BB213439AB25C4B9A815B4BDA89594BF3
:100BA4005B7B9BB213439AB2574BDA81564BDB897A
:100BB4001B029AB2544BDA81534BDA89514B9B7B1B
:100BC4009BB213439AB2504BDA814F4B1A8A4D4B66
:100BD400DB7B9BB213439AB24B4B1A824A4B1B8A60
:100BE4001B029AB2484B1A82474B1A8A454BDB7C4C
:100BF4009BB213439AB2444B1A82434B5A8A414BD9
:100C04005B7C9BB213439AB23F4B5A823E4B5B8A46
:100C14001B029AB23C4B5A823B4B5A8A394B9B7CFF
:100C24009BB213439AB2384B5A82374B9A8A354B4C
:100C3400DB7C9BB213439AB2334B9A82324B9B8A2E
:100C44001B029AB2304B9A822F4B9A8A2D4B1B7DF2
:100C54009BB213439AB22C4B9A822B4BDA8A294BC0
:100C64005B7D9BB213439AB2274BDA82264BDB8A15
:100C74001B029AB2244BDA82234BDA8A214B9B7DE6
:100C84009BB213439AB2204BDA821F4B1A8B1D4B33
:100C9400DB7D9BB213439AB21B4B1A831A4B1B8BFB
:100CA4001B029AB2184B1A83174B1A8B154B1B7ED7
:100CB4009BB213439AB2144B1A83134B5A8B114BA6
:100CC4005B7E9BB213439AB20F4B5A830E4B5B8BE2
:100CD4001B029AB20C4B5A830B4B5A8B094B9B7ECB
:100CE4009BB213439AB2084B5A83074BB3F91C20A7
:100CF400044BDB7E1BB213431AB207E0070000204B
:100D040008000020040200204C0200207E4B9A833D
:100D14007D4BB3F91C301B021AB27B4B9A837A4B7E
:100D2400B3F91C20794B1B7F1BB213431AB2764BC9
:100D34009A83754BB3F91E20744B5B7F1BB213432C
:100D44001AB2714BDA83704BB3F91E301B021AB21C
:100D54006D4BDA836C4BB3F91E206C4B9B7F1BB23B
:100D640013431AB2684BDA83674BB3F92020674BFD
:100D7400DB7F1BB213431AB2634B1A84624BB3F981
:100D840020301B021AB2604B1A845F4BB3F9202047
:100D94005E4B93F820301BB213431AB25A4B1A8499
:100DA400594BB3F92220594B93F821301BB213430A
:100DB4001AB2554B5A84544BB3F922301B021AB25F
:100DC400514B5A84504BB3F92220504B93F82230A4
:100DD4001BB213431AB24C4B5A844B4BB3F9242025
:100DE4004A4B93F823301BB213431AB2464B9A84EE
:100DF400454BB3F924301B021AB2434B9A84424B3D
:100E0400B3F92420414B93F824301BB213431AB294
:100E14003D4B9A843C4BDA8C3C4B93F825309BB287
:100E240013439AB2384BDA84374BDB8C1B029AB2E9
:100E3400354BDA84344BDA8C344B93F826309BB23E
:100E440013439AB2304BDA842F4BDB8C002B04D142
:100E5400FFF7E2FD01F016FE48E0282200212A48AF
:100E64000EF016FA2A4B1B78012B09D1264B0122CE
:100E74009A83254B0122DA83234B01221A840BE047
:100E8400214B4FF6FF729A831F4B4FF6FF72DA83A2
:100E94001D4B4FF6FF721A8401F0F4FD1D4B1B68C5
:100EA40032225A631B4B1B6832229A63194B1B680C
:100EB4003222DA63174B1B6832221A64164B1B6802
:100EC40032225A63144B1B6832229A63124B1B68FA
:100ED4003222DA63104B1B6832221A640F4B1B68F0
:100EE40032229A630D4B1B683222DA630C4B0022C8
:100EF4001A70272205490B4808F016FF052002F056
:100F040019F800BF80BD00BF4C020020040200207D
:100F14000600002064040020AC0400203C050020EE
:100F2400080000209805002080B500AF334B1B78E3
:100F3400012B61D1324B1B78012B5DD12F4B002249
:100F44001A702F4B00221A702E4B1B689BB2184646
:100F5400FFF7C8FC03461A462B4B1A82294B5B68E1
:100F64009BB21846FFF7BEFC03461A46264B5A822C
:100F7400244B9B689BB21846FFF7B4FC03461A4601
:100F8400214BDA801F4BDB689BB21846FFF7AAFCA3
:100F940003461A461C4B1A811A4B1B699BB218460E
:100FA400FFF7A0FC03461A46174B5A81154B5B69A1
:100FB4009BB21846FFF796FC03461A46124B9A81D9
:100FC400104B9B699BB21846FFF78CFC03461A46EC
:100FD4000D4BDA8101F02FFF03469BB21846FFF751
:100FE40081FC03461A46084B9A82072205490748A2
:100FF40002F018F9FFF7CCFC00BF80BDE40100202B
:1010040007000020E80100202C0200203C01002001
:1010140080B500AF054B1B78002B02D1FFF784FF8E
:1010240001E0FFF753FD00BF80BD00BFE5010020D4
:1010340080B500AF084B1B68084A93420AD1064B9F
:1010440000221A60064B1B681A46064B1A60054BB1
:101054001B68984700BF80BDFCFF0120EFBEADDEDA
:101064000400FF1F7402002080B500AF034B044A44
:101074001A6002F012FE00BF80BD00BFFCFF012019
:10108400EFBEADDE80B582B000AF00237B601B4BAA
:101094001B6B1A4A43F480031363184B1B6B03F452
:1010A40080037B607B6800233B60144B1B6B134AFB
:1010B40043F400131363114B1B6B03F400133B60E5
:1010C4003B6800220021102002F0BDFD102002F038
:1010D400D6FD00220021112002F0B5FD112002F0FE
:1010E400CEFD00220021382002F0ADFD382002F0B0
:1010F400C6FD00BF0837BD4680BD00BF00380240B2
:1011040080B58CB000AF07F11C0300221A605A604E
:101114009A60DA601A610023BB61944B1B6B934A9B
:1011240043F010031363914B1B6B03F01003BB617B
:10113400BB6900237B618D4B1B6B8C4A43F004031A
:1011440013638A4B1B6B03F004037B617B690023ED
:101154003B61864B1B6B854A43F080031363834BCF
:101164001B6B03F080033B613B690023FB607F4BF7
:101174001B6B7E4A43F0010313637C4B1B6B03F030
:101184000103FB60FB680023BB60784B1B6B774A51
:1011940043F002031363754B1B6B03F00203BB6044
:1011A400BB6800237B60714B1B6B704A43F00803E0
:1011B40013636E4B1B6B03F008037B607B68002298
:1011C40048F27F016A4803F01BFB002248F2121127
:1011D400684803F015FB002240F20441664803F01E
:1011E4000FFB002240F6FF71644803F009FB48F24C
:1011F4007F03FB6101233B6200237B620023BB620C
:1012040007F11C0319465A4803F04EF94FF478438A
:10121400FB614FF444133B6200237B6207F11C0320
:101224001946574803F040F90123FB614FF4441376
:101234003B6201237B6207F11C0319464D4803F00E
:1012440033F948F20213FB6101233B6200237B6202
:101254000023BB6207F11C031946464803F024F936
:101264001023FB6101233B6201237B620023BB62E9
:1012740007F11C0319463F4803F016F91023FB61DC
:1012840000233B6201237B6207F11C0319463C489F
:1012940003F00AF90423FB6101233B6202237B620E
:1012A4000023BB6207F11C031946334803F0FCF822
:1012B4004FF48063FB6101233B6200237B620023C4
:1012C400BB6207F11C0319462B4803F0EDF840F606
:1012D400FF73FB6101233B6200237B620023BB623B
:1012E40007F11C031946254803F0DEF84FF4007398
:1012F400FB6102233B6200237B620023BB620F235A
:10130400FB6207F11C0319461A4803F0CDF84FF4A9
:101314008063FB6100233B6200237B6207F11C03B3
:101324001946144803F0C0F84FF48063FB614FF48E
:1013340044133B6201237B6207F11C0319461048E6
:1013440003F0B2F800220021062002F07CFC062003
:1013540002F095FC00220021282002F074FC2820D1
:1013640002F08DFC00BF3037BD4680BD003802401E
:10137400001002400000024000040240000C024041
:101384000008024080B500AF124B134A1A60114B9B
:10139400124A5A600F4B00229A600E4B0022DA6008
:1013A4000C4B4FF480421A610A4B00225A61094BDC
:1013B40000229A61074B0022DA61064B00221A626E
:1013C400044803F069FA0346002B01D000F0B2F997
:1013D40000BF80BD7802002000540040A0860100B8
:1013E40080B58AB000AF786007F1140300221A6058
:1013F4005A609A60DA601A617B681B68194A9342E2
:101404002BD100233B61184B1B6B174A43F002039B
:101414001363154B1B6B03F002033B613B69C02351
:101424007B611223BB610023FB6102233B62042323
:101434007B6207F1140319460C4803F035F80023C6
:10144400FB60094B1B6C084A43F400131364064BFE
:101454001B6C03F40013FB60FB6800BF2837BD4618
:1014640080BD00BF00540040003802400004024028
:1014740080B586B002AFFFF7DBFD01F019FD00F087
:101484008BF8FFF73DFEFFF7FDFDFFF7D1F800F005
:1014940023FD00F0B9FD00F09FFE00F051F900F0CB
:1014A400BBF900F083F900F0CBFCFFF76BFF0DF004
:1014B4003FF901F0F5FA00F03FFE2E4807F02AFB51
:1014C4002D4807F027FB2D4807F024FB2C4807F094
:1014D40021FB2C4807F01EFB2B4A3B1D07CA03C304
:1014E4001A800021244807F0DFFB0421224807F07A
:1014F400DBFB0821204807F0D7FB0C211E4807F02E
:10150400D3FB00211D4807F0CFFB04211B4807F043
:10151400CBFB0821194807F0C7FB0C21174807F03B
:10152400C3FB0421174807F0BFFB0821154807F047
:10153400BBFB07221549164801F074FE391D4FF60E
:10154400FF730A22134806F076FD391D4FF6FF7328
:101554000A22104806F0ABFE3A1D391D4FF6FF7300
:1015640000930A230B4806F0B3FFFFF797FAFFF73F
:101574004FFDFCE71C04002064040020AC040020A0
:10158400F40400203C050020E8F20008E8010020F3
:101594003C010020CC02002080B594B000AF07F1DC
:1015A4001C033422002118460DF072FE07F10803D3
:1015B40000221A605A609A60DA601A6100237B6024
:1015C400294B1B6C284A43F080531364264B1B6C35
:1015D40003F080537B607B6800233B60234B1B68D4
:1015E40023F44043214A43F4804313601F4B1B6898
:1015F40003F440433B603B680123FB614FF48033B9
:101604003B6202237B634FF48003BB630623FB63CB
:1016140048233B6402237B640323BB640223FB64EF
:1016240007F11C03184606F0DFF90346002B01D02E
:1016340000F080F80F23BB600323FB6000233B61B1
:101644004FF480537B610023BB6107F1080302213F
:10165400184605F0A9FB0346002B01D000F06AF8F8
:1016640000BF5037BD4680BD0038024000700040C6
:1016740080B582B000AF78607B681B68234A9342D0
:1016840001D101F037FC7B681B68B3F1804F29D18D
:101694001F4B1B68002B03D002211E4803F0C9F81E
:1016A4001D4B1B68002B03D010211A4803F0C1F80E
:1016B4001A4B1B68002B03D08021164803F0B9F89D
:1016C400174B1B68002B04D04FF40071114803F032
:1016D400B0F8144B1B68002B04D04FF4004112489F
:1016E40003F0A7F87B681B68104A934209D1104B9A
:1016F4001B78002B0CBF01230023DBB21A460C4BD2
:101704001A7000BF0837BD4680BD00BF000001400D
:1017140084050020000C0240880500208C05002070
:10172400900500209405002000100240000C0040A9
:101734000600002080B400AF72B600BFFEE70000D0
:1017440080B500AF174B184A1A60164B4FF48272DB
:101754005A60144B00229A60124B0022DA60114B3B
:1017640000221A610F4B00225A610E4B4FF4007293
:101774009A610C4B3022DA610A4B00221A62094B3F
:1017840000225A62074B00229A62064B0A22DA624E
:10179400044806F0C7FB0346002B01D0FFF7CAFF3D
:1017A40000BF80BDCC0200200030014080B500AFF6
:1017B400174B184A1A60164B4FF482725A60144B36
:1017C40000229A60124B0022DA60114B02221A6145
:1017D4000F4B01225A610E4B4FF400729A610C4B6D
:1017E4003022DA610A4B00221A62094B00225A6243
:1017F400074B00229A62064B0A22DA62044806F07A
:1018040091FB0346002B01D0FFF794FF00BF80BD7E
:1018140024030020003C004080B500AF174B184A59
:101824001A60164B4FF482725A60144B00229A606D
:10183400124B0022DA60114B00221A610F4B002276
:101844005A610E4B4FF400729A610C4B0022DA611C
:101854000A4B00221A62094B00225A62074B0022EB
:101864009A62064B0A22DA62044806F05BFB0346DE
:10187400002B01D0FFF75EFF00BF80BD7C0300207A
:101884000034014080B58EB000AF786007F12403C6
:1018940000221A605A609A60DA601A617B681B68D9
:1018A4004B4A93422CD100233B624A4B5B6C494A1E
:1018B40043F480535364474B5B6C03F480533B62A3
:1018C4003B6A0023FB61434B1B6B424A43F0010319
:1018D4001363404B1B6B03F00103FB61FB69E023C3
:1018E4007B620223BB620023FB6203233B63052369
:1018F4007B6307F124031946374802F0D5FD63E002
:101904007B681B68354A93422CD10023BB61314B61
:101914001B6C304A43F4004313642E4B1B6C03F4DA
:101924000043BB61BB6900237B612A4B1B6B294AC3
:1019340043F002031363274B1B6B03F002037B6129
:101944007B6938237B620223BB620023FB6203238F
:101954003B6306237B6307F124031946204802F006
:10196400A3FD31E07B681B681E4A93422CD10023FF
:101974003B61184B5B6C174A43F400535364154B9B
:101984005B6C03F400533B613B690023FB60114B28
:101994001B6B104A43F0100313630E4B1B6B03F0D5
:1019A4001003FB60FB684FF4E0437B620223BB62DD
:1019B4000023FB6203233B6305237B6307F12403BA
:1019C4001946094802F070FD00BF3837BD4680BD96
:1019D400003001400038024000000240003C00405A
:1019E40000040240003401400010024080B483B07F
:1019F40000AF00237B60104B5B6C0F4A43F48043C1
:101A040053640D4B5B6C03F480437B607B68002361
:101A14003B60094B1B6C084A43F080531364064B2C
:101A24001B6C03F080533B603B6800BF0C37BD4622
:101A34005DF8047B704700BF0038024080B58CB06D
:101A440000AF78600023BB6200237B620023BB608D
:101A54002E4B5B6C2D4A43F0010353642B4B5B6CA0
:101A640003F00103BB60BB6807F10C0207F110032C
:101A74001146184605F0B2FA05F09CFAB862BB6A42
:101A8400234AA2FB03239B0C013B7B62214B224A8A
:101A94001A60204B40F2E732DA601E4A7B6A5360D8
:101AA4001C4B00221A611B4B00229A60194B002226
:101AB4009A61184806F0DEFF034687F82F3097F83E
:101AC4002F30002B1BD1134807F024F8034687F866
:101AD4002F3097F82F30002B11D1192002F0CFF8B6
:101AE4007B680F2B08D800227968192002F0ABF824
:101AF4000A4A7B68136002E0012387F82F3097F8C5
:101B04002F3018463037BD4680BD00BF0038024034
:101B140083DE1B43D403002000000140100000209A
:101B240080B400AFFEE780B400AFFEE780B400AF3E
:101B3400FEE780B400AFFEE780B400AFFEE780B4F8
:101B440000AF00BFBD465DF8047B704780B400AFB2
:101B540000BFBD465DF8047B704780B400AF00BF92
:101B6400BD465DF8047B704780B400AF00BFBD463E
:101B74005DF8047B704780B500AF012002F074FE6D
:101B840000BF80BD80B500AF024802F023FA00BF59
:101B940080BD00BFDC05002080B500AF024802F024
:101BA40019FA00BF80BD00BF3C06002080B500AF1D
:101BB400024801F026FA00BF80BD00BF3C010020AE
:101BC40080B500AF024807F037F900BF80BD00BF01
:101BD400D403002080B500AF024807F02DF900BF00
:101BE40080BD00BF1C04002080B500AF024807F090
:101BF40023F900BF80BD00BF6404002080B500AF9E
:101C0400024807F019F900BF80BD00BFAC040020F2
:101C140080B500AF024808F0B7F800BF80BD00BF30
:101C24009805002080B500AF4FF4806002F01CFEE0
:101C34004FF4006002F018FE4FF4805002F014FEDE
:101C44004FF4005002F010FE4FF4804002F00CFEFE
:101C54004FF4004002F008FE00BF80BD80B500AF25
:101C6400024807F0E9F800BF80BD00BF3C05002032
:101C740080B500AF024807F0DFF800BF80BD00BFA9
:101C84003C05002080B500AF024807F0D5F800BF3E
:101C940080BD00BF3C05002080B500AF024807F0BE
:101CA400CBF800BF80BD00BF3C05002080B500AF6D
:101CB400024807F0C1F800BF80BD00BFF404002053
:101CC40080B500AF024802F085F900BF80BD00BFB7
:101CD4008401002080B500AF024803F0F3FE00BF8A
:101CE40080BD00BF801B002080B582B000AF0346DA
:101CF400FB80FB88B3F5806F0FD14FF480614448BB
:101D040002F066FD0346002B0CBF01230023DBB267
:101D14001A4604213F4802F073FDFB88B3F5006FB7
:101D24000FD14FF400613A4802F052FD0346002BF4
:101D34000CBF01230023DBB21A460421354802F00C
:101D44005FFDFB88B3F5805F0FD14FF480513048BD
:101D540002F03EFD0346002B0CBF01230023DBB23F
:101D64001A4604212B4802F04BFDFB88B3F5804F43
:101D74000FD14FF48041264802F02AFD0346002B80
:101D84000CBF01230023DBB21A460421214802F0D0
:101D940037FDFB88B3F5004F0FD14FF400411C48C9
:101DA40002F016FD0346002B0CBF01230023DBB217
:101DB4001A460421174802F023FDFB88012B0ED19B
:101DC4000121154802F004FD0346002B0CBF01233A
:101DD4000023DBB21A4604210E4802F011FDFB88F1
:101DE400B3F5005F0FD14FF40051094802F0F0FC45
:101DF4000346002B0CBF01230023DBB21A46042147
:101E0400044802F0FDFC00BF0837BD4680BD00BF9A
:101E140000080240000402400000024080B400AF09
:101E2400064BD3F88830054A43F47003C2F888306F
:101E340000BFBD465DF8047B704700BF00ED00E0C5
:101E440080B586B000AF07F1080300221A605A601B
:101E54009A60DA603B4600221A605A601D4B4FF0CC
:101E640080421A601B4B47225A601A4B00229A6028
:101E7400184B3122DA60174B00221A61154B0022ED
:101E84009A61144806F0F6FD0346002B01D0FFF7D3
:101E940051FC4FF48053BB6007F1080319460D4809
:101EA40007F094F90346002B01D0FFF743FC00230D
:101EB4003B6000237B603B461946064807F086FDDD
:101EC4000346002B01D0FFF735FC00BF1837BD4691
:101ED40080BD00BF1C04002080B58EB000AF07F1A8
:101EE400280300221A605A609A60DA6007F120031E
:101EF40000221A605A603B1D00221A605A609A60E0
:101F0400DA601A615A619A613D4B3E4A1A603C4B51
:101F140040F2CF225A603A4B00229A60384B642236
:101F2400DA60374B00221A61354B00229A6134483B
:101F340006F0A0FD0346002B01D0FFF7FBFB4FF496
:101F44008053BB6207F1280319462D4807F03EF978
:101F54000346002B01D0FFF7EDFB294806F04AFEAB
:101F64000346002B01D0FFF7E5FB00233B6200236F
:101F74007B6207F120031946214807F027FD034639
:101F8400002B01D0FFF7D6FB60237B600023BB60EE
:101F94000023FB6000237B613B1D00221946184887
:101FA40007F052F80346002B01D0FFF7C3FB3B1D9B
:101FB40004221946124807F047F80346002B01D0C3
:101FC400FFF7B8FB3B1D082219460D4807F03CF803
:101FD4000346002B01D0FFF7ADFB3B1D0C22194635
:101FE400074807F031F80346002B01D0FFF7A2FBA6
:101FF400034800F053FA00BF3837BD4680BD00BF28
:10200400640400200004004080B58EB000AF07F1E6
:10201400280300221A605A609A60DA6007F12003EC
:1020240000221A605A603B1D00221A605A609A60AE
:10203400DA601A615A619A613D4B3E4A1A603C4B20
:1020440040F2CF225A603A4B00229A60384B642205
:10205400DA60374B00221A61354B00229A6134480A
:1020640006F008FD0346002B01D0FFF763FB4FF495
:102074008053BB6207F1280319462D4807F0A6F8E0
:102084000346002B01D0FFF755FB294806F0B2FDAB
:102094000346002B01D0FFF74DFB00233B620023D6
:1020A4007B6207F120031946214807F08FFC0346A1
:1020B400002B01D0FFF73EFB60237B600023BB6055
:1020C4000023FB6000237B613B1D00221946184856
:1020D40006F0BAFF0346002B01D0FFF72BFB3B1D94
:1020E40004221946124806F0AFFF0346002B01D024
:1020F400FFF720FB3B1D082219460D4806F0A4FFFC
:102104000346002B01D0FFF715FB3B1D0C2219469B
:10211400074806F099FF0346002B01D0FFF70AFB9E
:10212400034800F0BBF900BF3837BD4680BD00BF8F
:10213400AC0400200008004080B586B000AF07F171
:10214400080300221A605A609A60DA603B46002253
:102154001A605A601D4B1E4A1A601C4B41F61F42FE
:102164005A601A4B00229A60184B1A4ADA60174BCD
:1021740000221A61154B00229A61144806F07AFC79
:102184000346002B01D0FFF7D5FA4FF48053BB6010
:1021940007F1080319460D4807F018F80346002B09
:1021A40001D0FFF7C7FA00233B6000237B603B4666
:1021B4001946064807F00AFC0346002B01D0FFF736
:1021C400B9FA00BF1837BD4680BD00BFF404002033
:1021D400000C0040A086010080B596B000AF07F166
:1021E400480300221A605A609A60DA6007F14003DB
:1021F40000221A605A6007F1240300221A605A6010
:102204009A60DA601A615A619A613B1D20220021AA
:1022140018460DF03DF8444B444A1A60424B40F2D4
:10222400CF225A60404B00229A603F4B6322DA600F
:102234003D4B00221A613C4B00225A613A4B00226A
:102244009A61394806F016FC0346002B01D0FFF7CB
:1022540071FA4FF48053BB6407F1480319463248BE
:1022640006F0B4FF0346002B01D0FFF763FA2E48B3
:1022740006F0C0FC0346002B01D0FFF75BFA0023F5
:102284003B6400237B6407F140031946264807F0AA
:102294009DFB0346002B01D0FFF74CFA60237B62C1
:1022A4000023BB620023FB6200233B6300237B63A8
:1022B4000023BB630023FB6307F1240304221946B4
:1022C400194806F0C1FE0346002B01D0FFF732FA8D
:1022D40007F1240308221946134806F0B5FE034605
:1022E400002B01D0FFF726FA00237B600023BB609C
:1022F4000023FB6000233B6100237B614FF4005308
:10230400BB6100233B623B1D1946074807F0DAFB1B
:102314000346002B01D0FFF70DFA034800F0BEF886
:1023240000BF5837BD4680BD3C0500200004014075
:1023340080B588B000AF78607B681B68B3F1804FCC
:1023440016D10023FB61504B1B6C4F4A43F0010331
:1023540013644D4B1B6C03F00103FB61FB6900220A
:1023640000211C2001F06FFC1C2001F088FC86E099
:102374007B681B68454A934216D10023BB61424BDC
:102384001B6C414A43F0020313643F4B1B6C03F084
:102394000203BB61BB69002200211D2001F053FC34
:1023A4001D2001F06CFC6AE07B681B68384A93428C
:1023B40016D100237B61344B1B6C334A43F0040376
:1023C4001364314B1B6C03F004037B617B690022B3
:1023D40000211E2001F037FC1E2001F050FC4EE0CD
:1023E4007B681B682B4A934216D100233B61264B22
:1023F4001B6C254A43F008031364234B1B6C03F046
:1024040008033B613B6900220021322001F01BFCE0
:10241400322001F034FC32E07B681B681E4A934290
:102424002DD10023FB60184B5B6C174A43F0020369
:102434005364154B5B6C03F00203FB60FB680022E2
:1024440000212B2001F0FFFB2B2001F018FC0022BF
:1024540000212C2001F0F7FB2C2001F010FC0022BD
:1024640000212D2001F0EFFB2D2001F008FC0022BB
:1024740000212E2001F0E7FB2E2001F000FC00BF1C
:102484002037BD4680BD00BF003802400004004034
:1024940000080040000C00400004014080B58AB0F0
:1024A40000AF786007F1140300221A605A609A6042
:1024B400DA601A617B681B68374A93421FD1002394
:1024C4003B61364B1B6B354A43F004031363334BB8
:1024D4001B6B03F004033B613B694FF470737B6136
:1024E4000223BB610023FB6100233B6202237B6266
:1024F40007F1140319462A4801F0D6FF48E07B6827
:102504001B68284A93421FD10023FB60234B1B6B9B
:10251400224A43F008031363204B1B6B03F00803A8
:10252400FB60FB684FF470437B610223BB610023B3
:10253400FB6100233B6202237B6207F1140319460B
:10254400194801F0B1FF23E07B681B68174A9342E6
:102554001ED10023BB60114B1B6B104A43F00203D6
:1025640013630E4B1B6B03F00203BB60BB684FF499
:1025740040437B610223BB610023FB6100233B6278
:1025840003237B6207F114031946094801F08CFF09
:1025940000BF2837BD4680BD00040040003802401B
:1025A4000008024000080040000C02400004014002
:1025B4000004024080B58CB000AF3B4683E80300C2
:1025C4004F4A07F1280392E8030018600433197096
:1025D4004C4A07F1200392E8030018600433197091
:1025E400494A07F1180392E803001860043319708C
:1025F400464A07F1100392E8030018600433197087
:10260400434A07F1080392E8030018600433197081
:102614003B68B9880022184602F0F2F807F1280155
:102624004FF4805305223B4805F005FD3B68B9880B
:102634000122184602F0E4F8012000F07BFC3B681C
:10264400B9880022184602F0DBF807F120014FF4A4
:10265400805305222F4805F0EEFC3B68B98801221F
:10266400184602F0CDF8012000F064FC3B68B988FC
:102674000022184602F0C4F807F118014FF4805301
:102684000522244805F0D7FC3B68B9880122184686
:1026940002F0B6F8012000F04DFC3B68B988002236
:1026A400184602F0ADF807F110014FF480530522EB
:1026B400184805F0C0FC3B68B9880122184602F0AE
:1026C4009FF8012000F036FC3B68B98800221846C8
:1026D40002F096F807F108014FF4805305220D48E3
:1026E40005F0A9FC3B68B9880122184602F088F875
:1026F400012000F01FFC00BF3037BD4680BD00BF85
:10270400F4F20008FCF2000804F300080CF30008DB
:1027140014F300082403002080B582B000AF064BF8
:102724003B600423BB803B4693E80300FFF742FF72
:1027340000BF0837BD4680BD0010024080B582B09E
:1027440000AF064B3B600823BB803B4693E8030085
:10275400FFF730FF00BF0837BD4680BD00100240C0
:1027640080B582B000AF064B3B601023BB803B4674
:1027740093E80300FFF71EFF00BF0837BD4680BD86
:102784000010024080B582B000AF064B3B600123CD
:10279400BB803B4693E80300FFF70CFF00BF0837FC
:1027A400BD4680BD0010024080B582B000AF064B2C
:1027B4003B600223BB803B4693E80300FFF7FAFE2D
:1027C40000BF0837BD4680BD0010024080B500AF91
:1027D400FFF7A2FFFFF7B2FFFFF7C2FFFFF7D2FF39
:1027E400FFF7E2FF00BF80BD80B500AF1C4BB3F91B
:1027F4001C30002B06D101224FF40041194801F08E
:10280400FFFF2BE0164BB3F91C30002B11DD002227
:102814004FF40041134801F0F3FF01220121124853
:1028240001F0EEFF0E4BB3F91C301A460F4B1A6041
:1028340014E000224FF400410A4801F0E1FF0022B5
:102844000121094801F0DCFF054BB3F91C30002BD2
:10285400B8BF5B429BB21A46044B1A6000BF80BDEE
:102864004C02002000000240000C024084050020BD
:1028740080B500AF1B4BB3F91E30002B05D10122EC
:102884000421194801F0BCFF29E0164BB3F91E30AE
:10289400002B10DD00220421134801F0B1FF0122B6
:1028A4000821114801F0ACFF0E4BB3F91E301A4653
:1028B4000E4B1A6013E0002204210B4801F0A0FF24
:1028C40000220821084801F09BFF064BB3F91E3093
:1028D400002BB8BF5B429BB21A46044B1A6000BF80
:1028E40080BD00BF4C020020000C0240880500207F
:1028F40080B500AF1B4BB3F92030002B05D101226A
:102904002021194801F07CFF29E0164BB3F920304F
:10291400002B10DD00222021134801F071FF012259
:102924004021114801F06CFF0E4BB3F920301A46D8
:102934000E4B1A6013E0002220210B4801F060FFC7
:1029440000224021084801F05BFF064BB3F9203018
:10295400002BB8BF5B429BB21A46044B1A6000BFFF
:1029640080BD00BF4C020020000C02408C050020FA
:1029740080B500AF1D4BB3F92230002B06D10122E4
:102984004FF400611A4801F03BFF2DE0174BB3F9F7
:102994002230002B12DD00224FF40061144801F0B4
:1029A4002FFF01224FF48061114801F029FF0F4BE2
:1029B400B3F922301A460F4B1A6015E000224FF487
:1029C40000610B4801F01CFF00224FF480610848AD
:1029D40001F016FF054BB3F92230002BB8BF5B4260
:1029E4009BB21A46034B1A6000BF80BD4C02002004
:1029F400000C02409005002080B500AF1D4BB3F9D8
:102A04002430002B06D101224FF480711A4801F0C2
:102A1400F7FE2DE0174BB3F92430002B12DD002212
:102A24004FF48071144801F0EBFE01224FF48061F1
:102A3400124801F0E5FE0F4BB3F924301A46104B4F
:102A44001A6015E000224FF480710B4801F0D8FEA3
:102A540000224FF48061094801F0D2FE054BB3F91E
:102A64002430002BB8BF5B429BB21A46044B1A6059
:102A740000BF80BD4C020020000C02400004024054
:102A84009405002080B500AFFFF7AEFEFFF7F0FE1F
:102A9400FFF72EFFFFF76CFFFFF7AEFF00BF80BD0F
:102AA40080B500AF114B124A1A60104B4FF4E1325B
:102AB4005A600E4B00229A600C4B0022DA600B4BDA
:102AC40000221A61094B0C225A61084B00229A61B8
:102AD400064B0022DA61054807F05AF80346002B3A
:102AE40001D0FEF727FE00BF80BD00BF980500207F
:102AF4000044004080B58AB000AF786007F1140349
:102B040000221A605A609A60DA601A617B681B6856
:102B14004B4A934240F0908000233B61494B1B6C2D
:102B2400484A43F400331364464B1B6C03F40033EC
:102B34003B613B690023FB60424B1B6B414A43F002
:102B4400010313633F4B1B6B03F00103FB60FB6842
:102B54000C237B610223BB610023FB6103233B62E3
:102B640007237B6207F114031946374801F09CFCE4
:102B7400364B374A1A60354B4FF000625A60334B7C
:102B840000229A60314B0022DA60304B4FF48062AD
:102B94001A612E4B00225A612C4B00229A612B4B56
:102BA4000022DA61294B00221A62284B00225A6261
:102BB400264801F077F80346002B01D0FEF7BAFD52
:102BC4007B68224A9A63214A7B689363214B224A99
:102BD4001A60204B4FF000625A601E4B40229A60EC
:102BE4001C4B0022DA601B4B4FF480621A61194BB4
:102BF40000225A61174B00229A61164B0022DA61B7
:102C0400144B00221A62134B00225A62114801F03D
:102C140049F80346002B01D0FEF78CFD7B680D4A72
:102C24005A630C4A7B68936300220021262001F03A
:102C34000AF8262001F023F800BF2837BD4680BDDE
:102C4400004400400038024000000240DC0500203F
:102C5400886002403C060020A060024080B483B03B
:102C640000AF78607B680B4A93420CD10A4B012277
:102C74001A700A4B1B78002B0CBF01230023DBB214
:102C84001A46064B1A7000BF0C37BD465DF8047B2C
:102C9400704700BF9805002007000020E5010020D0
:102CA40080B483B000AF78607B68064A934202D157
:102CB400054B01221A7000BF0C37BD465DF8047B3A
:102CC400704700BF980500200800002080B586B03A
:102CD40002AF0346FB7107F10F02F91D4FF47A733B
:102CE40000930123034805F0F3FBFB7B18461037E0
:102CF400BD4680BDCC02002080B582B000AF034643
:102D0400FB71F91D4FF47A730122054805F093F91C
:102D14004FF44870FDF7FCFD00BF0837BD4680BD89
:102D2400CC02002080B582B000AF0A20FDF7F0FD90
:102D3400FF20FFF7CBFF0346FB71FB7918460837EA
:102D4400BD4680BD80B582B000AF0346FB71012251
:102D540010210D4801F054FDC820FDF7D9FD0022D3
:102D64001021094801F04CFDF91D4FF47A7301223A
:102D7400064805F060F940F2A460FDF7C9FD00BF04
:102D84000837BD4680BD00BF00000240CC020020D1
:102D940080B500AF01221021024801F031FD00BFCF
:102DA40080BD00BF0000024080B582B000AF10219A
:102DB400074801F00DFD0346002B0CBF012300233F
:102DC400DBB2FB71FB7918460837BD4680BD00BFF6
:102DD4000008024080B582B000AF4FF4FA7000F0F2
:102DE400A9F80620FFF7AEFF5520FFF785FFFFF790
:102DF40099FF0346FB71FFF7CBFFFB79AA2B01D0A8
:102E0400AA2314E01520FFF79DFF0620FFF774FFA7
:102E14001420FDF77DFDFFF785FF0346FB71FFF7E7
:102E2400B7FFFB79512B01D1142300E0FA23184694
:102E34000837BD4680BD80B582B000AFFDF7E8FB22
:102E44000346142B03D10023FB71FB7902E0012319
:102E5400FB71FB7918460837BD4680BDDFF834D0D6
:102E64000D480E490E4A002302E0D458C4500433DE
:102E7400C4188C42F9D30B4A0B4C002301E01360B5
:102E84000432A242FBD3FEF7C9FF0CF0DDF9FEF7D2
:102E9400EFFA7047D8FF012000000020180100203D
:102EA4009CF3000818010020AC220020FEE700007B
:102EB40080B500AF0E4B1B680D4A43F400731360DA
:102EC4000B4B1B680A4A43F480631360084B1B686E
:102ED400074A43F480731360032000F0A9FE0F2017
:102EE400FEF7ACFDFEF782FD0023184680BD00BF4F
:102EF400003C024080B400AF064B1B781A46064BD8
:102F04001B681344044A136000BFBD465DF8047B8C
:102F1400704700BF140000209C06002080B400AF5E
:102F2400034B1B681846BD465DF8047B704700BF21
:102F34009C06002080B584B000AF7860FFF7EEFFF8
:102F4400B8607B68FB60FB68B3F1FF3F05D00A4BB8
:102F54001B781A46FB681344FB6000BFFFF7DEFFD3
:102F64000246BB68D31AFA689A42F7D800BF00BF7A
:102F74001037BD4680BD00BF1400002080B584B06A
:102F840000AF78600023FB737B68002B01D1012321
:102F940033E07B681B6C002B09D17868FDF7EEFBEE
:102FA4007B6800225A647B68002283F83C207B689B
:102FB4001B6C03F01003002B18D17B681B6C23F4EB
:102FC400885323F0020343F002027B681A64786892
:102FD40000F0E2FB7B6800225A647B681B6C23F0E0
:102FE400030343F001027B681A6401E00123FB73CD
:102FF4007B68002283F83C20FB7B18461037BD46D3
:1030040080BD80B586B000AF786000237B6100236B
:103014003B617B681B681B68FB607B681B685B68A3
:10302400BB60FB6803F002037B61BB6803F0200311
:103034003B617B69002B49D03B69002B46D07B6800
:103044001B6C03F01003002B05D17B681B6C43F44D
:1030540000727B681A647B681B689B6803F04053AA
:10306400002B2BD17B681B7E002B27D17B681B6830
:10307400DB6A03F47003002B06D07B681B689B6833
:1030840003F48063002B19D17B681B685A687B6842
:103094001B6822F020025A607B681B6C23F4807248
:1030A4007B681A647B681B6C03F48053002B05D186
:1030B4007B681B6C43F001027B681A647868FDF737
:1030C400F7FB7B681B686FF012021A60FB6803F061
:1030D40004037B61BB6803F080033B617B69002BC5
:1030E40057D03B69002B54D07B681B6C03F0100352
:1030F400002B05D17B681B6C43F400527B681A6477
:103104007B681B689B6803F44013002B39D17B68F0
:103114001B689B6B03F44013002B06D07B681B6871
:103124009B6803F48063002B2BD17B681B685B686E
:1031340003F48063002B24D17B681B689B6803F035
:103144004053002B1DD17B681B7E002B19D17B685B
:103154001B685A687B681B6822F080025A607B688F
:103164001B6C23F480527B681A647B681B6C03F429
:103174008073002B05D17B681B6C43F001027B68D4
:103184001A64786800F086FC7B681B686FF00C0298
:103194001A60FB6803F001037B61BB6803F0400322
:1031A4003B617B69002B17D03B69002B14D07B68F3
:1031B4001B681B6803F00103012B0DD17B681B6C9A
:1031C40043F480327B681A64786800F09FF97B6866
:1031D4001B686FF001021A60FB6803F020037B6137
:1031E400BB6803F080633B617B69002B15D03B69AE
:1031F400002B12D07B685B6C43F002027B685A643C
:103204007B681B686FF020021A60786800F088F908
:103214007B681B686FF020021A6000BF1837BD4638
:1032240080BD000080B586B000AFF860B9607A60F8
:1032340000233B61FB6893F83C30012B01D102234E
:10324400E9E0FB68012283F83C20FB681B689B686B
:1032540003F00103012B18D0FB681B689A68FB6814
:103264001B6842F001029A606D4B1B686D4AA2FB19
:1032740003239A0C13465B0013443B6102E03B6951
:10328400013B3B613B69002BF9D1FB681B689B68E0
:1032940003F48073B3F5807F07D1FB681B689A68D9
:1032A400FB681B6822F480729A60FB681B689B6849
:1032B40003F00103012B40F0A180FB681B6C23F495
:1032C400E06323F0010343F48072FB681A64FB6833
:1032D4001B685B6803F48063002B07D0FB681B6CDE
:1032E40023F4405343F48052FB681A64FB681B6C5C
:1032F40003F48053B3F5805F06D1FB685B6C23F065
:103304000602FB685A6402E0FB6800225A64FB6808
:10331400002283F83C20444B7B61FB689B6B434A4F
:10332400DA63FB689B6B424A1A64FB689B6B414AF5
:10333400DA64FB681B686FF022021A60FB681B6882
:103344005A68FB681B6842F080625A60FB681B681D
:103354009A68FB681B6842F480729A60FB68986BF9
:10336400FB681B684C331946BA687B6800F048FD5B
:103374007B695B6803F01F03002B2AD1FB681B6881
:103384002D4A934215D0FB681B682C4A934205D101
:10339400254B5B6803F01F03002B0AD0FB681B68F6
:1033A400274A934236D1204B5B6803F01003002B6D
:1033B40030D1FB681B689B6803F04053002B29D174
:1033C400FB681B689A68FB681B6842F080429A603D
:1033D40020E0FB681B68184A93421BD1FB681B68FA
:1033E4009B6803F04053002B14D1FB681B689A6858
:1033F400FB681B6842F080429A600BE0FB681B6C20
:1034040043F01002FB681A64FB685B6C43F0010232
:10341400FB685A64002318461837BD4680BD00BFB8
:103424000C00002083DE1B43002301409539000873
:103434004F3A00086B3A0008002001400021014087
:103444000022014080B584B000AF78600023FB7394
:103454007B6893F83C30012B01D1022348E07B6860
:10346400012283F83C207B681B689A687B681B6890
:1034740022F001029A607B681B689B6803F00103D9
:10348400002B30D17B681B689A687B681B6822F428
:1034940080729A607B689B6B93F83530DBB2022BA9
:1034A4000FD17B689B6B184600F002FD0346FB734B
:1034B400FB7B002B05D07B681B6C43F040027B68D0
:1034C4001A647B681B685A687B681B6822F08062F8
:1034D4005A607B681B6C23F4885323F0010343F088
:1034E40001027B681A647B68002283F83C20FB7B22
:1034F40018461037BD4680BD80B483B000AF7860F5
:1035040000BF0C37BD465DF8047B704780B483B0C0
:1035140000AF786000BF0C37BD465DF8047B704790
:1035240080B483B000AF786000BF0C37BD465DF84F
:10353400047B704780B485B000AF786039600023A5
:10354400BB607B6893F83C30012B01D1022313E16B
:103554007B68012283F83C203B681B68092B25D932
:103564007B681B68D9683B681B689BB21A46134684
:103574005B0013441E3B072202FA03F3DA437B6821
:103584001B680A40DA607B681B68D9683B689A68E4
:103594003B681B689BB2184603465B0003441E3B12
:1035A4009A407B681B680A43DA6022E07B681B68E8
:1035B40019693B681B689BB21A4613465B001344A7
:1035C400072202FA03F3DA437B681B680A401A6194
:1035D4007B681B6819693B689A683B681B689BB2E7
:1035E400184603465B0003449A407B681B680A4301
:1035F4001A613B685B68062B24D87B681B68596B8F
:103604003B685A6813469B001344053B1F2202FA89
:1036140003F3DA437B681B680A405A637B681B68C0
:10362400596B3B681B689BB218463B685A68134643
:103634009B001344053B00FA03F27B681B680A43B2
:103644005A634CE03B685B680C2B24D87B681B688E
:10365400196B3B685A6813469B001344233B1F2293
:1036640002FA03F3DA437B681B680A401A637B6837
:103674001B68196B3B681B689BB218463B685A6809
:1036840013469B001344233B00FA03F27B681B6838
:103694000A431A6323E07B681B68D96A3B685A684B
:1036A40013469B001344413B1F2202FA03F3DA43FF
:1036B4007B681B680A40DA627B681B68D96A3B68CE
:1036C4001B689BB218463B685A6813469B00134418
:1036D400413B00FA03F27B681B680A43DA62294B18
:1036E400FB607B681B68284A93420FD13B681B68C8
:1036F400122B0BD1FB685B6823F40002FB685A6051
:10370400FB685B6843F48002FB685A607B681B6853
:103714001D4A93422BD13B681B681C4A934203D039
:103724003B681B68112B22D1FB685B6823F4800281
:10373400FB685A60FB685B6843F40002FB685A60EC
:103744003B681B68114A934211D1114B1B68114A03
:10375400A2FB03239A0C13469B0013445B00BB603B
:1037640002E0BB68013BBB60BB68002BF9D17B68FE
:10377400002283F83C20002318461437BD465DF828
:10378400047B704700230140002001401200001018
:103794000C00002083DE1B4380B485B000AF78604A
:1037A400794BFB60FB685B6823F44032FB685A602A
:1037B400FB685A687B685B681A43FB685A607B68DD
:1037C4001B685A687B681B6822F480725A607B68A5
:1037D4001B6859687B681B691A027B681B680A436B
:1037E4005A607B681B685A687B681B6822F04072C9
:1037F4005A607B681B6859687B689A687B681B6899
:103804000A435A607B681B689A687B681B6822F4C9
:1038140000629A607B681B6899687B68DA687B68D9
:103824001B680A439A607B689B6A584A934222D079
:103834007B681B689A687B681B6822F070629A60D8
:103844007B681B6899687B689A6A7B681B680A4373
:103854009A607B681B689A687B681B6822F04052F8
:103864009A607B681B6899687B68DA6A7B681B6866
:103874000A439A600FE07B681B689A687B681B6840
:1038840022F070629A607B681B689A687B681B6888
:1038940022F040529A607B681B689A687B681B68B8
:1038A40022F002029A607B681B6899687B681B7E21
:1038B4005A007B681B680A439A607B6893F820303F
:1038C400002B1BD07B681B685A687B681B6842F41A
:1038D40000625A607B681B685A687B681B6822F424
:1038E40060425A607B681B6859687B685B6A013B6D
:1038F4005A037B681B680A435A6007E07B681B68AD
:103904005A687B681B6822F400625A607B681B68F3
:10391400DA6A7B681B6822F47002DA627B681B68CF
:10392400D96A7B68DB69013B1A057B681B680A431B
:10393400DA627B681B689A687B681B6822F40072F1
:103944009A607B681B6899687B6893F830305A02E8
:103954007B681B680A439A607B681B689A687B686B
:103964001B6822F480629A607B681B6899687B6894
:103974005B699A027B681B680A439A6000BF14372C
:10398400BD465DF8047B7047002301400100000F31
:1039940080B584B000AF78607B689B6BFB60FB688C
:1039A4001B6C03F05003002B3CD1FB681B6C43F4ED
:1039B4000072FB681A64FB681B689B6803F0405341
:1039C400002B2BD1FB681B7E002B27D1FB681B68C7
:1039D400DB6A03F47003002B06D0FB681B689B684A
:1039E40003F48063002B19D1FB681B685A68FB68D9
:1039F4001B6822F020025A60FB681B6C23F480725F
:103A0400FB681A64FB681B6C03F48053002B05D11C
:103A1400FB681B6C43F00102FB681A64F868FCF74E
:103A240047FF0EE0FB681B6C03F01003002B03D070
:103A3400F868FFF775FD04E0FB689B6BDB6C786846
:103A4400984700BF1037BD4680BD80B584B000AF35
:103A540078607B689B6BFB60F868FFF74DFD00BFE7
:103A64001037BD4680BD80B584B000AF78607B68F8
:103A74009B6BFB60FB6840221A64FB685B6C43F041
:103A84000402FB685A64F868FFF74AFD00BF103768
:103A9400BD4680BD80B483B000AF786000BF0C37F2
:103AA400BD465DF8047B704780B485B000AF786094
:103AB4007B6803F00703FB600C4BDB68BB60BA68F0
:103AC4004FF6FF031340BB60FB681A02BB68134345
:103AD40043F0BF6343F40033BB60044ABB68D36064
:103AE40000BF1437BD465DF8047B704700ED00E06D
:103AF40080B400AF044BDB681B0A03F007031846CD
:103B0400BD465DF8047B704700ED00E080B483B0EF
:103B140000AF0346FB7197F90730002B0BDBFB79F1
:103B240003F01F02074997F907305B09012000FAE7
:103B340002F241F8232000BF0C37BD465DF8047B38
:103B4400704700BF00E100E080B483B000AF0346DB
:103B54003960FB7197F90730002B0ADB3B68DAB256
:103B64000C4997F907301201D2B20B4483F80023B1
:103B74000AE03B68DAB20849FB7903F00F03043B1F
:103B84001201D2B20B441A7600BF0C37BD465DF861
:103B9400047B704700E100E000ED00E080B489B0F0
:103BA40000AFF860B9607A60FB6803F00703FB615B
:103BB400FB69C3F10703042B28BF0423BB61FB6922
:103BC4000433062B02D9FB69033B00E000237B612D
:103BD4004FF0FF32BB6902FA03F3DA43BB681A40C1
:103BE4007B699A404FF0FF317B6901FA03F3D943B3
:103BF4007B680B40134318462437BD465DF8047BAD
:103C04007047000080B400AFBFF34F8F00BF064B76
:103C1400DB6803F4E0620449044B1343CB60BFF355
:103C24004F8F00BF00BFFDE700ED00E00400FA0580
:103C340080B582B000AF78607868FFF735FF00BFC9
:103C44000837BD4680BD80B586B000AF0346B96075
:103C54007A60FB7300237B61FFF74AFF78617A681F
:103C6400B9687869FFF79AFF024697F90F30114651
:103C74001846FFF769FF00BF1837BD4680BD80B501
:103C840082B000AF0346FB7197F907301846FFF77F
:103C94003DFF00BF0837BD4680BD80B500AFFFF7CC
:103CA400B1FF000080B586B000AF786000237B616F
:103CB400FFF734F938617B68002B01D1012399E0C7
:103CC4007B68022283F835207B68002283F8342045
:103CD4007B681B681A687B681B6822F001021A6003
:103CE4000FE0FFF71BF902463B69D31A052B08D9ED
:103CF4007B6820225A657B68032283F835200323DE
:103D040078E07B681B681B6803F00103002BE8D193
:103D14007B681B681B687B617A69384B13407B6145
:103D24007B685A687B689B681A437B68DB681A4324
:103D34007B681B691A437B685B691A437B689B69D0
:103D44001A437B68DB691A437B681B6A13437A69ED
:103D540013437B617B685B6A042B07D17B68DA6A57
:103D64007B681B6B13437A6913437B617B681B6815
:103D74007A691A607B681B685B697B617B6923F0E5
:103D840007037B617B685B6A7A6913437B617B68A9
:103D94005B6A042B17D17B689B6A7A6913437B6146
:103DA4007B68DB6A002B0ED0786800F001FB0346C9
:103DB400002B08D07B6840225A657B68012283F877
:103DC4003520012316E07B681B687A695A6178689C
:103DD40000F0B8FA0346FB607B68DB6D3F229A4033
:103DE400FB689A607B6800225A657B68012283F82D
:103DF4003520002318461837BD4680BD3F8010F09B
:103E040080B586B000AFF860B9607A603B6000238B
:103E1400FB75FB689B6D3B61FB6893F83430012BA9
:103E240001D1022340E0FB68012283F83420FB68BF
:103E340093F83530DBB2012B2FD1FB68022283F8D3
:103E44003520FB6800225A653B687A68B968F868CF
:103E540000F04AFAFB68DB6D3F229A403B699A60A6
:103E6400FB681B681A68FB681B6842F016021A603C
:103E7400FB681B6C002B07D0FB681B681A68FB6887
:103E84001B6842F008021A60FB681B681A68FB682A
:103E94001B6842F001021A6005E0FB68002283F807
:103EA40034200223FB75FB7D18461837BD4680BDC0
:103EB40080B584B000AF78607B689B6DFB60FFF7D2
:103EC4002DF8B8607B6893F83530DBB2022B08D04C
:103ED4007B6880225A657B68002283F834200123A2
:103EE40052E07B681B681A687B681B6822F0160224
:103EF4001A607B681B685A697B681B6822F0800221
:103F04005A617B681B6C002B03D17B689B6C002B74
:103F140007D07B681B681A687B681B6822F008025C
:103F24001A607B681B681A687B681B6822F00102B0
:103F34001A6013E0FEF7F2FF0246BB68D31A052BA2
:103F44000CD97B6820225A657B68032283F83520CC
:103F54007B68002283F83420032315E07B681B6808
:103F64001B6803F00103002BE4D17B68DB6D3F2267
:103F74009A40FB689A607B68012283F835207B684D
:103F8400002283F83420002318461037BD4680BD34
:103F940080B483B000AF78607B6893F83530DBB2CF
:103FA400022B04D07B6880225A6501230CE07B68D5
:103FB400052283F835207B681B681A687B681B68B8
:103FC40022F001021A60002318460C37BD465DF842
:103FD400047B704780B586B000AF78600023BB6077
:103FE4008E4B1B688E4AA2FB03239B0A7B617B6872
:103FF4009B6D3B613B691B68FB607B68DB6D082242
:104004009A40FB681340002B1AD07B681B681B681E
:1040140003F00403002B13D07B681B681A687B68C9
:104024001B6822F004021A607B68DB6D08229A4048
:104034003B699A607B685B6D43F001027B685A655B
:104044007B68DB6D01229A40FB681340002B12D081
:104054007B681B685B6903F08003002B0BD07B68D3
:10406400DB6D01229A403B699A607B685B6D43F08B
:1040740002027B685A657B68DB6D04229A40FB6808
:104084001340002B12D07B681B681B6803F00203EB
:10409400002B0BD07B68DB6D04229A403B699A604D
:1040A4007B685B6D43F004027B685A657B68DB6D5B
:1040B40010229A40FB681340002B43D07B681B6896
:1040C4001B6803F00803002B3CD07B68DB6D1022D7
:1040D4009A403B699A607B681B681B6803F48023E1
:1040E400002B18D07B681B681B6803F40023002B8B
:1040F40008D17B681B6C002B24D07B681B6C786810
:1041040098471FE07B689B6C002B1BD07B689B6CE3
:104114007868984716E07B681B681B6803F4807313
:10412400002B07D17B681B681A687B681B6822F028
:1041340008021A607B681B6C002B03D07B681B6C25
:10414400786898477B68DB6D20229A40FB681340AF
:10415400002B00F08F807B681B681B6803F0100342
:10416400002B00F087807B68DB6D20229A403B693E
:104174009A607B6893F83530DBB2052B36D17B68C7
:104184001B681A687B681B6822F016021A607B6839
:104194001B685A697B681B6822F080025A617B683D
:1041A4001B6C002B03D17B689B6C002B07D07B68B6
:1041B4001B681A687B681B6822F008021A607B6817
:1041C400DB6D3F229A403B699A607B68012283F849
:1041D40035207B68002283F834207B681B6D002B1C
:1041E4007ED07B681B6D7868984779E07B681B6894
:1041F4001B6803F48023002B1DD07B681B681B689D
:1042040003F40023002B0DD17B685B6C002B31D0B1
:104214007B685B6C786898472CE000BF0C0000203A
:10422400B5814E1B7B68DB6B002B23D07B68DB6B7B
:10423400786898471EE07B681B681B6803F48073EA
:10424400002B0FD17B681B681A687B681B6822F0FF
:1042540010021A607B68012283F835207B680022F3
:1042640083F834207B68DB6B002B03D07B68DB6B2B
:10427400786898477B685B6D002B32D07B685B6DF8
:1042840003F00103002B22D07B68052283F835203C
:104294007B681B681A687B681B6822F001021A603D
:1042A400BB680133BB607A699A4207D37B681B6899
:1042B4001B6803F00103002BF2D100E000BF7B6810
:1042C400012283F835207B68002283F834207B6840
:1042D400DB6C002B05D07B68DB6C7868984700E0CA
:1042E40000BF1837BD4680BD80B485B000AFF8600C
:1042F400B9607A603B60FB681B681A68FB681B68DE
:1043040022F480221A60FB681B683A685A60FB68D2
:104314009B68402B08D1FB681B687A689A60FB682D
:104324001B68BA68DA6007E0FB681B68BA689A60C1
:10433400FB681B687A68DA6000BF1437BD465DF815
:10434400047B704780B485B000AF78607B681B68DD
:10435400DBB2103B144AA2FB03231B09FB60134A84
:10436400FB6813441B781A467B68DA65FB68032BE9
:1043740009D97B681B6823F47F7323F003031A1D98
:104384007B689A6507E07B681B6823F47F7323F0DE
:1043940003037A6893657B689B6D18461437BD46A2
:1043A4005DF8047B704700BFABAAAAAA84F3000897
:1043B40080B485B000AF78600023FB737B689B6A90
:1043C400BB607B689B69002B1FD1BB68032B56D84D
:1043D40001A252F823F000BFED430008FF43000898
:1043E400ED430008834400087B68DB6A03F08073B4
:1043F400002B46D00123FB7343E07B68DB6AB3F1F7
:10440400C07F40D10123FB733DE07B689B69B3F51A
:10441400005F21D1BB68032B37D801A252F823F0E7
:10442400354400083B440008354400084D44000866
:104434000123FB7330E07B68DB6A03F08073002B9D
:1044440025D00123FB7322E07B68DB6AB3F1C07FD4
:104454001FD10123FB731CE0BB68022B03D9BB688B
:10446400032B03D018E00123FB7315E07B68DB6AA0
:1044740003F08073002B0ED00123FB730BE000BF0D
:104484000AE000BF08E000BF06E000BF04E000BF90
:1044940002E000BF00E000BFFB7B18461437BD46B6
:1044A4005DF8047B704700BF80B489B000AF7860CA
:1044B400396000237B6100233B610023BB6100233F
:1044C400FB6165E10122FB6902FA03F37B613B684E
:1044D4001B687A6913403B613A697B699A4240F0F0
:1044E40054813B685B6803F00303012B05D03B68F0
:1044F4005B6803F00303022B30D17B689B68BB61CC
:10450400FB695B00032202FA03F3DB43BA6913403D
:10451400BB613B68DA68FB695B0002FA03F3BA69C2
:104524001343BB617B68BA699A607B685B68BB6153
:104534000122FB6902FA03F3DB43BA691340BB614E
:104544003B685B681B0903F00102FB6902FA03F391
:10455400BA691343BB617B68BA695A603B685B689C
:1045640003F00303032B17D07B68DB68BB61FB6993
:104574005B00032202FA03F3DB43BA691340BB6115
:104584003B689A68FB695B0002FA03F3BA69134358
:10459400BB617B68BA69DA603B685B6803F003035C
:1045A400022B23D1FB69DA087B68083253F82230E6
:1045B400BB61FB6903F007039B000F2202FA03F3BC
:1045C400DB43BA691340BB613B681A69FB6903F0BA
:1045D40007039B0002FA03F3BA691343BB61FB6947
:1045E400DA087B680832B96943F822107B681B68D3
:1045F400BB61FB695B00032202FA03F3DB43BA6984
:104604001340BB613B685B6803F00302FB695B001A
:1046140002FA03F3BA691343BB617B68BA691A608F
:104624003B685B6803F44033002B00F0AE8000234A
:10463400FB605D4B5B6C5C4A43F4804353645A4BB0
:104644005B6C03F48043FB60FB68584AFB699B087E
:10465400023352F82330BB61FB6903F003039B0070
:104664000F2202FA03F3DB43BA691340BB617B6890
:104674004F4A934225D07B684E4A93421FD07B68B1
:104684004D4A934219D07B684C4A934213D07B68BD
:104694004B4A93420DD07B684A4A934207D07B68C9
:1046A400494A934201D106230CE007230AE005237B
:1046B40008E0042306E0032304E0022302E00123CC
:1046C40000E00023FA6902F0030292009340BA6901
:1046D4001343BB613549FB699B080233BA6941F84E
:1046E40023203A4B9B68BB613B69DB43BA691340A7
:1046F400BB613B685B6803F48013002B03D0BA6989
:104704003B691343BB61314ABB6993602F4BDB6840
:10471400BB613B69DB43BA691340BB613B685B68BF
:1047240003F40013002B03D0BA693B691343BB6144
:10473400264ABB69D360254B5B68BB613B69DB439D
:10474400BA691340BB613B685B6803F40033002B18
:1047540003D0BA693B691343BB611C4ABB6953600C
:104764001A4B1B68BB613B69DB43BA691340BB61ED
:104774003B685B6803F48033002B03D0BA693B6960
:104784001343BB61114ABB691360FB690133FB61CD
:10479400FB690F2B7FF696AE00BF00BF2437BD46E2
:1047A4005DF8047B704700BF0038024000380140C8
:1047B400000002400004024000080240000C0240D5
:1047C400001002400014024000180240003C014066
:1047D40080B485B000AF78600B467B807B681A6933
:1047E4007B881340002B02D00123FB7301E00023DC
:1047F400FB73FB7B18461437BD465DF8047B70479A
:1048040080B483B000AF78600B467B8013467B7026
:104814007B78002B03D07A887B689A6103E07B88DD
:104824001A047B689A6100BF0C37BD465DF8047BAF
:10483400704780B485B000AF78600B467B807B689E
:104844005B69FB607A88FB6813401A04FB68D943F0
:104854007B880B401A437B689A6100BF1437BD46BE
:104864005DF8047B7047000080B582B000AF03465A
:10487400FB80084B5A69FB881340002B06D0054A7D
:10488400FB885361FB881846FDF72EFA00BF0837F2
:10489400BD4680BD003C014080B584B000AF786067
:1048A4007B68002B01D101232BE17B6893F83D3019
:1048B400DBB2002B06D17B68002283F83C207868A9
:1048C400FCF78EFD7B68242283F83D207B681B68FF
:1048D4001A687B681B6822F001021A607B681B68F7
:1048E4001A687B681B6842F400421A607B681B6884
:1048F4001A687B681B6822F400421A6002F046FBC7
:10490400F8607B685B68814A934207D8FB68804AF9
:10491400934294BF01230023DBB206E0FB687D4A87
:10492400934294BF01230023DBB2002B01D0012367
:10493400E7E0FB68784AA2FB03239B0CBB607B681F
:104944001B685B6823F03F017B681B68BA680A43F5
:104954005A607B681B681B6A23F03F017B685B68B5
:104964006A4A934202D8BB68013309E0BB684FF43A
:10497400967202FB03F3694AA2FB03239B090133EA
:104984007A6812680B4313627B681B68DB6923F443
:104994004F4222F0FF027B685B685C498B4219D866
:1049A400FB68591E7B685B685B00B1FBF3F3591C21
:1049B40040F6FC730B40002B0AD0FB68591E7B6841
:1049C4005B685B00B1FBF3F30133C3F30B0351E00A
:1049D40004234FE07B689B68002B11D1FB68581EB1
:1049E4007B6859680B465B000B44B0FBF3F301335F
:1049F400C3F30B03002B0CBF01230023DBB212E033
:104A0400FB68581E7B6859680B469B000B44990051
:104A14000B44B0FBF3F30133C3F30B03002B0CBFC4
:104A240001230023DBB2002B01D0012322E07B68A9
:104A34009B68002B0ED1FB68581E7B6859680B4697
:104A44005B000B44B0FBF3F30133C3F30B0343F4F8
:104A540000430FE0FB68581E7B6859680B469B00B7
:104A64000B4499000B44B0FBF3F30133C3F30B0382
:104A740043F44043796809681343CB617B681B683E
:104A84001B6823F0C0017B68DA697B681B6A1A43E0
:104A94007B681B680A431A607B681B689B6823F465
:104AA400034323F0FF037A6811697A68D2681143DB
:104AB4007A6812680B4393607B681B68DB6823F099
:104AC400FF017B685A697B689B691A437B681B6892
:104AD4000A43DA607B681B681A687B681B6842F0CB
:104AE40001021A607B6800221A647B68202283F822
:104AF4003D207B6800221A637B68002283F83E20F5
:104B0400002318461037BD4680BD00BFA0860100B3
:104B14007F841E00FF083D0083DE1B43D34D6210DB
:104B240080B588B002AFF860084611461A460346BD
:104B34007B810B463B811346FB80FEF7EFF97861DE
:104B4400FB6893F83D30DBB2202B40F0D9807B69C1
:104B54000093192301226D49F86800F07FFC034695
:104B6400002B01D00223CCE0FB6893F83C30012BEE
:104B740001D10223C5E0FB68012283F83C20FB68D5
:104B84001B681B6803F00103012B07D0FB681B683B
:104B94001A68FB681B6842F001021A60FB681B6814
:104BA4001A68FB681B6822F400621A60FB68212201
:104BB40083F83D20FB68402283F83E20FB680022F6
:104BC4001A64FB683A6A5A62FB68BA8C5A85FB68B5
:104BD4005B8D9AB2FB681A85FB684D4ADA62F888E5
:104BE4003A8979897B690193BB6A00930346F86823
:104BF40000F0B6FA0346002B52D0012381E07A6913
:104C0400B96AF86800F000FD0346002B0DD0FB687C
:104C14001B6C042B07D1FB681B681A68FB681B68B4
:104C240042F400721A6001236BE0FB685B6A1A7835
:104C3400FB681B681A61FB685B6A5A1CFB685A6252
:104C4400FB681B8D013B9AB2FB681A85FB685B8D80
:104C54009BB2013B9AB2FB685A85FB681B685B698F
:104C640003F00403042B1BD1FB681B8D002B17D00E
:104C7400FB685B6A1A78FB681B681A61FB685B6AED
:104C84005A1CFB685A62FB681B8D013B9AB2FB6895
:104C94001A85FB685B8D9BB2013B9AB2FB685A850F
:104CA400FB681B8D002BAAD17A69B96AF86800F0F9
:104CB400ECFC0346002B0DD0FB681B6C042B07D1C6
:104CC400FB681B681A68FB681B6842F400721A6070
:104CD400012316E0FB681B681A68FB681B6842F432
:104CE40000721A60FB68202283F83D20FB680022D2
:104CF40083F83E20FB68002283F83C20002300E078
:104D0400022318461837BD4680BD00BF02001000BC
:104D14000000FFFF80B58CB002AFF8600846114672
:104D24001A4603467B810B463B811346FB80FEF704
:104D3400F5F87862FB6893F83D30DBB2202B40F045
:104D440008827B6A0093192301227B49F86800F0EA
:104D540085FB0346002B01D00223FBE1FB6893F89B
:104D64003C30012B01D10223F4E1FB68012283F8DA
:104D74003C20FB681B681B6803F00103012B07D070
:104D8400FB681B681A68FB681B6842F001021A6022
:104D9400FB681B681A68FB681B6822F400621A60CF
:104DA400FB68222283F83D20FB68402283F83E20E2
:104DB400FB6800221A64FB683A6B5A62FB68BA8E7D
:104DC4005A85FB685B8D9AB2FB681A85FB685B4A5F
:104DD400DA62F8883A8979897B6A0193BB6B00931C
:104DE4000346F86800F052FA0346002B01D0012371
:104DF400B0E1FB681B8D002B13D100233B62FB68E1
:104E04001B685B693B62FB681B689B693B623B6A8E
:104E1400FB681B681A68FB681B6842F400721A601E
:104E240084E1FB681B8D012B1BD1FB681B681A688E
:104E3400FB681B6822F480621A600023FB61FB6834
:104E44001B685B69FB61FB681B689B69FB61FB6911
:104E5400FB681B681A68FB681B6842F400721A60DE
:104E640064E1FB681B8D022B1BD1FB681B681A686D
:104E7400FB681B6822F480621A60FB681B681A686E
:104E8400FB681B6842F400621A600023BB61FB6884
:104E94001B685B69BB61FB681B689B69BB61BB6981
:104EA40044E100237B61FB681B685B697B61FB68F1
:104EB4001B689B697B617B6938E1FB681B8D032B55
:104EC40000F2F180FB681B8D012B23D17A6AB96B48
:104ED400F86800F01BFC0346002B01D0012339E1E4
:104EE400FB681B681A69FB685B6AD2B21A70FB68BC
:104EF4005B6A5A1CFB685A62FB681B8D013B9AB2C1
:104F0400FB681A85FB685B8D9BB2013B9AB2FB6818
:104F14005A850BE1FB681B8D022B4ED17B6A0093F3
:104F2400BB6B00220649F86800F098FA0346002B90
:104F340008D001230EE100BF020010000000FFFFB3
:104F440004000100FB681B681A68FB681B6842F4D4
:104F540000721A60FB681B681A69FB685B6AD2B24C
:104F64001A70FB685B6A5A1CFB685A62FB681B8DEB
:104F7400013B9AB2FB681A85FB685B8D9BB2013BCF
:104F84009AB2FB685A85FB681B681A69FB685B6AFE
:104F9400D2B21A70FB685B6A5A1CFB685A62FB68DF
:104FA4001B8D013B9AB2FB681A85FB685B8D9BB233
:104FB400013B9AB2FB685A85B8E07B6A0093BB6BED
:104FC40000226649F86800F049FA0346002B01D034
:104FD4000123BFE0FB681B681A68FB681B6822F4A6
:104FE40080621A60FB681B681A69FB685B6AD2B24C
:104FF4001A70FB685B6A5A1CFB685A62FB681B8D5B
:10500400013B9AB2FB681A85FB685B8D9BB2013B3E
:105014009AB2FB685A857B6A0093BB6B00224F49A6
:10502400F86800F01BFA0346002B01D0012391E03D
:10503400FB681B681A68FB681B6842F400721A60FC
:10504400FB681B681A69FB685B6AD2B21A70FB685A
:105054005B6A5A1CFB685A62FB681B8D013B9AB25F
:10506400FB681A85FB685B8D9BB2013B9AB2FB68B7
:105074005A85FB681B681A69FB685B6AD2B21A70AE
:10508400FB685B6A5A1CFB685A62FB681B8D013B18
:105094009AB2FB681A85FB685B8D9BB2013B9AB29E
:1050A400FB685A8542E07A6AB96BF86800F02EFB17
:1050B4000346002B01D001234CE0FB681B681A69EE
:1050C400FB685B6AD2B21A70FB685B6A5A1CFB68A5
:1050D4005A62FB681B8D013B9AB2FB681A85FB6818
:1050E4005B8D9BB2013B9AB2FB685A85FB681B68D7
:1050F4005B6903F00403042B18D1FB681B681A696D
:10510400FB685B6AD2B21A70FB685B6A5A1CFB6864
:105114005A62FB681B8D013B9AB2FB681A85FB68D7
:105124005B8D9BB2013B9AB2FB685A85FB681B8D71
:10513400002B7FF4C2AEFB68202283F83D20FB687D
:10514400002283F83E20FB68002283F83C200023E1
:1051540000E0022318462837BD4680BD0400010044
:1051640080B588B002AFF860084611461A46034677
:105174007B810B463B811346FB80FB681B681A68E6
:10518400FB681B6842F480721A607B6A00933B6A76
:1051940000224FF00111F86800F060F90346002B7B
:1051A4000DD0FB681B681B6803F48073B3F5807F24
:1051B40003D1FB684FF400721A6403235FE07B8918
:1051C400DBB21A46FB681B6802F0FE021A617B6AB6
:1051D4003A6A2D49F86800F098F90346002B01D08B
:1051E40001234CE000237B61FB681B685B697B61E6
:1051F400FB681B689B697B617B697A6A396AF8681A
:1052040000F002FA0346002B0DD0FB681B6C042B44
:1052140007D1FB681B681A68FB681B6842F40072BC
:105224001A6001232BE0FB88012B05D13B89DAB2FC
:10523400FB681B681A6121E03B891B0A9BB2DAB246
:10524400FB681B681A617A6A396AF86800F0DCF94D
:105254000346002B0DD0FB681B6C042B07D1FB68A5
:105264001B681A68FB681B6842F400721A60012309
:1052740005E03B89DAB2FB681B681A610023184613
:105284001837BD4680BD00BF0200010080B588B05C
:1052940002AFF860084611461A4603467B810B4666
:1052A4003B811346FB80FB681B681A68FB681B681C
:1052B40042F480621A60FB681B681A68FB681B680A
:1052C40042F480721A607B6A00933B6A00224FF0BA
:1052D4000111F86800F0C2F80346002B0DD0FB68FA
:1052E4001B681B6803F48073B3F5807F03D1FB68EC
:1052F4004FF400721A640323AAE07B89DBB21A46D6
:10530400FB681B6802F0FE021A617B6A3A6A524922
:10531400F86800F0FAF80346002B01D0012397E067
:1053240000237B61FB681B685B697B61FB681B680E
:105334009B697B617B697A6A396AF86800F064F971
:105344000346002B0DD0FB681B6C042B07D1FB68B4
:105354001B681A68FB681B6842F400721A60012318
:1053640076E0FB88012B05D13B89DAB2FB681B6828
:105374001A6121E03B891B0A9BB2DAB2FB681B6805
:105384001A617A6A396AF86800F03EF90346002B1C
:105394000DD0FB681B6C042B07D1FB681B681A68D3
:1053A400FB681B6842F400721A60012350E03B89D9
:1053B400DAB2FB681B681A617A6A396AF86800F025
:1053C40023F90346002B0DD0FB681B6C042B07D17B
:1053D400FB681B681A68FB681B6842F400721A6059
:1053E400012335E0FB681B681A68FB681B6842F4FC
:1053F40080721A607B6A00933B6A00224FF00111AD
:10540400F86800F02BF80346002B0DD0FB681B68EE
:105414001B6803F48073B3F5807F03D1FB684FF4FA
:1054240000721A64032313E07B89DBB243F00103A7
:10543400DAB2FB681B681A617B6A3A6A0649F86843
:1054440000F063F80346002B01D0012300E00023A1
:1054540018461837BD4680BD0200010080B584B0EF
:1054640000AFF860B9603B601346FB7125E03B6810
:10547400B3F1FF3F21D0FDF751FD0246BB69D31ABA
:105484003A689A4202D33B68002B16D1FB6800228B
:105494001A63FB68202283F83D20FB68002283F80E
:1054A4003E20FB681B6C43F02002FB681A64FB6817
:1054B400002283F83C20012323E0BB681B0CDBB2F1
:1054C400012B0DD1FB681B685B69DA43BB68134091
:1054D4009BB2002B0CBF01230023DBB21A460CE065
:1054E400FB681B689B69DA43BB6813409BB2002BC3
:1054F4000CBF01230023DBB21A46FB799A42B6D0D3
:10550400002318461037BD4680BD80B584B000AF77
:10551400F860B9607A603B6051E0FB681B685B69C6
:1055240003F48063B3F5806F23D1FB681B681A68AA
:10553400FB681B6842F400721A60FB681B686FF416
:1055440080625A61FB6800221A63FB68202283F898
:105554003D20FB68002283F83E20FB681B6C43F06F
:105564000402FB681A64FB68002283F83C200123D0
:1055740046E07B68B3F1FF3F21D0FDF7CFFC024644
:105584003B68D31A7A689A4202D37B68002B16D1FF
:10559400FB6800221A63FB68202283F83D20FB6825
:1055A400002283F83E20FB681B6C43F02002FB685A
:1055B4001A64FB68002283F83C20012320E0BB68C6
:1055C4001B0CDBB2012B0CD1FB681B685B69DA4353
:1055D400BB6813409BB2002B14BF01230023DBB232
:1055E4000BE0FB681B689B69DA43BB6813409BB202
:1055F400002B14BF01230023DBB2002B8DD1002329
:1056040018461037BD4680BD80B584B000AFF86041
:10561400B9607A602DE0F86800F0CEF80346002BFC
:1056240001D001232DE0BB68B3F1FF3F21D0FDF78A
:1056340075FC02467B68D31ABA689A4202D3BB68E7
:10564400002B16D1FB6800221A63FB68202283F822
:105654003D20FB68002283F83E20FB681B6C43F06E
:105664002002FB681A64FB68002283F83C200123B3
:1056740007E0FB681B685B6903F08003802BCAD1D9
:10568400002318461037BD4680BD80B584B000AFF6
:10569400F860B9607A602DE0F86800F08DF8034690
:1056A400002B01D001232DE0BB68B3F1FF3F21D0D3
:1056B400FDF734FC02467B68D31ABA689A4202D3D7
:1056C400BB68002B16D1FB6800221A63FB682022FA
:1056D40083F83D20FB68002283F83E20FB681B6CA6
:1056E40043F02002FB681A64FB68002283F83C2024
:1056F400012307E0FB681B685B6903F00403042BC8
:10570400CAD1002318461037BD4680BD80B584B089
:1057140000AFF860B9607A6042E0FB681B685B69BF
:1057240003F01003102B19D1FB681B686FF01002F3
:105734005A61FB6800221A63FB68202283F83D202B
:10574400FB68002283F83E20FB681A6CFB681A642D
:10575400FB68002283F83C20012329E0FDF7DEFBEF
:1057640002467B68D31ABA689A4202D3BB68002BFC
:1057740016D1FB6800221A63FB68202283F83D20BF
:10578400FB68002283F83E20FB681B6C43F0200278
:10579400FB681A64FB68002283F83C20012307E0BD
:1057A400FB681B685B6903F04003402BB5D1002301
:1057B40018461037BD4680BD80B483B000AF786012
:1057C4007B681B685B6903F48063B3F5806F1BD14E
:1057D4007B681B686FF480625A617B6800221A63DD
:1057E4007B68202283F83D207B68002283F83E20DA
:1057F4007B681B6C43F004027B681A647B6800229C
:1058040083F83C20012300E0002318460C37BD46F2
:105814005DF8047B7047F0B58FB00AAF78607B68A1
:10582400002B01D1012316E17B681B68BB607B68F8
:1058340093F8BD34DBB2002B06D17B68002283F8D9
:10584400BC24786809F088F97B68032283F8BD24B6
:10585400BB68DB6B03F48073002B02D17B680022EE
:105864001A617B681B68184605F083FC7B681B681B
:105874003B607E686D4606F110040FCC0FC50FCC5B
:105884000FC594E8030085E80300331D0ECB386888
:1058940005F05AFB0346002B05D07B68022283F8EF
:1058A400BD240123D7E07B681B680021184605F05E
:1058B40071FC0023FB734AE0FA7B79681346DB0032
:1058C40013449B000B443D3301221A70FA7B796820
:1058D4001346DB0013449B000B443C33FA7B1A70E1
:1058E400FA7BFB7B98B279681346DB0013449B0078
:1058F4000B44443302461A80FA7B79681346DB0072
:1059040013449B000B44403300221A70FA7B7968DD
:105914001346DB0013449B000B44483300221A60F7
:10592400FA7B79681346DB0013449B000B444C3329
:1059340000221A60FA7B79681346DB0013449B004B
:105944000B44543300221A60FB7B0133FB73FA7B54
:105954007B685B689A42AFD30023FB7344E0FA7B15
:1059640079681346DB0013449B000B4403F27D2348
:1059740000221A70FA7B79681346DB0013449B00FB
:105984000B4403F51F73FA7B1A70FA7B796813468C
:10599400DB0013449B000B4403F5207300221A70B0
:1059A400FA7B79681346DB0013449B000B4403F530
:1059B400227300221A60FA7B79681346DB001344D1
:1059C4009B000B4403F5237300221A60FA7B796869
:1059D4001346DB0013449B000B4403F5257300229C
:1059E4001A60FB7B0133FB73FA7B7B685B689A422A
:1059F400B5D37B681B683B607E686D4606F1100476
:105A04000FCC0FC50FCC0FC594E8030085E8030045
:105A1400331D0ECB386805F009FC0346002B05D076
:105A24007B68022283F8BD24012314E07B680022F2
:105A340083F838207B68012283F8BD247B685B6A85
:105A4400012B02D1786801F08BF97B681B6818463A
:105A540006F04BFD002318461437BD46F0BD80B553
:105A640084B000AF78607B681B68FB607B6893F848
:105A7400BC34012B01D1022320E07B68012283F88E
:105A8400BC247B689B6A012B09D17B689B69012B31
:105A940005D0FB689B6B43F48032FB689A637B6898
:105AA4001B68184605F054FB7B681B68184606F013
:105AB400FBFC7B68002283F8BC24002318461037C3
:105AC400BD4680BD90B58DB000AF78607B681B6823
:105AD4003B623B6AFB617B681B68184606F0B9FDB4
:105AE4000346002B40F0B7847B681B68184606F019
:105AF4001DFD0346002B00F0AD84FB6903F5006334
:105B04009B681B0AC3F30D027B68C3F8FC247B6803
:105B14001B68184606F00AFD034603F00203022B35
:105B240007D17B681B685A697B681B6802F0020214
:105B34005A617B681B68184606F0F8FC034603F0BC
:105B44001003102B61D17B681B689A697B681B6802
:105B540022F010029A613B6A1B6ABB61BB6903F0C5
:105B64000F021346DB0013449B0003F51E737A688F
:105B7400134404337B61BB695B0C03F00F03022BFA
:105B840024D1BA6947F6F0731340002B35D07B69F2
:105B94001969BB691B099BB2C3F30A039BB21A467A
:105BA400386A06F02FFB7B691A69BB691B09C3F3CA
:105BB4000A031A447B691A617B691A6ABB691B0967
:105BC400C3F30A031A447B691A6216E0BB695B0CCF
:105BD40003F00F03062B10D17B6803F2C4430822A1
:105BE4001946386A06F00EFB7B691A6ABB691B0901
:105BF400C3F30A031A447B691A627B681B689A69B7
:105C04007B681B6842F010029A617B681B68184627
:105C140006F08CFC034603F40023B3F5002F40F098
:105C2400A78000237B627B681B68184606F091FC02
:105C3400B86299E0BB6A03F00103002B00F08E8088
:105C44007B681B687A6AD2B21146184606F0B5FC26
:105C540038613B6903F00103002B0CD07B6A5A01C5
:105C6400FB69134403F530631A4601239360796A90
:105C7400786800F0EFFE3B6903F00803002B0CD0BA
:105C84007B6A5A01FB69134403F530631A460823FF
:105C94009360796A786800F0C5FF3B6903F01003EC
:105CA400002B08D07B6A5A01FB69134403F5306367
:105CB4001A46102393603B6903F00203002B30D093
:105CC4003B6A5B6903F08003802B09D1FB6903F510
:105CD40000635B68FA6902F5006243F48063536011
:105CE4007A6A1346DB0013449B0003F51E737A683B
:105CF400134404337B617B69DB78012B08D17B6916
:105D04000022DA707B6ADBB21946786809F040F841
:105D14007B6A5A01FB69134403F530631A46022374
:105D240093603B6903F02003002B08D07B6A5A017F
:105D3400FB69134403F530631A46202393603B69DF
:105D440003F40053002B09D07B6A5A01FB69134406
:105D540003F530631A464FF4005393607B6A0133B2
:105D64007B62BB6A5B08BB62BB6A002B7FF462AFD9
:105D74007B681B68184606F0D9FB034603F48023AE
:105D8400B3F5802F40F0DB807B681B68184606F073
:105D9400FAFBB86200237B62CDE0BB6A03F0010327
:105DA400002B00F0C2807B681B687A6AD2B211466D
:105DB400184606F020FC38613B6903F00103002B10
:105DC40057D07B6A03F00F03012202FA03F3FB604E
:105DD400FB6903F500635A6BFB68DB43F96901F562
:105DE400006113404B637B6A5A01FB69134403F55A
:105DF40010631A46012393607B681B69012B32D11F
:105E040079687A6A1346DB0013449B000B444C33D5
:105E1400196878687A6A1346DB0013449B000344CC
:105E240048331B68194478687A6A1346DB001344C4
:105E34009B0003444C3319607B6A002B13D17968AF
:105E44007A6A1346DB0013449B000B4454331B68EB
:105E5400002B08D17B6818687B6803F2C4431A4698
:105E6400012106F027FC7B6ADBB21946786808F04A
:105E74000AFF3B6903F00803002B08D07B6A5A0130
:105E8400FB69134403F510631A46082393603B69C6
:105E940003F01003002B08D07B6A5A01FB691344FA
:105EA40003F510631A46102393603B6903F0400323
:105EB400002B08D07B6A5A01FB69134403F5106375
:105EC4001A46402393603B6903F00203002B23D05E
:105ED400796A386A05F008FB7A6A1346DB001344D2
:105EE4009B0038337A68134404337B617B69DB7825
:105EF400012B08D17B690022DA707B6ADBB2194678
:105F0400786808F057FF7B6A5A01FB69134403F56C
:105F140010631A46022393603B6903F08003002B4D
:105F240003D0796A786800F008FD7B6A01337B62EC
:105F3400BB6A5B08BB62BB6A002B7FF42EAF7B6835
:105F44001B68184606F0F2FA034603F00043B3F167
:105F5400004F22D1FB6903F500635B68FA6902F51F
:105F6400006223F0010353607B6893F8F434012B3F
:105F740008D17B68002283F8F4240021786809F0B2
:105F8400D1F802E0786808F0F5FE7B681B685A696E
:105F94007B681B6802F000425A617B681B681846E4
:105FA40006F0C4FA034603F40063B3F5006F12D19C
:105FB400FB6903F500639B6803F00103012B02D125
:105FC400786808F0B1FE7B681B685A697B681B68B7
:105FD40002F400625A617B681B68184606F0A6FA50
:105FE400034603F00063B3F1006F21D17B681B68A3
:105FF4005A697B681B6802F000625A617B6893F8F7
:10600400F434002B11D17B68012283F8F4247B68DB
:106014001B685B6D9B0803F00F027B68C3F8F824D0
:106024000121786809F07EF802E0786808F07CFEC7
:106034007B681B68184606F079FA034603F480531C
:10604400B3F5805F40F0B780FB6903F500635B68DC
:10605400FA6902F5006223F0010353607B681B6850
:106064001021184605F040FA0023FB6246E0FB6A63
:106074005A01FB69134403F510631A464FF67F3344
:106084009360FB6A5A01FB69134403F510631B68B0
:10609400FA6A5101FA690A4402F5106223F4001302
:1060A4001360FB6A5A01FB69134403F530631A4613
:1060B4004FF67F339360FB6A5A01FB69134403F57F
:1060C40030631B68FA6A5101FA690A4402F53062C6
:1060D40023F400131360FB6A5A01FB69134403F5AC
:1060E40030631B68FA6A5101FA690A4402F53062A6
:1060F40043F000631360FB6A0133FB627B685B68F7
:10610400FA6A9A42B3D3FB6903F50063DB69FA695F
:1061140002F5006243F00113D3617B681B6B002B13
:1061240016D0FB6903F50063D3F88430FA6902F5ED
:10613400006243F00B03C2F88430FB6903F500638B
:106144005B6CFA6902F5006243F00B03536415E0DB
:10615400FB6903F500635B69FA6902F5006243F4C5
:10616400005343F02B035361FB6903F500631B6980
:10617400FA6902F5006243F00B031361FB6903F54E
:1061840000631B68FA6902F5006223F4FE6313607E
:106194007B6818687B681B69D9B27B6803F2C443C7
:1061A4001A4606F087FA7B681B685A697B681B6885
:1061B40002F480525A617B681B68184606F0B6F9EF
:1061C400034603F40053B3F5005F24D17B681B68D6
:1061D400184606F04CFA7B681B68184605F001FA6D
:1061E40003461A467B68DA607B681C6800F0C2FECE
:1061F40001467B68DB68DBB21A46204604F006FFE2
:10620400786808F068FD7B681B685A697B681B68BE
:1062140002F400525A617B681B68184606F086F93E
:10622400034603F00803082B0AD1786808F045FDFB
:106234007B681B685A697B681B6802F008025A6114
:106244007B681B68184606F071F9034603F0800367
:10625400802B22D13B6A9B6923F080023B6A9A61BE
:1062640001237B6214E079687A6A1346DB001344E5
:106274009B000B4403F27F231B78012B05D17B6A1F
:10628400DBB21946786800F027FB7B6A01337B6236
:106294007B685B687A6A9A42E5D37B681B68184618
:1062A40006F044F9034603F48013B3F5801F3BD191
:1062B40001237B622BE07B6A5A01FB69134403F5DB
:1062C40010631B68BB6179687A6A1346DB00134468
:1062D4009B000B4440331B78012B15D1BB69002B69
:1062E40012DA79687A6A1346DB0013449B000B4484
:1062F4003F3301221A707B6ADBB263F07F03DBB2A7
:106304001946786800F0E8FA7B6A01337B627B689F
:106314005B687A6A9A42CED37B681B685A697B6849
:106324001B6802F480125A617B681B68184606F0E9
:10633400FDF8034603F40013B3F5001F55D1012300
:106344007B6245E07B6A5A01FB69134403F53063C1
:106354001B68BB6179687A6A1346DB0013449B00AF
:106364000B4403F520731B78012B2ED1BB69002B42
:106374002BDABB6903F480327B68D3F8FC3403F076
:1063840001039A4221D179687A6A1346DB001344E7
:106394009B000B4403F27F2301221A703B6A9B6922
:1063A40043F080023B6A9A613B6A5B6903F08003B5
:1063B400002B0AD1FB6903F500635B68FA6902F5F7
:1063C400006243F40073536007E07B6A01337B622D
:1063D4007B685B687A6A9A42B4D37B681B685A69A3
:1063E4007B681B6802F400125A617B681B681846BC
:1063F40006F09CF8034603F08043B3F1804F0AD1C2
:10640400786808F0E9FC7B681B685A697B681B683C
:1064140002F080425A617B681B68184606F086F8D1
:10642400034603F00403042B15D17B681B685B68E7
:10643400BB61BB6903F00403002B02D0786808F049
:10644400D9FC7B681B6859687B681B68BA690A4376
:106454005A6000E000BF3437BD4690BD80B582B0BD
:1064640000AF78600B46FB707B6893F8BC34012B5B
:1064740001D1022313E07B68012283F8BC247B68EA
:10648400FA7883F838207B681B68FA781146184636
:1064940005F0E4FF7B68002283F8BC24002318463F
:1064A4000837BD4680BD80B584B000AF786008462B
:1064B40011461A460346FB700B463B801346BB70DD
:1064C4000023FB7297F90330002B0FDAFB7803F0FB
:1064D4000F021346DB0013449B0038337A681344DD
:1064E4000433FB60FB6801225A700FE0FB7803F071
:1064F4000F021346DB0013449B0003F51E737A68F6
:1065040013440433FB60FB6800225A70FB7803F0E9
:106514000F03DAB2FB681A703A88FB68DA60FB682A
:10652400BA781A71FB685B78002B04D0FB681B787F
:106534009AB2FB681A81BB78022B02D1FB68002255
:106544005A717B6893F8BC34012B01D102230EE00D
:106554007B68012283F8BC247B681B68F9681846B1
:1065640005F064F87B68002283F8BC24FB7A1846A3
:106574001037BD4680BD80B584B000AF78600B464F
:10658400FB7097F90330002B0FDAFB7803F00F024E
:106594001346DB0013449B0038337A6813440433F6
:1065A400FB60FB6801225A700FE0FB7803F00F02D6
:1065B4001346DB0013449B0003F51E737A681344EF
:1065C4000433FB60FB6800225A70FB7803F00F036E
:1065D400DAB2FB681A707B6893F8BC34012B01D1E2
:1065E40002230EE07B68012283F8BC247B681B68CD
:1065F400F968184605F0A2F87B68002283F8BC24E9
:10660400002318461037BD4680BD80B586B000AF64
:10661400F8607A603B600B46FB72FB7A03F00F0272
:106624001346DB0013449B0003F51E73FA681344FE
:1066340004337B617B697A681A617B693A689A6181
:106644007B6900221A627B6900225A70FB7A03F08C
:106654000F03DAB27B691A70FB681B69012B02D144
:106664007A687B695A61FB7A03F00F03002B09D126
:10667400FB681868FB681B69DBB21A46796905F088
:1066840081FB08E0FB681868FB681B69DBB21A46EB
:10669400796905F02FF9002318461837BD4680BDE7
:1066A40080B483B000AF78600B46FB70FB7803F0D6
:1066B4000F0279681346DB0013449B000B4403F577
:1066C40027731B6818460C37BD465DF8047B70477A
:1066D40080B586B000AFF8607A603B600B46FB7211
:1066E400FB7A03F00F021346DB0013449B0038339C
:1066F400FA68134404337B617B697A681A617B69A5
:106704003A689A617B6900221A627B6901225A7095
:10671400FB7A03F00F03DAB27B691A70FB681B691A
:10672400012B02D17A687B695A61FB7A03F00F036B
:10673400002B09D1FB681868FB681B69DBB21A4699
:10674400796905F01FFB08E0FB681868FB681B69A2
:10675400DBB21A46796905F0CDF8002318461837DC
:10676400BD4680BD80B584B000AF78600B46FB7039
:10677400FB7803F00F027B685B689A4201D901231E
:1067840050E097F90330002B0FDAFB7803F00F0287
:106794001346DB0013449B0038337A6813440433F4
:1067A400FB60FB6801225A700DE0FA781346DB00A7
:1067B40013449B0003F51E737A6813440433FB608F
:1067C400FB6800225A70FB6801229A70FB7803F080
:1067D4000F03DAB2FB681A707B6893F8BC34012BA0
:1067E40001D102231EE07B68012283F8BC247B686C
:1067F4001B68F968184605F05DFDFB7803F00F038C
:10680400002B0AD17B6818687B681B69D9B27B6846
:1068140003F2C4431A4605F04DFF7B68002283F857
:10682400BC24002318461037BD4680BD80B584B013
:1068340000AF78600B46FB70FB7803F00F027B68B7
:106844005B689A4201D9012342E097F90330002B97
:106854000FDAFB7803F00F021346DB0013449B00AE
:1068640038337A6813440433FB60FB6801225A709E
:106874000FE0FB7803F00F021346DB0013449B0088
:1068840003F51E737A6813440433FB60FB6800222B
:106894005A70FB6800229A70FB7803F00F03DAB297
:1068A400FB681A707B6893F8BC34012B01D1022376
:1068B4000EE07B68012283F8BC247B681B68F968BE
:1068C400184605F065FD7B68002283F8BC2400238C
:1068D40018461037BD4680BD80B584B000AF7860DF
:1068E4000B46FB7097F90330002B0CDAFB7803F0AE
:1068F4000F021346DB0013449B0038337A681344B9
:106904000433FB600CE0FB7803F00F021346DB005A
:1069140013449B0003F51E737A6813440433FB602D
:106924007B681B68F968184605F084FB0346FB7214
:10693400FB7A18461037BD4680BD80B58AB002AFD9
:10694400786039607B681B687B617B693B613A686E
:106954001346DB0013449B0038337A681344043332
:10696400FB60FB681A6AFB689B699A4201D90123A0
:106974006CE0FB689A69FB681B6AD31AFB61FB68CD
:10698400DB68FA699A4202D9FB68DB68FB61FB6940
:1069940003339B08BB612BE0FB689A69FB681B6AA5
:1069A400D31AFB61FB68DB68FA699A4202D9FB6877
:1069B400DB68FB61FB6903339B08BB61FB681969F6
:1069C4003B68DAB2FB6998B27B681B69DBB200935F
:1069D4000346786905F0D8FBFB681A69FB691A4419
:1069E400FB681A61FB681A6AFB691A44FB681A623D
:1069F4003B685A013B69134403F510639B699BB2DE
:106A0400BA699A4209D8FB681A6AFB689B699A4278
:106A140003D2FB689B69002BBED1FB689A69FB68B3
:106A24001B6A9A4211D83B6803F00F03012202FA51
:106A340003F3BB603B6903F500635A6BBB68DB433C
:106A4400396901F5006113404B6300231846203770
:106A5400BD4680BD80B588B000AF786039607B6882
:106A64001B68FB61FB69BB61FB693C3304331B6836
:106A74007B613B685A01BB69134403F530639B682F
:106A84003B617B681B69012B7BD13B6903F00803E5
:106A9400002B15D07B69614A934240F2B9803B696F
:106AA40003F40043002B00F0B3803B685A01BB6938
:106AB400134403F530631A464FF400439360A7E090
:106AC4003B6903F02003002B09D03B685A01BB69E2
:106AD400134403F530631A462023936098E03B691E
:106AE40003F02803002B40F093807B694B4A9342C8
:106AF4000FD93B6903F40043002B0AD03B685A01C9
:106B0400BB69134403F530631A464FF400439360A2
:106B14007EE03A681346DB0013449B0003F51E73C2
:106B24007A6813440433FB60FB68DA693B685901F3
:106B3400BB690B4403F530631B69C3F31203D21A18
:106B4400FB681A623B68002B14D1FB689B69002B1D
:106B540009D17B6818687B6803F2C4431A46012193
:106B640005F0A8FD06E0FB681A69FB681B6A1A4475
:106B7400FB681A613B68DBB21946786808F068F86C
:106B840046E07B69264A934224D13B6903F40043DF
:106B9400002B0AD03B685A01BB69134403F53063E8
:106BA4001A464FF40043936032E03B6903F020033C
:106BB400002B08D03B685A01BB69134403F53063CA
:106BC4001A46202393603B68DBB21946786808F0C4
:106BD4003FF81DE03B68002B14D179683A681346EE
:106BE400DB0013449B000B4403F525731B68002B47
:106BF40008D17B6818687B6803F2C4431A460021F5
:106C040005F058FD3B68DBB21946786808F020F8B7
:106C1400002318462037BD4680BD00BF0A30544FBC
:106C24000A31544F80B586B000AF786039607B6814
:106C34001B687B617B693B617B693C3304331B6864
:106C4400FB603B685A013B69134403F530639B685E
:106C5400BB60FB68154A93420ED9BB6803F400433A
:106C6400002B09D03B685A013B69134403F5306398
:106C74001A464FF400439360786807F0D7FFFB6827
:106C84000A4A93420CD97B681B69012B08D17B68A3
:106C940018687B6803F2C4431A46012105F00AFD13
:106CA400002318461837BD4680BD00BF0A30544F34
:106CB40080B485B000AF78600B46FB7013463B8010
:106CC4007B681B685B6ABB60FB78002B07D13B8841
:106CD40019047B681B68BA680A439A6228E07B68D7
:106CE4001B689B6A1B0CBA681344BB600023FB73CC
:106CF4000DE07B681A68FB7B40339B0013445B68A0
:106D04001B0CBA681344BB60FB7B0133FB73FA7B37
:106D1400FB78013B9A42ECD33B8818047B681968E2
:106D2400FB78013BBA68024340339B000B445A6032
:106D3400002318461437BD465DF8047B704780B4C1
:106D440083B000AF78600B467B807B681B687A88D1
:106D54005A62002318460C37BD465DF8047B704721
:106D640080B485B000AF78607B681B68FB607B688B
:106D74000122C3F800257B68002283F8F424FB6811
:106D84009B6943F00062FB689A61FB685B6D43F0AA
:106D9400805343F00303FA685365002318461437FD
:106DA400BD465DF8047B704780B584B000AF786061
:106DB40039607B68002B01D10123CCE0684B1B6850
:106DC40003F00F033A689A420CD9654B3A68D2B281
:106DD4001A70634B1B6803F00F033A689A4201D0A0
:106DE4000123B8E07B681B6803F00203002B20D06A
:106DF4007B681B6803F00403002B05D0594B9B6888
:106E0400584A43F4E05393607B681B6803F008031B
:106E1400002B05D0534B9B68524A43F46043936064
:106E2400504B9B6823F0F0027B689B684D491343E9
:106E34008B607B681B6803F00103002B44D07B68E4
:106E44005B68012B07D1474B1B6803F40033002B0D
:106E540019D101237FE07B685B68022B03D07B6838
:106E64005B68032B07D13F4B1B6803F00073002BB7
:106E740009D101236FE03B4B1B6803F00203002B95
:106E840001D1012367E0374B9B6823F003027B6841
:106E94005B68344913438B60FCF740F8F8600AE000
:106EA400FCF73CF80246FB68D31A41F2883293425D
:106EB40001D903234FE02B4B9B6803F00C027B6842
:106EC4005B689B009A42EBD1254B1B6803F00F03D0
:106ED4003A689A420CD2224B3A68D2B21A70204BCA
:106EE4001B6803F00F033A689A4201D0012332E091
:106EF4007B681B6803F00403002B08D0194B9B68C4
:106F040023F4E0527B68DB68164913438B607B688B
:106F14001B6803F00803002B09D0124B9B6823F471
:106F240060427B681B69DB000E4913438B6000F0F1
:106F3400B1FB02460B4B9B681B0903F00F030A4984
:106F4400CB5C22FA03F3094A1360094B1B68184609
:106F5400FAF774FD002318461037BD4680BD00BF04
:106F6400003C0240003802406CF300080C00002092
:106F74001000002080B400AF034B1B681846BD46C8
:106F84005DF8047B704700BF0C00002080B500AFA3
:106F9400FFF7F0FF0246054B9B689B0A03F00703CB
:106FA4000349CB5C22FA03F3184680BD0038024043
:106FB4007CF3000880B500AFFFF7DCFF0246054B09
:106FC4009B685B0B03F007030349CB5C22FA03F3D2
:106FD400184680BD003802407CF3000880B483B0BA
:106FE40000AF786039607B680F221A60124B9B688F
:106FF40003F003027B685A600F4B9B6803F0F002B6
:107004007B689A600C4B9B6803F4E0527B68DA60FF
:10701400094B9B68DB0803F4E0527B681A61074B59
:107024001B6803F00F023B681A6000BF0C37BD46B3
:107034005DF8047B704700BF00380240003C02400A
:1070440080B58CB000AF786000237B6200233B6284
:107054000023FB610023BB6100237B6100233B61B0
:107064000023FB600023FB620023BB627B681B6878
:1070740003F00103002B10D06F4BD3F88C3023F0B6
:10708400C0627B689B6B6C491343C1F88C307B688E
:107094009B6B002B01D10123FB627B681B6803F00F
:1070A4000203002B10D0644BD3F88C3023F0C05271
:1070B4007B68DB6B60491343C1F88C307B68DB6B06
:1070C400002B01D10123FB627B681B6803F00403DE
:1070D400002B17D0584BD3F88C3023F440127B6824
:1070E4001B6B55491343C1F88C307B681B6BB3F59C
:1070F400801F01D10123FB627B681B6B002B01D134
:107104000123BB627B681B6803F00803002B17D0C4
:10711400494BD3F88C3023F440027B685B6B4649BF
:107124001343C1F88C307B685B6BB3F5800F01D1DE
:107134000123FB627B685B6B002B01D10123BB62E3
:107144007B681B6803F02003002B00F08A80002377
:10715400BB60394B1B6C384A43F080531364364B85
:107164001B6C03F08053BB60BB68344B1B68334A11
:1071740043F480731360FBF7D1FE786208E0FBF7F9
:10718400CDFE02467B6AD31A022B01D9032378E28F
:107194002A4B1B6803F48073002BF0D0264B1B6F23
:1071A40003F440733B623B6A002B2FD07B681B6C5B
:1071B40003F440733A6A9A4228D01F4B1B6F23F49E
:1071C40040733B621E4B01221A601D4B00221A6061
:1071D400194A3B6A1367184B1B6F03F00103012B19
:1071E40014D1FBF79BFE78620AE0FBF797FE024698
:1071F4007B6AD31A41F28832934201D9032340E2D5
:107204000D4B1B6F03F00203002BEED07B681B6C4D
:1072140003F44073B3F5407F14D1074B9B6823F408
:10722400F8127B681B6C23F0704323F4407302490B
:1072340013438B600CE000BF003802400070004034
:10724400400E47424A4B9B68494A23F4F813936023
:10725400474B1A6F7B681B6CC3F30B0344491343FE
:107264000B677B681B6803F01003002B04D07B685A
:1072740093F858203F4B1A607B681B6803F0800327
:10728400002B0AD03A4BD3F8943023F440027B68A5
:10729400DB6C37491343C1F894307B681B6803F0F7
:1072A4004003002B0AD0324BD3F8943023F0806291
:1072B4007B689B6C2E491343C1F894307B681B6830
:1072C40003F48073002B11D0294BD3F8943023F0AE
:1072D40000627B685B6D26491343C1F894307B6878
:1072E4005B6DB3F1006F01D10123BB627B681B6846
:1072F40003F40073002B0AD01D4BD3F8943023F011
:1073040080527B685B6C1A491343C1F894307B68E4
:107314001B6803F48063002B11D0154BD3F8943011
:1073240023F000527B681B6D11491343C1F894305C
:107334007B681B6DB3F1005F01D10123FB62FB6A23
:10734400012B05D07B681B68B3F5006F40F0FF800C
:10735400094B00221A60FBF7E1FD78620EE0FBF7AF
:10736400DDFD02467B6AD31A022B07D9032388E189
:1073740000380240E0114742680047427E4B1B68D8
:1073840003F00063002BEAD17B681B6803F0010360
:10739400002B03D07B689B6B002B09D07B681B6898
:1073A40003F00203002B28D07B68DB6B002B24D175
:1073B400714BD3F884301B0C03F0030301335B00DF
:1073C400FB616D4BD3F884301B0E03F00F03BB61DC
:1073D4007B685A687B689B689B011A43FB695B085E
:1073E400013B1B041A43BB691B061A437B685B6998
:1073F4001B0761491343C1F884307B681B6803F0A1
:107404000403002B04D07B681B6BB3F5801F0AD0E8
:107414007B681B6803F00803002B35D07B685B6B2B
:10742400B3F5800F30D1544BD3F884301B0C03F0E8
:10743400030301335B00FB614F4BD3F884301B0F14
:1074440003F007037B617B685A687B689B689B0138
:107454001A43FB695B08013B1B041A437B681B69E5
:107464001B061A437B691B0743491343C1F8843045
:10747400414BD3F88C3023F01F027B689B6A013B9D
:107484003D491343C1F88C307B681B6803F4806367
:10749400002B29D07B681B6DB3F1005F24D1364BE0
:1074A400D3F884301B0C03F0030301335B00BB618E
:1074B400314BD3F884301B0F03F007037B617B68E7
:1074C4005A687B689B689B011A437B68DB685B088E
:1074D400013B1B041A43BB691B061A437B691B0748
:1074E40025491343C1F884307B681B6803F40063A7
:1074F400002B16D07B685A687B689B689B011A43F3
:107504007B68DB685B08013B1B041A437B681B69CF
:107514001B061A437B685B691B0717491343C1F8B1
:107524008430164B01221A60FBF7F8FC786208E0FD
:10753400FBF7F4FC02467B6AD31A022B01D903231E
:107544009FE00D4B1B6803F00063002BF0D0BB6A77
:10755400012B40F095800A4B00221A60FBF7DEFCF9
:1075640078620FE0FBF7DAFC02467B6AD31A022B3F
:1075740008D9032385E000BF003802406800474271
:1075840070004742414B1B6803F00053B3F1005FA6
:10759400E8D07B681B6803F00403002B03D07B68EE
:1075A4001B6B002B09D07B681B6803F00803002BBE
:1075B4002BD07B685B6B002B27D1344BD3F88830FE
:1075C4001B0C03F0030301335B003B617B689A6986
:1075D4007B68DB699B011A433B695B08013B1B0425
:1075E4001A437B685B6A1B0628491343C1F8883039
:1075F400264BD3F88C3023F4F8527B68DB6A013BCA
:107604001B0222491343C1F88C307B681B6803F4C6
:107614008073002B1DD07B685B6DB3F1006F18D1B4
:107624001A4BD3F888301B0E03F00F03FB607B6802
:107634009A697B68DB699B011A437B681B6A5B0858
:10764400013B1B041A43FB681B0610491343C1F892
:1076540088300F4B01221A60FBF760FC786208E067
:10766400FBF75CFC02467B6AD31A022B01D9032385
:1076740007E0064B1B6803F00053B3F1005FEFD142
:10768400002318463037BD4680BD00BF0038024095
:10769400700047422DE9B04FA6B000AF0023C7F8F1
:1076A4008C300023C7F894300023C7F888300023B7
:1076B400C7F884300023C7F89030C84B9B6803F0A8
:1076C4000C030C2B00F27E8101A252F823F000BFC0
:1076D40009770008C9790008C9790008C979000840
:1076E40011770008C9790008C9790008C979000828
:1076F40019770008C9790008C9790008C979000810
:1077040083780008B64BC7F890305FE1B54BC7F8F3
:1077140090305BE1B14B5B6803F03F03C7F88C30FA
:10772400AE4B5B6803F48003002B31D0AB4B5B683A
:107734009B090022BB66FA66BB6EC3F308033B6673
:1077440000237B66A74BD7E918452A4603FB02F2C0
:107754000023214601FB03F31344A24A2146A1FB63
:107764000212FA670A46BA67FA6F1344FB67D7F83E
:107774008C300022BB65FA65D7E91623D7E91E01D0
:10778400F8F746FD02460B461346C7F8943064E00A
:10779400924B5B689B0900223B657A653B6DC3F3A2
:1077A4000803BB640023FB64D7E9124522462B4639
:1077B4004FF000004FF00001590141EAD26150013D
:1077C40002460B462146511A3961294663EB0103EF
:1077D4007B614FF000024FF00003D7E904AB594638
:1077E4008B01514643EA916351468A015146B2EBFB
:1077F4000108594663EB01094FF000024FF0000302
:107804004FEAC90343EA58734FEAC80290469946BF
:10781400234618EB0303BB602B4649EB0303FB60D1
:107824004FF000024FF00003D7E9024529468B02CE
:10783400214643EA915321468A0210461946D7F855
:107844008C3000223B647A64D7E91023F8F7E0FC1B
:1078540002460B461346C7F89430604B5B681B0C1A
:1078640003F0030301335B00C7F88830D7F8942092
:10787400D7F88830B2FBF3F3C7F89030A6E0574B43
:107884005B6803F03F03C7F88C30544B5B6803F428
:107894008003002B2AD0514B5B689B090022BB63F9
:1078A400FA63BB6BC3F3080000214E4B03FB01F2E8
:1078B400002300FB03F313444A4AA0FB02127A6735
:1078C4000A463A677A6F13447B67D7F88C300022F4
:1078D4003B637A63D7E90C23D7E91C01F8F798FCDA
:1078E40002460B461346C7F894305BE03B4B5B689B
:1078F4009B090022BB62FA62BB6AC3F308033B62C2
:1079040000237B62D7E9088942464B464FF00000CA
:107914004FF00001590141EAD261500102460B4681
:107924004146B2EB010A494663EB010B4FF00002FA
:107934004FF000034FEA8B1343EA9A634FEA8A122B
:10794400B2EB0A0463EB0B054FF000024FF00003A7
:10795400EB0043EA5473E20014461D464346E31821
:107964003B604B4645EB03037B604FF000024FF056
:107974000003D7E9004529468B02214643EA915387
:1079840021468A0210461946D7F88C300022BB6182
:10799400FA61D7E90623F8F73BFC02460B46134687
:1079A400C7F894300D4B5B681B0F03F00703C7F84F
:1079B4008430D7F89420D7F88430B2FBF3F3C7F8B7
:1079C400903003E0064BC7F8903000BFD7F89030F2
:1079D40018469837BD46BDE8B08F00BF0038024056
:1079E4000024F400001BB70080B586B000AF7860B7
:1079F4007B68002B01D101238DE27B681B6803F0B7
:107A04000103002B00F08380944B9B6803F00C036C
:107A1400042B19D0914B9B6803F00C03082B06D15F
:107A24008E4B5B6803F48003B3F5800F0CD08B4B53
:107A34009B6803F00C030C2B12D1884B5B6803F496
:107A44008003B3F5800F0BD1844B1B6803F4003320
:107A5400002B5BD07B685B68002B57D101235AE273
:107A64007B685B68B3F5803F06D17C4B1B687B4A1F
:107A740043F4803313601DE07B685B68B3F5A02F8B
:107A84000CD1764B1B68754A43F480231360734B07
:107A94001B68724A43F4803313600BE06F4B1B681E
:107AA4006E4A23F4803313606C4B1B686B4A23F4D7
:107AB400802313607B685B68002B13D0FBF72EFADE
:107AC400386108E0FBF72AFA02463B69D31A642BB3
:107AD40001D903231FE2614B1B6803F40033002B1D
:107AE400F0D014E0FBF71AFA386108E0FBF716FA55
:107AF40002463B69D31A642B01D903230BE2574B8B
:107B04001B6803F40033002BF0D100E000BF7B6856
:107B14001B6803F00203002B6FD0504B9B6803F0EB
:107B24000C03002B17D04D4B9B6803F00C03082B60
:107B340005D14A4B5B6803F48003002B0BD0474B01
:107B44009B6803F00C030C2B1CD1444B5B6803F4BF
:107B54008003002B16D1414B1B6803F00203002B5A
:107B640005D07B68DB68012B01D00123D3E13B4BBB
:107B74001B6823F0F8027B681B69DB003749134359
:107B84000B603AE07B68DB68002B20D0344B012289
:107B94001A60FBF7C3F9386108E0FBF7BFF9024646
:107BA4003B69D31A022B01D90323B4E12B4B1B6885
:107BB40003F00203002BF0D0284B1B6823F0F802DB
:107BC4007B681B69DB00254913430B6015E0244BDC
:107BD40000221A60FBF7A2F9386108E0FBF79EF96E
:107BE40002463B69D31A022B01D9032393E11B4BB1
:107BF4001B6803F00203002BF0D17B681B6803F0C1
:107C04000803002B36D07B685B69002B16D0154B1C
:107C140001221A60FBF782F9386108E0FBF77EF96C
:107C240002463B69D31A022B01D9032373E10B4BA0
:107C34005B6F03F00203002BF0D01BE0094B002222
:107C44001A60FBF76BF938610EE0FBF767F902463F
:107C54003B69D31A022B07D903235CE100380240A5
:107C640000004742800E47428A4B5B6F03F00203D9
:107C7400002BEAD17B681B6803F00403002B00F09F
:107C840097800023FB75834B1B6C03F08053002B00
:107C94000FD10023BB607F4B1B6C7E4A43F08053A3
:107CA40013647C4B1B6C03F08053BB60BB680123E3
:107CB400FB75794B1B6803F48073002B18D1764B4A
:107CC4001B68754A43F480731360FBF727F9386126
:107CD40008E0FBF723F902463B69D31A022B01D9CA
:107CE400032318E16C4B1B6803F48073002BF0D062
:107CF4007B689B68012B06D1664B1B6F654A43F07A
:107D0400010313671CE07B689B68052B0CD1614B56
:107D14001B6F604A43F0040313675E4B1B6F5D4A9D
:107D240043F0010313670BE05A4B1B6F594A23F0CE
:107D340001031367574B1B6F564A23F00403136761
:107D44007B689B68002B15D0FBF7E8F838610AE0E4
:107D5400FBF7E4F802463B69D31A41F288329342B6
:107D640001D90323D7E04B4B1B6F03F00203002B15
:107D7400EED014E0FBF7D2F838610AE0FBF7CEF856
:107D840002463B69D31A41F28832934201D9032354
:107D9400C1E0404B1B6F03F00203002BEED1FB7DCF
:107DA400012B05D13B4B1B6C3A4A23F080531364DF
:107DB4007B689B69002B00F0AD80364B9B6803F019
:107DC4000C03082B60D07B689B69022B45D1334B95
:107DD40000221A60FBF7A2F8386108E0FBF79EF86E
:107DE40002463B69D31A022B01D9032393E0294BA2
:107DF4001B6803F00073002BF0D17B68DA697B68A1
:107E04001B6A1A437B685B6A9B011A437B689B6A03
:107E14005B08013B1B041A437B68DB6A1B061A439D
:107E24007B681B6B1B071B4913434B601B4B0122D5
:107E34001A60FBF773F8386108E0FBF76FF8024645
:107E44003B69D31A022B01D9032364E0114B1B684D
:107E540003F00073002BF0D05CE0104B00221A609A
:107E6400FBF75CF8386108E0FBF758F802463B6919
:107E7400D31A022B01D903234DE0064B1B6803F0F0
:107E84000073002BF0D145E07B689B69012B07D17F
:107E9400012340E000380240007000406000474287
:107EA4001F4B5B68FB607B689B69012B30D0FB68D0
:107EB40003F480027B68DB699A4229D1FB6803F0F2
:107EC4003F027B681B6A9A4222D1FA6847F6C07364
:107ED40013407A68526A9201934219D1FB6803F401
:107EE40040327B689B6A5B08013B1B049A420FD1BA
:107EF400FB6803F070627B68DB6A1B069A4207D159
:107F0400FB6803F0E0427B681B6B1B079A4201D0BD
:107F1400012300E0002318461837BD4680BD00BF8A
:107F24000038024080B582B000AF78607B68002BD7
:107F340001D101237BE07B685B6A002B08D17B685D
:107F44005B68B3F5827F09D07B680022DA6105E0C3
:107F54007B6800221A617B6800225A617B680022D8
:107F64009A627B6893F85130DBB2002B06D17B68B0
:107F7400002283F850207868F9F784FC7B68022299
:107F840083F851207B681B681A687B681B6822F0A1
:107F940040021A607B685B6803F482727B689B68AA
:107FA40003F404431A437B68DB6803F400631A4355
:107FB4007B681B6903F002031A437B685B6903F067
:107FC40001031A437B689B6903F400731A437B68BB
:107FD400DB6903F038031A437B681B6A03F08003F0
:107FE40042EA03017B689B6A03F400527B681B68C6
:107FF4000A431A607B689B691B0C03F004017B68CD
:108004005B6A03F010027B681B680A435A607B6852
:108014001B68DA697B681B6822F40062DA617B689A
:1080240000225A657B68012283F8512000231846F8
:108034000837BD4680BD80B588B000AFF860B96030
:108044003B601346FB800023FB77FB6893F85030BA
:10805400012B01D1022326E1FB68012283F8502081
:10806400FAF75CFFB861FB88FB82FB6893F8513038
:10807400DBB2012B02D00223FB770BE1BB68002BA0
:1080840002D0FB88002B02D10123FB7702E1FB68BD
:10809400032283F85120FB6800225A65FB68BA6802
:1080A4001A63FB68FA889A86FB68FA88DA86FB68A2
:1080B40000229A63FB6800229A87FB680022DA8711
:1080C400FB6800225A64FB6800221A64FB689B6800
:1080D400B3F5004F0FD1FB681B681A68FB681B6877
:1080E40022F040021A60FB681B681A68FB681B6870
:1080F40042F480421A60FB681B681B6803F040036B
:10810400402B07D0FB681B681A68FB681B6842F0A9
:1081140040021A60FB68DB68B3F5006F4BD1FB6863
:108124005B68002B02D0FB8A012B3ED1FB681B6BE2
:108134001A88FB681B68DA60FB681B6B9A1CFB6877
:108144001A63FB68DB8E9BB2013B9AB2FB68DA864A
:108154002BE0FB681B689B6803F00203022B12D11F
:10816400FB681B6B1A88FB681B68DA60FB681B6B77
:108174009A1CFB681A63FB68DB8E9BB2013B9AB2C4
:10818400FB68DA8611E0FAF7C9FE0246BB69D31A26
:108194003A689A4203D83B68B3F1FF3F02D13B6887
:1081A400002B02D10323FB7774E0FB68DB8E9BB2C8
:1081B400002BCED14CE0FB685B68002B02D0FB8A1D
:1081C400012B40D1FB681A6BFB681B680C331278D7
:1081D4001A70FB681B6B5A1CFB681A63FB68DB8E06
:1081E4009BB2013B9AB2FB68DA862CE0FB681B6801
:1081F4009B6803F00203022B13D1FB681A6BFB6824
:108204001B680C3312781A70FB681B6B5A1CFB68D2
:108214001A63FB68DB8E9BB2013B9AB2FB68DA8679
:1082240011E0FAF77BFE0246BB69D31A3A689A4218
:1082340003D83B68B3F1FF3F02D13B68002B02D166
:108244000323FB7726E0FB68DB8E9BB2002BCDD1AA
:10825400BA693968F86800F0CBFB0346002B02D0FA
:10826400FB6820225A65FB689B68002B0AD1002317
:108274003B61FB681B68DB683B61FB681B689B68B0
:108284003B613B69FB685B6D002B02D00123FB77EC
:1082940000E000BFFB68012283F85120FB68002244
:1082A40083F85020FB7F18462037BD4680BD80B53B
:1082B40088B002AFF860B9603B601346FB800023CE
:1082C400FB75FB685B68B3F5827F12D1FB689B6822
:1082D400002B0ED1FB68042283F85120FA883B68F6
:1082E40000931346BA68B968F86800F0F1F80346D9
:1082F400EAE0FB6893F85030012B01D10223E3E05C
:10830400FB68012283F85020FAF708FE3861FB6805
:1083140093F85130DBB2012B02D00223FB75CAE083
:10832400BB68002B02D0FB88002B02D10123FB7514
:10833400C1E0FB68042283F85120FB6800225A65DF
:10834400FB68BA689A63FB68FA889A87FB68FA88BC
:10835400DA87FB6800221A63FB6800229A86FB68AE
:108364000022DA86FB6800221A64FB6800225A6441
:10837400FB689B68B3F5004F0FD1FB681B681A6854
:10838400FB681B6822F040021A60FB681B681A68CD
:10839400FB681B6822F480421A60FB681B681B6838
:1083A40003F04003402B07D0FB681B681A68FB6886
:1083B4001B6842F040021A60FB68DB68002B62D144
:1083C4002EE0FB681B689B6803F00103012B15D1A9
:1083D400FB681B6803F10C02FB689B6B1278D2B23A
:1083E4001A70FB689B6B5A1CFB689A63FB68DB8FF3
:1083F4009BB2013B9AB2FB68DA8711E0FAF78EFD73
:1084040002463B69D31A3A689A4203D83B68B3F1EF
:10841400FF3F02D13B68002B02D10323FB754AE0E6
:10842400FB68DB8F9BB2002BCBD131E0FB681B6870
:108434009B6803F00103012B13D1FB681B68DA6806
:10844400FB689B6B92B21A80FB689B6B9A1CFB685F
:108454009A63FB68DB8F9BB2013B9AB2FB68DA87B5
:1084640011E0FAF75BFD02463B69D31A3A689A4277
:1084740003D83B68B3F1FF3F02D13B68002B02D124
:108484000323FB7517E0FB68DB8F9BB2002BCDD178
:108494003A693968F86800F045FA0346002B02D0BF
:1084A400FB6820225A65FB685B6D002B02D0012318
:1084B400FB7500E000BFFB68012283F85120FB68D4
:1084C400002283F85020FB7D18461837BD4680BD36
:1084D40080B58CB000AFF860B9607A607B8001230E
:1084E400FB62002387F82B30FB6893F85030012B94
:1084F40001D102238AE1FB68012283F85020FAF7B4
:108504000DFD7862FB6893F8513087F82330FB68DF
:108514005B68FB617B887B8397F82330012B0FD04A
:10852400FB69B3F5827F07D1FB689B68002B03D1FD
:1085340097F82330042B03D0022387F82B305BE118
:10854400BB68002B05D07B68002B02D07B88002BF6
:1085540003D1012387F82B304EE1FB6893F85130A7
:10856400DBB2042B03D0FB68052283F85120FB689F
:1085740000225A65FB687A689A63FB687A88DA870E
:10858400FB687A889A87FB68BA681A63FB687A88FA
:10859400DA86FB687A889A86FB6800221A64FB688C
:1085A40000225A64FB681B681B6803F04003402BDD
:1085B40007D0FB681B681A68FB681B6842F040021E
:1085C4001A60FB68DB68B3F5006F78D1FB685B6801
:1085D400002B02D07B8B012B66D1FB681B6B1A88A6
:1085E400FB681B68DA60FB681B6B9A1CFB681A63E8
:1085F400FB68DB8E9BB2013B9AB2FB68DA8653E0E0
:10860400FB681B689B6803F00203022B1BD1FB6809
:10861400DB8E9BB2002B16D0FB6A012B13D1FB68B7
:108624001B6B1A88FB681B68DA60FB681B6B9A1C5F
:10863400FB681A63FB68DB8E9BB2013B9AB2FB6852
:10864400DA860023FB62FB681B689B6803F0010366
:10865400012B19D1FB68DB8F9BB2002B14D0FB6874
:108664001B68DA68FB689B6B92B21A80FB689B6B91
:108674009A1CFB689A63FB68DB8F9BB2013B9AB23E
:10868400FB68DA870123FB62FAF748FC02467B6A3F
:10869400D31ABA6B9A4207D8BB6BB3F1FF3F03D02E
:1086A400032387F82B30A7E0FB68DB8E9BB2002BFB
:1086B400A6D1FB68DB8F9BB2002BA1D17CE0FB68C9
:1086C4005B68002B02D07B8B012B6BD1FB681A6B90
:1086D400FB681B680C3312781A70FB681B6B5A1CFE
:1086E400FB681A63FB68DB8E9BB2013B9AB2FB68A2
:1086F400DA8657E0FB681B689B6803F00203022BD1
:108704001CD1FB68DB8E9BB2002B17D0FB6A012BBC
:1087140014D1FB681A6BFB681B680C3312781A704F
:10872400FB681B6B5A1CFB681A63FB68DB8E9BB2ED
:10873400013B9AB2FB68DA860023FB62FB681B6884
:108744009B6803F00103012B19D1FB68DB8F9BB2FB
:10875400002B14D0FB681B68DA68FB689B6BD2B2F1
:108764001A70FB689B6B5A1CFB689A63FB68DB8F6F
:108774009BB2013B9AB2FB68DA870123FB62FAF7EA
:10878400CDFB02467B6AD31ABA6B9A4203D8BB6B01
:10879400B3F1FF3F02D1BB6B002B03D1032387F856
:1087A4002B3029E0FB68DB8E9BB2002BA2D1FB6847
:1087B400DB8F9BB2002B9DD17A6AB96BF86800F00D
:1087C40017F90346002B06D0012387F82B30FB68EA
:1087D40020225A6510E0FB689B68002B0BD1002314
:1087E4007B61FB681B68DB687B61FB681B689B68BB
:1087F4007B617B6900E000BFFB68012283F85120A4
:10880400FB68002283F8502097F82B301846303745
:10881400BD4680BD80B588B000AFF860B9603B60EC
:108824001346FB71FAF77AFB0246BB6A9B1A3A6855
:108834001344FB61FAF772FBB861394B1B685B01A7
:108844001B0DFA6902FB03F37B6154E03B68B3F14F
:10885400FF3F50D0FAF762FB0246BB69D31AFA69AC
:108864009A4202D9FB69002B3DD1FB681B685A6808
:10887400FB681B6822F0E0025A60FB685B68B3F592
:10888400827F11D1FB689B68B3F5004F04D0FB686D
:108894009B68B3F5806F07D1FB681B681A68FB6897
:1088A4001B6822F040021A60FB689B6AB3F5005F04
:1088B4000FD1FB681B681A68FB681B6822F400521E
:1088C4001A60FB681B681A68FB681B6842F4005254
:1088D4001A60FB68012283F85120FB68002283F8A8
:1088E4005020032317E07B69002B01D10023FB6197
:1088F4007B69013B7B61FB681B689A68BB6813401A
:10890400BA689A420CBF01230023DBB21A46FB79F2
:108914009A429BD1002318462037BD4680BD00BF34
:108924000C00002080B586B002AFF860B9607A60B0
:10893400FB685B68B3F5827F11D1FB689B68B3F574
:10894400004F04D0FB689B68B3F5806F07D1FB68C8
:108954001B681A68FB681B6822F040021A60FB68F7
:108964005B68B3F5827F2AD1FB689B68B3F5806F9F
:1089740012D07B680093BB6800228021F868FFF75F
:1089840049FF0346002B2DD0FB685B6D43F02002AA
:10899400FB685A65032326E07B680093BB680022CA
:1089A4000121F868FFF736FF0346002B1AD0FB6855
:1089B4005B6D43F02002FB685A65032313E07B6878
:1089C4000093BB6800220121F868FFF723FF0346E8
:1089D400002B07D0FB685B6D43F02002FB685A65EF
:1089E400032300E0002318461037BD4680BD000075
:1089F40080B588B002AFF860B9607A601B4B1B6821
:108A04001B4AA2FB03235B0D4FF47A7202FB03F3B0
:108A14007B61FB685B68B3F5827F12D17B6800934E
:108A2400BB6800228021F868FFF7F4FE0346002BA0
:108A340016D0FB685B6D43F02002FB685A65032384
:108A44000FE07B69002B0AD07B69013B7B61FB68EB
:108A54001B689B6803F08003802BF2D000E000BF0A
:108A6400002318461837BD4680BD00BF0C00002007
:108A7400819F5E1680B582B000AF78607B68002B62
:108A840001D1012341E07B6893F83D30DBB2002B38
:108A940006D17B68002283F83C207868F9F748FC0B
:108AA4007B68022283F83D207B681A687B68043364
:108AB4001946104600F07AFC7B68012283F84620B0
:108AC4007B68012283F83E207B68012283F83F20E3
:108AD4007B68012283F840207B68012283F84120CF
:108AE4007B68012283F842207B68012283F84320BB
:108AF4007B68012283F844207B68012283F84520A7
:108B04007B68012283F83D20002318460837BD46C0
:108B140080BD000080B485B000AF78607B6893F8B6
:108B24003D30DBB2012B01D001234EE07B680222F1
:108B340083F83D207B681B68DA687B681B6842F019
:108B44000102DA607B681B68234A934222D07B6867
:108B54001B68B3F1804F1DD07B681B681F4A93428A
:108B640018D07B681B681E4A934213D07B681B682D
:108B74001C4A93420ED07B681B681B4A934209D05F
:108B84007B681B68194A934204D07B681B68184AA7
:108B9400934211D17B681B689B6803F00703FB6059
:108BA400FB68062B10D07B681B681A687B681B68FF
:108BB40042F001021A6007E07B681B681A687B6850
:108BC4001B6842F001021A60002318461437BD46A0
:108BD4005DF8047B704700BF0000014000040040C2
:108BE40000080040000C0040000401400040014027
:108BF4000018004080B582B000AF78607B68002B1D
:108C040001D1012341E07B6893F83D30DBB2002BB6
:108C140006D17B68002283F83C20786800F039F89C
:108C24007B68022283F83D207B681A687B680433E2
:108C34001946104600F0BAFB7B68012283F84620EF
:108C44007B68012283F83E207B68012283F83F2061
:108C54007B68012283F840207B68012283F841204D
:108C64007B68012283F842207B68012283F8432039
:108C74007B68012283F844207B68012283F8452025
:108C84007B68012283F83D20002318460837BD463F
:108C940080BD80B483B000AF786000BF0C37BD46A0
:108CA4005DF8047B7047000080B584B000AF786045
:108CB40039603B68002B09D17B6893F83E30DBB206
:108CC400012B14BF01230023DBB222E03B68042BF9
:108CD40009D17B6893F83F30DBB2012B14BF012329
:108CE4000023DBB215E03B68082B09D17B6893F8BD
:108CF4004030DBB2012B14BF01230023DBB208E0B8
:108D04007B6893F84130DBB2012B14BF01230023AD
:108D1400DBB2002B01D001237CE03B68002B04D1A3
:108D24007B68022283F83E2013E03B68042B04D1C5
:108D34007B68022283F83F200BE03B68082B04D1B8
:108D44007B68022283F8402003E07B68022283F8D8
:108D540041207B681B6801223968184600F010FE28
:108D64007B681B682D4A934204D07B681B682C4A9D
:108D7400934201D1012300E00023002B07D07B683C
:108D84001B685A6C7B681B6842F400425A647B6817
:108D94001B68224A934222D07B681B68B3F1804F40
:108DA4001DD07B681B681F4A934218D07B681B68E0
:108DB4001D4A934213D07B681B681C4A93420ED011
:108DC4007B681B68164A934209D07B681B68184A63
:108DD400934204D07B681B68164A934211D17B6886
:108DE4001B689B6803F00703FB60FB68062B10D02D
:108DF4007B681B681A687B681B6842F001021A6072
:108E040007E07B681B681A687B681B6842F00102F4
:108E14001A60002318461037BD4680BD000001408B
:108E2400000401400004004000080040000C004021
:108E3400004001400018004080B582B000AF786067
:108E44007B681B681B6903F00203022B22D17B6839
:108E54001B68DB6803F00203022B1BD17B681B68D1
:108E64006FF002021A617B6801221A777B681B6823
:108E74009B6903F00303002B03D0786800F077FAB2
:108E840005E0786800F069FA786800F07AFA7B689F
:108E940000221A777B681B681B6903F00403042B08
:108EA40022D17B681B68DB6803F00403042B1BD10D
:108EB4007B681B686FF004021A617B6802221A77D0
:108EC4007B681B689B6903F44073002B03D07868AC
:108ED40000F04DFA05E0786800F03FFA786800F099
:108EE40050FA7B6800221A777B681B681B6903F0C1
:108EF4000803082B22D17B681B68DB6803F0080396
:108F0400082B1BD17B681B686FF008021A617B6811
:108F140004221A777B681B68DB6903F00303002BC8
:108F240003D0786800F023FA05E0786800F015FAB9
:108F3400786800F026FA7B6800221A777B681B6841
:108F44001B6903F01003102B22D17B681B68DB68BC
:108F540003F01003102B1BD17B681B686FF0100209
:108F64001A617B6808221A777B681B68DB6903F443
:108F74004073002B03D0786800F0F9F905E07868B5
:108F840000F0EBF9786800F0FCF97B6800221A77AE
:108F94007B681B681B6903F00103012B0ED17B68FE
:108FA4001B68DB6803F00103012B07D17B681B6896
:108FB4006FF001021A617868F8F75AFB7B681B6846
:108FC4001B6903F08003802B0ED17B681B68DB6870
:108FD40003F08003802B07D17B681B686FF080024D
:108FE4001A61786800F0CAFD7B681B681B6903F08E
:108FF4004003402B0ED17B681B68DB6803F0400301
:10900400402B07D17B681B686FF040021A617868B7
:1090140000F0C1F97B681B681B6903F02003202B57
:109024000ED17B681B68DB6803F02003202B07D17B
:109034007B681B686FF020021A61786800F094FD69
:1090440000BF0837BD4680BD80B586B000AFF8606C
:10905400B9607A600023FB75FB6893F83C30012B00
:1090640001D10223AEE0FB68012283F83C207B6837
:109074000C2B00F29F8001A252F823F0B590000857
:10908400B9910008B9910008B9910008F590000859
:10909400B9910008B9910008B99100083791000806
:1090A400B9910008B9910008B991000877910008B6
:1090B400FB681B68B968184600F018FAFB681B685F
:1090C4009A69FB681B6842F008029A61FB681B6896
:1090D4009A69FB681B6822F004029A61FB681B68AA
:1090E4009969BB681A69FB681B680A439A6164E062
:1090F400FB681B68B968184600F068FAFB681B68CF
:109104009A69FB681B6842F400629A61FB681B68F9
:109114009A69FB681B6822F480629A61FB681B6889
:109124009969BB681B691A02FB681B680A439A6148
:1091340043E0FB681B68B968184600F0BDFAFB6899
:109144001B68DA69FB681B6842F00802DA61FB6895
:109154001B68DA69FB681B6822F00402DA61FB68A9
:109164001B68D969BB681A69FB681B680A43DA6122
:1091740023E0FB681B68B968184600F011FBFB6824
:109184001B68DA69FB681B6842F40062DA61FB68F9
:109194001B68DA69FB681B6822F48062DA61FB6889
:1091A4001B68D969BB681B691A02FB681B680A4300
:1091B400DA6102E00123FB7500BFFB68002283F83B
:1091C4003C20FB7D18461837BD4680BD80B584B071
:1091D40000AF786039600023FB737B6893F83C3000
:1091E400012B01D10223B4E07B68012283F83C20E7
:1091F4007B68022283F83D207B681B689B68BB6008
:10920400BB6823F07703BB60BB6823F47F43BB6078
:109214007B681B68BA689A603B681B68B3F5005F9B
:109224003ED0B3F5005F00F28780B3F5805F00F0B5
:109234008680B3F5805F7FD8702B1AD0702B7BD8D3
:10924400602B50D0602B77D8502B3CD0502B73D848
:10925400402B58D0402B6FD8302B64D0302B6BD898
:10926400202B60D0202B67D8002B5CD0102B5AD039
:1092740062E07B6818683B6899683B685A683B6899
:10928400DB6800F05DFB7B681B689B68BB60BB68A8
:1092940043F07703BB607B681B68BA689A604FE051
:1092A4007B6818683B6899683B685A683B68DB6868
:1092B40000F046FB7B681B689A687B681B6842F475
:1092C40080429A603CE07B6818683B6859683B6858
:1092D400DB681A4600F0BAFA7B681B68502118460E
:1092E40000F013FB2CE07B6818683B6859683B6806
:1092F400DB681A4600F0D9FA7B681B6860211846BF
:1093040000F003FB1CE07B6818683B6859683B6805
:10931400DB681A4600F09AFA7B681B6840211846FD
:1093240000F0F3FA0CE07B681A683B681B68194686
:10933400104600F0EAFA03E00123FB7300E000BFEB
:109344007B68012283F83D207B68002283F83C205F
:10935400FB7B18461037BD4680BD80B483B000AF98
:10936400786000BF0C37BD465DF8047B704780B45D
:1093740083B000AF786000BF0C37BD465DF8047B56
:10938400704780B483B000AF786000BF0C37BD462F
:109394005DF8047B704780B483B000AF786000BF91
:1093A4000C37BD465DF8047B7047000080B485B07F
:1093B40000AF786039607B681B68FB607B68404A5B
:1093C400934213D07B68B3F1804F0FD07B683D4A42
:1093D40093420BD07B683C4A934207D07B683B4A5C
:1093E400934203D07B683A4A934208D1FB6823F046
:1093F4007003FB603B685B68FA681343FB607B683F
:109404002F4A93422BD07B68B3F1804F27D07B68DF
:109414002C4A934223D07B682B4A93421FD07B680B
:109424002A4A93421BD07B68294A934217D07B680F
:10943400284A934213D07B68274A93420FD07B6813
:10944400264A93420BD07B68254A934207D07B6817
:10945400244A934203D07B68234A934208D1FB6891
:1094640023F44073FB603B68DB68FA681343FB60DA
:10947400FB6823F080023B685B691343FB607B68F5
:10948400FA681A603B689A687B68DA623B681A6813
:109494007B689A627B680A4A934203D07B680C4AD1
:1094A400934203D13B681A697B681A637B68012283
:1094B4005A6100BF1437BD465DF8047B704700BF96
:1094C400000001400004004000080040000C00407F
:1094D40000040140004001400044014000480140B4
:1094E40000180040001C00400020004080B487B0F9
:1094F40000AF786039607B681B6A23F001027B68E7
:109504001A627B681B6A7B617B685B683B617B6872
:109514009B69FB60FB6823F07003FB60FB6823F02E
:109524000303FB603B681B68FA681343FB607B69B9
:1095340023F002037B613B689B687A6913437B6178
:109544007B68204A934203D07B681F4A93420CD124
:109554007B6923F008037B613B68DB687A6913430A
:109564007B617B6923F004037B617B68154A93422A
:1095740003D07B68144A934211D13B6923F480736E
:109584003B613B6923F400733B613B685B693A6967
:1095940013433B613B689B693A6913433B617B68B6
:1095A4003A695A607B68FA689A613B685A687B68D2
:1095B4005A637B687A691A6200BF1C37BD465DF83E
:1095C400047B7047000001400004014080B487B070
:1095D40000AF786039607B681B6A23F010027B68F7
:1095E4001A627B681B6A7B617B685B683B617B6892
:1095F4009B69FB60FB6823F4E043FB60FB6823F496
:109604004073FB603B681B681B02FA681343FB60F2
:109614007B6923F020037B613B689B681B017A69AB
:1096240013437B617B68224A934203D07B68214ABF
:1096340093420DD17B6923F080037B613B68DB6837
:109644001B017A6913437B617B6923F040037B61CF
:109654007B68174A934203D07B68164A934213D11E
:109664003B6923F480633B613B6923F400633B6102
:109674003B685B699B003A6913433B613B689B69A8
:109684009B003A6913433B617B683A695A607B6883
:10969400FA689A613B685A687B689A637B687A695E
:1096A4001A6200BF1C37BD465DF8047B704700BFDB
:1096B400000001400004014080B487B000AF78602E
:1096C40039607B681B6A23F480727B681A627B684A
:1096D4001B6A7B617B685B683B617B68DB69FB6061
:1096E400FB6823F07003FB60FB6823F00303FB605B
:1096F4003B681B68FA681343FB607B6923F40073BF
:109704007B613B689B681B027A6913437B617B68BE
:10971400214A934203D07B68204A93420DD17B694E
:1097240023F400637B613B68DB681B027A691343A3
:109734007B617B6923F480637B617B68164A934277
:1097440003D07B68154A934213D13B6923F48053B9
:109754003B613B6923F400533B613B685B691B013C
:109764003A6913433B613B689B691B013A691343A4
:109774003B617B683A695A607B68FA68DA613B68E6
:109784005A687B68DA637B687A691A6200BF1C379F
:10979400BD465DF8047B70470000014000040140B1
:1097A40080B487B000AF786039607B681B6A23F4AB
:1097B40080527B681A627B681B6A3B617B685B68CA
:1097C4007B617B68DB69FB60FB6823F4E043FB603F
:1097D400FB6823F44073FB603B681B681B02FA6858
:1097E4001343FB603B6923F400533B613B689B6874
:1097F4001B033A6913433B617B68124A934203D0CB
:109804007B68114A934209D17B6923F480437B61CD
:109814003B685B699B017A6913437B617B687A6966
:109824005A607B68FA68DA613B685A687B681A6434
:109834007B683A691A6200BF1C37BD465DF8047B39
:10984400704700BF000001400004014080B487B0AD
:1098540000AFF860B9607A60FB681B6A7B61FB68E3
:109864001B6A23F00102FB681A62FB689B693B6177
:109874003B6923F0F0033B617B681B013A691343A6
:109884003B617B6923F00A037B617A69BB681343FC
:109894007B61FB683A699A61FB687A691A6200BF66
:1098A4001C37BD465DF8047B704780B487B000AFB9
:1098B400F860B9607A60FB681B6A23F01002FB68E9
:1098C4001A62FB689B697B61FB681B6A3B617B696D
:1098D40023F470437B617B681B037A6913437B61C8
:1098E4003B6923F0A0033B61BB681B013A69134346
:1098F4003B61FB687A699A61FB683A691A6200BF46
:109904001C37BD465DF8047B704780B485B000AF5A
:10991400786039607B689B68FB60FB6823F07003A8
:10992400FB603A68FB68134343F00703FB607B6802
:10993400FA689A6000BF1437BD465DF8047B70472F
:1099440080B487B000AFF860B9607A603B60FB68B0
:109954009B687B617B6923F47F437B613B681A02CC
:109964007B681A43BB6813437A6913437B61FB68C2
:109974007A699A6000BF1C37BD465DF8047B704766
:1099840080B487B000AFF860B9607A60BB6803F058
:109994001F03012202FA03F37B61FB681A6A7B69E5
:1099A400DB431A40FB681A62FB681A6ABB6803F05F
:1099B4001F03796801FA03F31A43FB681A6200BFB4
:1099C4001C37BD465DF8047B7047000080B485B049
:1099D40000AF786039607B6893F83C30012B01D18B
:1099E40002235AE07B68012283F83C207B68022230
:1099F40083F83D207B681B685B68FB607B681B68A1
:109A04009B68BB60FB6823F07003FB603B681B68CA
:109A1400FA681343FB607B681B68FA685A607B68CA
:109A24001B68214A934222D07B681B68B3F1804FA4
:109A34001DD07B681B681D4A934218D07B681B6845
:109A44001B4A934213D07B681B681A4A93420ED078
:109A54007B681B68184A934209D07B681B68174AC5
:109A6400934204D07B681B68154A93420CD1BB68AF
:109A740023F08003BB603B685B68BA681343BB6038
:109A84007B681B68BA689A607B68012283F83D2072
:109A94007B68002283F83C20002318461437BD4617
:109AA4005DF8047B704700BF0000014000040040E3
:109AB40000080040000C0040000401400040014048
:109AC4000018004080B485B000AF7860396000238E
:109AD400FB607B6893F83C30012B01D102233DE00D
:109AE4007B68012283F83C20FB6823F0FF023B687B
:109AF400DB681343FB60FB6823F440723B689B689C
:109B04001343FB60FB6823F480623B685B68134388
:109B1400FB60FB6823F400623B681B681343FB6033
:109B2400FB6823F480523B681B691343FB60FB68AA
:109B340023F400523B685B691343FB60FB6823F426
:109B440080423B68DB691343FB607B681B68FA68EF
:109B54005A647B68002283F83C200023184614379B
:109B6400BD465DF8047B704780B483B000AF786075
:109B740000BF0C37BD465DF8047B704780B483B0EA
:109B840000AF786000BF0C37BD465DF8047B7047BA
:109B940080B582B000AF78607B68002B01D10123CF
:109BA4003FE07B6893F83D30DBB2002B06D17B6845
:109BB400002283F83C207868F8F79CFF7B68242215
:109BC40083F83D207B681B68DA687B681B6822F495
:109BD4000052DA60786800F043FF7B681B681A69FA
:109BE4007B681B6822F490421A617B681B685A697F
:109BF4007B681B6822F02A025A617B681B68DA685A
:109C04007B681B6842F40052DA607B6800221A64A5
:109C14007B68202283F83D207B68202283F83E2045
:109C2400002318460837BD4680BD000080B58CB0BF
:109C340000AFF860B9601346FB80FB6893F83D30D1
:109C4400DBB2202B65D1BB68002B02D0FB88002B34
:109C540001D101235EE0FB6893F83C30012B01D174
:109C6400022357E0FB68012283F83C20BA68FB68B2
:109C74001A62FB68FA889A84FB68FA88DA84FB68BB
:109C840000221A64FB68212283F83D20FB685B6B89
:109C9400224ADA63FB685B6B214A1A64FB685B6BDC
:109CA400204ADA64FB685B6B00221A6507F108033B
:109CB400FB62FB68586BFB6A1968FB681B6804331A
:109CC4001A46FB88FAF79CF8FB681B686FF04002A1
:109CD4001A60FB68002283F83C20FB681B6814337D
:109CE400BB61BB6953E8003F7B617B6943F0800340
:109CF400BB62FB681B681433BA6A7A623B62396AD6
:109D04007A6A41E80023FB61FB69002BE5D100235B
:109D140000E0022318463037BD4680BDFDA200088E
:109D240097A300080FA5000880B584B000AFF860C1
:109D3400B9601346FB80FB6893F83E30DBB2202BFE
:109D44001DD1BB68002B02D0FB88002B01D101235D
:109D540016E0FB6893F83C30012B01D102230FE09D
:109D6400FB68012283F83C20FB6800221A63FB880D
:109D74001A46B968F86800F013FC034600E00223B1
:109D840018461037BD4680BD80B5BAB000AF7860C4
:109D94007B681B681B68C7F8E4307B681B68DB685A
:109DA400C7F8E0307B681B685B69C7F8DC300023C8
:109DB400C7F8D8300023C7F8D430D7F8E43003F01C
:109DC4000F03C7F8D830D7F8D830002B0FD1D7F805
:109DD400E43003F02003002B09D0D7F8E03003F07F
:109DE4002003002B03D0786800F07FFD56E2D7F8FB
:109DF400D830002B00F0DE80D7F8DC3003F001030C
:109E0400002B06D1D7F8E03003F49073002B00F058
:109E1400D180D7F8E43003F00103002B0BD0D7F83E
:109E2400E03003F48073002B05D07B681B6C43F097
:109E340001027B681A64D7F8E43003F00403002BB2
:109E44000BD0D7F8DC3003F00103002B05D07B687E
:109E54001B6C43F002027B681A64D7F8E43003F009
:109E64000203002B0BD0D7F8DC3003F00103002BE6
:109E740005D07B681B6C43F004027B681A64D7F836
:109E8400E43003F00803002B11D0D7F8E03003F0DE
:109E94002003002B05D1D7F8DC3003F00103002B9D
:109EA40005D07B681B6C43F008027B681A647B68EE
:109EB4001B6C002B00F0ED81D7F8E43003F0200395
:109EC400002B08D0D7F8E03003F02003002B02D099
:109ED400786800F00AFD7B681B685B6903F0400347
:109EE400402B0CBF01230023DBB2C7F8D4307B68BE
:109EF4001B6C03F00803002B03D1D7F8D430002BDC
:109F04004FD0786800F012FC7B681B685B6903F033
:109F14004003402B41D17B681B681433C7F89C3045
:109F2400D7F89C3053E8003FC7F89830D7F89830FA
:109F340023F04003C7F8D0307B681B681433D7F88C
:109F4400D020C7F8A820C7F8A430D7F8A410D7F8B1
:109F5400A82041E80023C7F8A030D7F8A030002B90
:109F6400D9D17B689B6B002B13D07B689B6B7D4A9C
:109F74001A657B689B6B1846FAF70AF80346002BB0
:109F840016D07B689B6B1B6D7A68926B1046984762
:109F94000EE0786800F09AF90AE0786800F096F923
:109FA40006E0786800F092F97B6800221A6470E198
:109FB40000BF6EE17B681B6B012B40F04A81D7F830
:109FC400E43003F01003002B00F04381D7F8E030B5
:109FD40003F01003002B00F03C810023BB607B687E
:109FE4001B681B68BB607B681B685B68BB60BB68E5
:109FF4007B681B685B6903F04003402B40F0B4802E
:10A004007B689B6B1B685B68A7F8BE30B7F8BE30F3
:10A01400002B00F040817B689B8DB7F8BE209A42EC
:10A0240080F039817B68B7F8BE20DA857B689B6B4A
:10A03400DB69B3F5807F00F088807B681B680C3394
:10A04400C7F88830D7F8883053E8003FC7F8843021
:10A05400D7F8843023F48073C7F8B8307B681B6862
:10A064000C33D7F8B820C7F89420C7F89030D7F845
:10A074009010D7F8942041E80023C7F88C30D7F823
:10A084008C30002BD9D17B681B6814337B677B6FC2
:10A0940053E8003F3B673B6F23F00103C7F8B4303C
:10A0A4007B681B681433D7F8B420C7F88020FB679B
:10A0B400F96FD7F8802041E80023BB67BB6F002B02
:10A0C400E1D17B681B6814333B663B6E53E8003F69
:10A0D400FB65FB6D23F04003C7F8B0307B681B6859
:10A0E4001433D7F8B020FA66BB66B96EFA6E41E84D
:10A0F40000237B667B6E002BE3D17B68202283F8F0
:10A104003E207B6800221A637B681B680C33FB6467
:10A11400FB6C53E8003FBB64BB6C23F01003C7F82F
:10A12400AC307B681B680C33D7F8AC20BA657B6510
:10A13400796DBA6D41E800233B653B6D002BE3D19B
:10A144007B689B6B1846F9F7B3FE7B689A8D7B6836
:10A15400DB8D9BB2D31A9BB21946786800F0C0F825
:10A1640099E000BFF7A700087B689A8D7B68DB8DB8
:10A174009BB2D31AA7F8CE307B68DB8D9BB2002B41
:10A1840000F08B80B7F8CE30002B00F086807B681F
:10A194001B680C33BB63BB6B53E8003F7B637B6B77
:10A1A40023F49073C7F8C8307B681B680C33D7F866
:10A1B400C8207A643B64396C7A6C41E80023FB6301
:10A1C400FB6B002BE3D17B681B6814337B627B6AD7
:10A1D40053E8003F3B623B6A23F00103C7F8C430F5
:10A1E4007B681B681433D7F8C4203A63FB62F96AAE
:10A1F4003A6B41E80023BB62BB6A002BE3D17B6866
:10A20400202283F83E207B6800221A637B681B6847
:10A214000C333B613B6953E8003FFB60FB6823F070
:10A224001003C7F8C0307B681B680C33D7F8C02014
:10A23400FA61BB61B969FA6941E800237B617B6912
:10A24400002BE3D1B7F8CE301946786800F048F80F
:10A2540023E0D7F8E43003F08003002B09D0D7F8CB
:10A26400E03003F08003002B03D0786800F0D5FAC7
:10A2740014E0D7F8E43003F04003002B0ED0D7F8F5
:10A28400E03003F04003002B08D0786800F015FBA1
:10A2940004E000BF02E000BF00E000BFE837BD46B5
:10A2A40080BD00BF80B483B000AF786000BF0C37BE
:10A2B400BD465DF8047B704780B483B000AF78601E
:10A2C40000BF0C37BD465DF8047B704780B483B093
:10A2D40000AF786000BF0C37BD465DF8047B704763
:10A2E40080B483B000AF78600B467B8000BF0C372E
:10A2F400BD465DF8047B704780B590B000AF7860D0
:10A304007B689B6BFB637B681B681B6803F480732F
:10A31400002B37D1FB6B0022DA84FB6B1B681433F0
:10A324007B627B6A53E8003F3B623B6A23F0800315
:10A33400BB63FB6B1B681433BA6B3A63FB62F96A49
:10A344003A6B41E80023BB62BB6A002BE5D1FB6B8F
:10A354001B680C333B613B6953E8003FFB60FB68BF
:10A3640043F040037B63FB6B1B680C337A6BFA612D
:10A37400BB61B969FA6941E800237B617B69002B01
:10A38400E5D102E0F86BF8F769FC00BF4037BD4641
:10A3940080BD80B584B000AF78607B689B6BFB6048
:10A3A400F868FFF77FFF00BF1037BD4680BD80B55A
:10A3B4009CB000AF78607B689B6BFB667B681B6816
:10A3C4001B6803F48073002B72D1FB6E0022DA85C4
:10A3D400FB6E1B680C33FB64FB6C53E8003FBB64EF
:10A3E400BB6C23F48073BB66FB6E1B680C33BA6EC4
:10A3F400BA657B65796DBA6D41E800233B653B6DB9
:10A40400002BE5D1FB6E1B681433BB63BB6B53E8B5
:10A41400003F7B637B6B23F001037B66FB6E1B6851
:10A4240014337A6E7A643B64396C7A6C41E80023A5
:10A43400FB63FB6B002BE5D1FB6E1B6814337B6263
:10A444007B6A53E8003F3B623B6A23F040033B6670
:10A45400FB6E1B6814333A6E3A63FB62F96A3A6B1B
:10A4640041E80023BB62BB6A002BE5D1FB6E2022CE
:10A4740083F83E20FB6E1B6B012B19D1FB6E1B680E
:10A484000C333B613B6953E8003FFB60FB6823F0FE
:10A494001003FB65FB6E1B680C33FA6DFA61BB613C
:10A4A400B969FA6941E800237B617B69002BE5D136
:10A4B400FB6E1B6B012B06D1FB6E9B8D1946F86E50
:10A4C400FFF70EFF02E0F86EF8F7EAFB00BF703703
:10A4D400BD4680BD80B584B000AF78607B689B6B5F
:10A4E400FB60FB681B6B012B08D1FB689B8D5B0831
:10A4F4009BB21946F868FFF7F3FE02E0F868FFF72D
:10A50400DBFE00BF1037BD4680BD80B584B000AF10
:10A5140078600023FB607B689B6BBB60BB681B6837
:10A524005B6903F08003802B0CBF01230023DBB2A3
:10A53400FB60BB6893F83D30DBB2212B08D1FB688C
:10A54400002B05D0BB680022DA84B86800F0C6F896
:10A55400BB681B685B6903F04003402B0CBF0123FD
:10A564000023DBB2FB60BB6893F83E30DBB2222BE6
:10A5740008D1FB68002B05D0BB680022DA85B868D7
:10A5840000F0D4F8BB681B6C43F01002BB681A647B
:10A59400B868FFF79BFE00BF1037BD4680BD0000C2
:10A5A40080B598B000AFF860B9601346FB80BA6814
:10A5B400FB689A62FB68FA889A85FB6800221A6431
:10A5C400FB68222283F83E20FB689B6B404ADA63D7
:10A5D400FB689B6B3F4A1A64FB689B6B3E4ADA64D8
:10A5E400FB689B6B00221A6507F10803FB65FB6897
:10A5F400986BFB681B6804331946FB6D1A68FB886B
:10A60400F9F7FEFB00233B61FB681B681B683B6199
:10A61400FB681B685B683B613B69FB68002283F84D
:10A624003C20FB681B69002B19D0FB681B680C33AA
:10A634003B643B6C53E8003FFB63FB6B43F4807368
:10A64400BB65FB681B680C33BA6DFA64BB64B96CF8
:10A65400FA6C41E800237B647B6C002BE5D1FB683A
:10A664001B681433FB62FB6A53E8003FBB62BB6A9E
:10A6740043F001037B65FB681B6814337A6DBA638E
:10A684007B63796BBA6B41E800233B633B6B002B24
:10A69400E5D1FB681B681433BB61BB6953E8003F19
:10A6A4007B617B6943F040033B65FB681B681433A3
:10A6B4003A6D7A623B62396A7A6A41E80023FB6147
:10A6C400FB69002BE5D1002318466037BD4680BDE9
:10A6D400B3A30008D9A400080FA5000880B489B06A
:10A6E40000AF78607B681B680C33FB60FB6853E841
:10A6F400003FBB60BB6823F0C003FB617B681B6841
:10A704000C33FA69BA617B617969BA6941E800235B
:10A714003B613B69002BE5D17B68202283F83D2017
:10A7240000BF2437BD465DF8047B704780B495B004
:10A7340000AF78607B681B680C337B637B6B53E8EA
:10A74400003F3B633B6B23F49073FB647B681B68A3
:10A754000C33FA6C3A64FB63F96B3A6C41E80023FE
:10A76400BB63BB6B002BE5D17B681B6814333B6276
:10A774003B6A53E8003FFB61FB6923F00103BB64C0
:10A784007B681B681433BA6CFA62BB62B96AFA6AF2
:10A7940041E800237B627B6A002BE5D17B681B6B5D
:10A7A400012B19D17B681B680C33FB60FB6853E8F1
:10A7B400003FBB60BB6823F010037B647B681B68AD
:10A7C4000C337A6CBA617B617969BA6941E8002318
:10A7D4003B613B69002BE5D17B68202283F83E2056
:10A7E4007B6800221A6300BF5437BD465DF8047BC2
:10A7F400704780B584B000AF78607B689B6BFB606A
:10A80400FB680022DA85FB680022DA84F868FFF727
:10A814005DFD00BF1037BD4680BD80B485B000AF7C
:10A8240078607B6893F83D30DBB2212B3ED17B68A6
:10A834009B68B3F5805F14D17B681B69002B10D132
:10A844007B681B6AFB60FB681B881A467B681B6875
:10A85400C2F308025A607B681B6A9A1C7B681A62FE
:10A8640008E07B681B6A591C7A6811621A787B6855
:10A874001B685A607B68DB8C9BB2013B9BB27A6895
:10A884001946D184002B0FD17B681B68DA687B687A
:10A894001B6822F08002DA607B681B68DA687B68D8
:10A8A4001B6842F04002DA60002300E002231846ED
:10A8B4001437BD465DF8047B704780B582B000AFA5
:10A8C40078607B681B68DA687B681B6822F040024A
:10A8D400DA607B68202283F83D207868F8F7BEF9B7
:10A8E400002318460837BD4680BD80B58CB000AF44
:10A8F40078607B6893F83E30DBB2222B40F0AB806B
:10A904007B689B68B3F5805F17D17B681B69002B5C
:10A9140013D10023FB627B689B6ABB627B681B6864
:10A924005B689BB2C3F308039AB2BB6A1A807B6864
:10A934009B6A9A1C7B689A6226E07B689B6AFB622E
:10A944000023BB627B689B68B3F5805F07D07B689C
:10A954009B68002B0AD17B681B69002B06D17B689E
:10A964001B685B68DAB2FB6A1A7008E07B681B68D4
:10A974005B68DBB203F07F03DAB2FB6A1A707B68B0
:10A984009B6A5A1C7B689A627B68DB8D9BB2013B95
:10A994009BB27A681946D185002B5AD17B681B6813
:10A9A400DA687B681B6822F02002DA607B681B6827
:10A9B400DA687B681B6822F48072DA607B681B6843
:10A9C4005A697B681B6822F001025A617B68202265
:10A9D40083F83E207B681B6B012B35D17B680022FA
:10A9E4001A637B681B680C337B617B6953E8003F07
:10A9F4003B613B6923F010037B627B681B680C336B
:10AA04007A6A3A62FB61F9693A6A41E80023BB61F8
:10AA1400BB69002BE5D17B681B681B6803F010033E
:10AA2400102B0AD10023FB607B681B681B68FB604A
:10AA34007B681B685B68FB60FB687B689B8D1946C1
:10AA44007868FFF74DFC02E07868F8F729F90023ED
:10AA540002E0002300E0022318463037BD4680BDE3
:10AA64002DE9B04FC0B000AFC7F8F400D7F8F43008
:10AA74001B681B6923F44050D7F8F430D968D7F821
:10AA8400F4301A6840EA01031361D7F8F4309A6885
:10AA9400D7F8F4301B691A43D7F8F4305B691A43CA
:10AAA400D7F8F430DB691343C7F8F830D7F8F4303B
:10AAB4001B68DB6823F4164121F00C01D7F8F4304D
:10AAC4001A68D7F8F8300B43D360D7F8F4301B6812
:10AAD4005B6923F44070D7F8F4309969D7F8F430FF
:10AAE4001A6840EA01035361D7F8F4301A688F4BAF
:10AAF4009A4205D0D7F8F4301A688D4B9A4204D1A3
:10AB0400FCF758FAC7F8FC0003E0FCF73FFAC7F873
:10AB1400FC00D7F8F430DB69B3F5004F40F00C814A
:10AB2400D7F8FC300022C7F8E830C7F8EC20D7E9A2
:10AB34003A4522462B469118B9655B41FB65D7E936
:10AB44001623214612EB0108294643EB01094FF075
:10AB540000024FF000034FEAC90343EA58734FEA77
:10AB6400C80290469946234618EB0303C7F8E03021
:10AB74002B4649EB0303C7F8E430D7F8F4305B689D
:10AB84000022C7F8D830C7F8DC20D7E936120B46C4
:10AB9400DB183B65134642EB03037B65D7E91423BB
:10ABA400D7E93801F5F734FB02460B46614BA3FBAA
:10ABB40002235B091C01D7F8FC300022C7F8D0300F
:10ABC400C7F8D420D7E9348942464B469118B96472
:10ABD4005B41FB64D7E91223414612EB010A494663
:10ABE40043EB010B4FF000024FF000034FEACB039D
:10ABF40043EA5A734FEACA0292469B4643461AEB0B
:10AC04000303C7F8C8304B464BEB0303C7F8CC30FB
:10AC1400D7F8F4305B680022C7F8C030C7F8C42006
:10AC2400D7E930120B46DB183B64134642EB0303AF
:10AC34007B64D7E91023D7E93201F5F7E9FA024634
:10AC44000B4611463B4BA3FB01235B09642202FB29
:10AC540003F3CB1ADB0003F13202364BA3FB0223CE
:10AC64005B095B0003F4F8731C44D7F8FC30002242
:10AC7400C7F8B830C7F8BC20D7E92E8942464B46FE
:10AC84009118B9635B41FB63D7E90E234146511820
:10AC9400396349464B417B634FF000024FF0000398
:10ACA400D7E90CAB5946CB00514643EA51735146A0
:10ACB400CA0010461946034642469B18C7F8B030EE
:10ACC4004B460A4642EB0303C7F8B430D7F8F430D6
:10ACD4005B680022C7F8A830C7F8AC20D7E92A126D
:10ACE4000B46DB18BB62134642EB0303FB62D7E956
:10ACF4000A23D7E92C01F5F78BFA02460B460D4BD4
:10AD0400A3FB02135B09642101FB03F3D31ADB00E9
:10AD14003233084AA2FB03235B0903F00702D7F886
:10AD2400F4301B6822449A6005E100BF0010014022
:10AD3400001401401F85EB51D7F8FC300022C7F8FE
:10AD4400A030C7F8A420D7E9288942464B46911879
:10AD540039625B417B62D7E908234146541849466E
:10AD640043EB01054FF000024FF00003EB0043EA10
:10AD74005473E20014461D464346E318C7F898305E
:10AD84004B4645EB0303C7F89C30D7F8F4305B68B7
:10AD94000022C7F89030C7F894204FF000024FF01B
:10ADA4000003D7E9244529468B00214643EA9173E1
:10ADB40021468A00D7E92601F5F72AFA02460B460E
:10ADC400604BA3FB02235B091C01D7F8FC30002273
:10ADD400C7F88830C7F88C20D7E9228942464B4609
:10ADE4009118B9615B41FB61D7E9062341465118CB
:10ADF400396149464B417B614FF000024FF000033B
:10AE0400D7E904AB5946CB00514643EA5173514646
:10AE1400CA0010461946034642469B18C7F88030BC
:10AE24004B460A4642EB0303C7F88430D7F8F430A4
:10AE34005B680022BB67FA674FF000024FF0000323
:10AE4400D7E91E8949468B00414643EA917341463E
:10AE54008A00D7E92001F5F7DBF902460B46394BA6
:10AE6400A3FB02135B09642101FB03F3D31A1B0147
:10AE74003233344AA2FB03235B0903F0F0031C447E
:10AE8400D7F8FC3000223B677A67D7E91C89424631
:10AE94004B469118B9605B41FB60D7E902234146F8
:10AEA4005118396049464B417B604FF000024FF026
:10AEB4000003D7E900AB5946CB00514643EA51732E
:10AEC4005146CA0010461946034642469B18BB66C3
:10AED4004B460A4642EB0303FB66D7F8F4305B6843
:10AEE40000223B667A664FF000024FF00003D7E978
:10AEF400188949468B00414643EA917341468A00CA
:10AF0400D7E91A01F5F784F902460B460D4BA3FB6A
:10AF140002135B09642101FB03F3D31A1B013233CF
:10AF2400084AA2FB03235B0903F00F02D7F8F430AD
:10AF34001B6822449A6000BF07F58077BD46BDE8D0
:10AF4400B08F00BF1F85EB5184B080B584B000AFD3
:10AF5400786007F11C0080E80E003B6B012B22D1C6
:10AF64007B689B6B23F480327B689A637B68DB6825
:10AF740023F4840323F040037A68D3607B68DB689E
:10AF840023F440127B68DA60FB6C012B05D17B68EB
:10AF9400DB6843F480127B68DA60786801F0E8FBD0
:10AFA4000346FB731AE07B68DB6843F040027B686E
:10AFB400DA60786801F0DCFB0346FB733B6C002B22
:10AFC40006D17B689B6B43F480327B689A6305E00F
:10AFD4007B689B6B23F480327B689A63BB6A012B8A
:10AFE4000BD17B689B6843F006027B689A607B68A0
:10AFF4009B6843F020027B689A60FB7B18461037FD
:10B00400BD46BDE8804004B07047000080B487B0FE
:10B0140000AFF860B9601346FB71FB79022B65D170
:10B02400BB68414A934206D9BB68404A934202D264
:10B034000F237B6162E0BB683C4A934206D3BB6842
:10B044003B4A934202D20E237B6157E0BB68384AE5
:10B05400934206D3BB68374A934202D20D237B61E5
:10B064004CE0BB68334A934206D3BB68324A9342EE
:10B0740002D80C237B6141E0BB682F4A934206D976
:10B08400BB682E4A934202D80B237B6136E0BB682F
:10B094002A4A934206D9BB68294A934202D80A2312
:10B0A4007B612BE0BB68264A934206D9BB68254ADC
:10B0B400934202D209237B6120E0BB68214A934278
:10B0C40006D3BB68204A934202D808237B6115E06B
:10B0D400BB681D4A934206D9BB681C4A934202D2FC
:10B0E40007237B610AE006237B6107E0FB79002BE1
:10B0F40002D109237B6101E009237B61FB68DB68E2
:10B1040023F47052FB68DA60FB68DA687B699B029F
:10B1140003F470531A43FB68DA60002318461C37A3
:10B12400BD465DF8047B7047BFACD800C0E1E400C5
:10B134000024F400807306019F491A01FF2C310199
:10B144003FA44C0100366E011FABA6010048E80184
:10B1540080B483B000AF78607B689B6843F00102E1
:10B164007B689A60002318460C37BD465DF8047B63
:10B17400704780B483B000AF78607B689B6823F02D
:10B1840001027B689A60002318460C37BD465DF8BF
:10B19400047B704780B584B000AF78600B46FB70C9
:10B1A4000023FB607B68DB6823F0C0427B68DA60C5
:10B1B400FB78012B15D17B68DB6843F000527B6878
:10B1C400DA600120F7F7B6FEFB680133FB607868AC
:10B1D40001F03FFA0346012B1ED0FB68312BF0D956
:10B1E4001AE0FB78002B15D17B68DB6843F08042C2
:10B1F4007B68DA600120F7F79DFEFB680133FB6092
:10B20400786801F026FA0346002B05D0FB68312B41
:10B21400F0D901E0012305E0FB68322B01D10123C1
:10B2240000E0002318461037BD4680BD84B080B5C9
:10B2340086B000AF786007F1240080E80E00002398
:10B24400FB757B68FB6000233B6109E07A683B691E
:10B2540040339B00134400225A603B6901333B6135
:10B264003B690E2BF2D9FB6C002B1CD1FB6803F558
:10B2740000635B68FA6802F5006243F002035360FE
:10B284007B689B6B23F400127B689A637B681B6862
:10B2940043F040027B681A607B681B6843F08002BD
:10B2A4007B681A6005E07B689B6B43F400127B6843
:10B2B4009A63FB6803F560631A4600231360FB6816
:10B2C40003F500631946FB6803F500631A460B682F
:10B2D4001360BB6B012B0CD1FB6A002B04D1002142
:10B2E400786800F065F908E00121786800F060F9F9
:10B2F40003E00321786800F05BF91021786800F01E
:10B30400F3F80346002B01D00123FB75786800F0A5
:10B314001FF90346002B01D00123FB75FB6803F5DD
:10B3240000631A4600231361FB6803F500631A46A1
:10B3340000235361FB6803F500631A460023D361BD
:10B3440000233B6143E03B695A01FB68134403F566
:10B3540010631B6803F00043B3F1004F18D13B693D
:10B36400002B0AD13B695A01FB68134403F51063AF
:10B374001A464FF00063136013E03B695A01FB68FF
:10B38400134403F510631A464FF09043136008E02A
:10B394003B695A01FB68134403F510631A46002302
:10B3A40013603B695A01FB68134403F510631A46A2
:10B3B400002313613B695A01FB68134403F51063CE
:10B3C4001A464FF67F3393603B6901333B617B6AD6
:10B3D4003A699A42B7D300233B6143E03B695A017F
:10B3E400FB68134403F530631B6803F00043B3F1B7
:10B3F400004F18D13B69002B0AD13B695A01FB6805
:10B40400134403F530631A464FF00063136013E0EE
:10B414003B695A01FB68134403F530631A464FF045
:10B424009043136008E03B695A01FB68134403F539
:10B4340030631A46002313603B695A01FB681344C6
:10B4440003F530631A46002313613B695A01FB6814
:10B45400134403F530631A464FF67F3393603B6918
:10B4640001333B617B6A3A699A42B7D3FB6803F5BF
:10B4740000631B69FA6802F5006223F480731361A8
:10B484007B6800229A617B686FF080425A613B6B53
:10B49400002B05D17B689B6943F010027B689A619D
:10B4A4007B689A690F4B13437A689361FB6B002B9B
:10B4B40005D07B689B6943F008027B689A61FB6C4A
:10B4C400012B07D17B689B6943F0804343F004035D
:10B4D4007A689361FB7D18461837BD46BDE8804005
:10B4E40004B0704700383C8080B485B000AF786009
:10B4F40039600023FB60FB680133FB60FB68134A7F
:10B50400934201D903231BE07B681B69002BF2DA09
:10B514000023FB603B689B0143F020027B681A61B7
:10B52400FB680133FB60FB68084A934201D903239B
:10B5340006E07B681B6903F02003202BF0D0002376
:10B5440018461437BD465DF8047B7047400D030070
:10B5540080B485B000AF78600023FB60FB680133E2
:10B56400FB60FB68114A934201D9032318E07B680E
:10B574001B69002BF2DA0023FB607B6810221A613E
:10B58400FB680133FB60FB68084A934201D903233B
:10B5940006E07B681B6903F01003102BF0D0002336
:10B5A40018461437BD465DF8047B7047400D030010
:10B5B40080B485B000AF78600B46FB707B68FB609D
:10B5C400FB6803F500631A68FB78F96801F500610C
:10B5D40013430B60002318461437BD465DF8047B03
:10B5E400704780B487B000AF78607B683B613B698B
:10B5F40003F500639B6803F00603FB60FB68002B04
:10B6040002D10023FB750AE0FB68022B02D0FB6821
:10B61400062B02D10223FB7501E00F23FB75FB7D92
:10B6240018461C37BD465DF8047B704780B485B06E
:10B6340000AF786039607B68FB603B681B78BB6057
:10B644003B685B78012B3AD1FB6803F50063DA6948
:10B654003B681B7803F00F03012101FA03F39BB24B
:10B66400F96801F500611343CB61BB685A01FB68BB
:10B67400134403F510631B6803F40043002B55D1F6
:10B68400BB685A01FB68134403F510631A683B68EE
:10B69400DB68C3F30A013B681B799B041943BB684D
:10B6A4009B050B431343BA685101FA680A4402F537
:10B6B400106243F0805343F40043136036E0FB68A8
:10B6C40003F50063DA693B681B7803F00F0301217B
:10B6D40001FA03F31B04F96801F500611343CB611C
:10B6E400BB685A01FB68134403F530631B6803F419
:10B6F4000043002B1AD1BB685A01FB68134403F5BD
:10B7040030631A683B68DB68C3F30A013B681B7942
:10B714009B040B431343BA685101FA680A4402F5C7
:10B72400306243F0805343F400431360002318460F
:10B734001437BD465DF8047B7047000080B485B0C3
:10B7440000AF786039607B68FB603B681B78BB6046
:10B754003B685B78012B61D1BB685A01FB681344D9
:10B7640003F510631B6803F00043B3F1004F1FD1CE
:10B77400BB685A01FB68134403F510631B68BA687D
:10B784005101FA680A4402F5106243F00063136041
:10B79400BB685A01FB68134403F510631B68BA685D
:10B7A4005101FA680A4402F5106243F080431360C1
:10B7B400FB6803F50063DA6B3B681B7803F00F0347
:10B7C400012101FA03F39BB2DB43F96801F500613F
:10B7D4001340CB63FB6803F50063DA693B681B78AD
:10B7E40003F00F03012101FA03F39BB2DB43F96871
:10B7F40001F500611340CB61BB685A01FB68134437
:10B8040003F510631A68BB685901FB680B4403F520
:10B8140010631946354B13400B6060E0BB685A0156
:10B82400FB68134403F530631B6803F00043B3F172
:10B83400004F1FD1BB685A01FB68134403F5306302
:10B844001B68BA685101FA680A4402F5306243F091
:10B8540000631360BB685A01FB68134403F530634B
:10B864001B68BA685101FA680A4402F5306243F071
:10B8740080431360FB6803F50063DA6B3B681B7855
:10B8840003F00F03012101FA03F31B04DB43F968FE
:10B8940001F500611340CB63FB6803F50063DA69CB
:10B8A4003B681B7803F00F03012101FA03F31B0427
:10B8B400DB43F96801F500611340CB61BB685A01B1
:10B8C400FB68134403F530631A68BB685901FB68CD
:10B8D4000B4403F530631946054B13400B600023FA
:10B8E40018461437BD465DF8047B7047007833EC86
:10B8F4000078F3EF80B58AB002AFF860B960134600
:10B90400FB71FB68FB61BB681B78BB61BB685B7840
:10B91400012B40F05C81BB689B69002B32D1BB6971
:10B924005A01FB69134403F510631B69BA69510199
:10B93400FA690A4402F5106223F0FF5323F4C0139A
:10B944001361BB695A01FB69134403F510631B6956
:10B95400BA695101FA690A4402F5106243F40023FA
:10B964001361BB695A01FB69134403F510631B6936
:10B97400BA695101FA690A4402F51062DB0CDB046E
:10B98400136174E0BB695A01FB69134403F5106346
:10B994001B69BA695101FA690A4402F51062DB0CA9
:10B9A400DB041361BB695A01FB69134403F510639B
:10B9B4001B69BA695101FA690A4402F5106223F05D
:10B9C400FF5323F4C0131361BB695A01FB69134489
:10B9D40003F510631A69BB689969BB68DB680B449B
:10B9E400591EBB68DB68B1FBF3F3D9049D4B0B40D4
:10B9F400B9694801F969014401F5106113430B6108
:10BA0400BB695A01FB69134403F510631A69BB68E7
:10BA14009B69C3F31203B9694801F969014401F54B
:10BA2400106113430B61BB681B79012B1FD1BB69E8
:10BA34005A01FB69134403F510631B69BA69510188
:10BA4400FA690A4402F5106223F0C0431361BB692A
:10BA54005A01FB69134403F510631B69BA69510168
:10BA6400FA690A4402F5106243F000531361FB794A
:10BA7400012B4BD1BB685B69002B09D0BB695A0110
:10BA8400FB69134403F510631A46BB685B69536191
:10BA9400BB681B79012B28D1FB6903F500639B6804
:10BAA40003F48073002B10D1BB695A01FB69134462
:10BAB40003F510631B68BA695101FA690A4402F577
:10BAC400106243F0005313600FE0BB695A01FB6935
:10BAD400134403F510631B68BA695101FA690A44F7
:10BAE40002F5106243F080531360BB695A01FB698D
:10BAF400134403F510631B68BA695101FA690A44D7
:10BB040002F5106243F00443136033E1BB695A0148
:10BB1400FB69134403F510631B68BA695101FA69A0
:10BB24000A4402F5106243F004431360BB681B79B6
:10BB3400012B15D0BB689B69002B00F01B81FB69AE
:10BB440003F500635A6BBB681B7803F00F030121F4
:10BB540001FA03F3F96901F5006113434B6309E149
:10BB6400FB6903F500639B6803F48073002B10D119
:10BB7400BB695A01FB69134403F510631B68BA6976
:10BB84005101FA690A4402F5106243F0005313604C
:10BB94000FE0BB695A01FB69134403F510631B688A
:10BBA400BA695101FA690A4402F5106243F08053FC
:10BBB4001360BB681969BB681A78BB689B6998B243
:10BBC400FB7900930346F86800F0DEFAD2E0BB6923
:10BBD4005A01FB69134403F530631B69BA695101C7
:10BBE400FA690A4402F53062DB0CDB041361BB69B9
:10BBF4005A01FB69134403F530631B69BA695101A7
:10BC0400FA690A4402F5306223F0FF5323F4C013A7
:10BC14001361BB689B69002B26D1BB695A01FB6980
:10BC2400134403F530631A69BB68DB68C3F312037A
:10BC3400B9694801F969014401F5306113430B61A5
:10BC4400BB695A01FB69134403F530631B69BA6984
:10BC54005101FA690A4402F5306243F40023136186
:10BC64003AE000BF0000F81FBB689A69BB68DB6854
:10BC740013445A1EBB68DB68B2FBF3F3FB82BB6858
:10BC8400DB68FA8A03FB02F2BB68DA61BB695A011A
:10BC9400FB69134403F530631A69FB8AD904384BF2
:10BCA4000B40B9694801F969014401F53061134356
:10BCB4000B61BB695A01FB69134403F530631A69CC
:10BCC400BB68DB69C3F31203B9694801F96901442C
:10BCD40001F5306113430B61FB79012B0DD1BB6876
:10BCE4001B69002B09D0BB681969BB695A01FB6940
:10BCF400134403F530630A465A61BB681B79012B70
:10BD040028D1FB6903F500639B6803F48073002B5F
:10BD140010D1BB695A01FB69134403F530631B68F6
:10BD2400BA695101FA690A4402F5306243F00053DA
:10BD340013600FE0BB695A01FB69134403F53063D8
:10BD44001B68BA695101FA690A4402F5306243F08A
:10BD540080531360BB695A01FB69134403F53063D4
:10BD64001B68BA695101FA690A4402F5306243F06A
:10BD740004431360002318462037BD4680BD00BF2E
:10BD84000000F81F80B487B000AFF860B9601346B4
:10BD9400FB71FB687B61BB681B783B61BB685B78AC
:10BDA400012B40F0CE80BB689B69002B32D13B69EC
:10BDB4005A017B69134403F510631B693A69510105
:10BDC4007A690A4402F5106223F0FF5323F4C01386
:10BDD40013613B695A017B69134403F510631B69C2
:10BDE4003A6951017A690A4402F5106243F4002366
:10BDF40013613B695A017B69134403F510631B69A2
:10BE04003A6951017A690A4402F51062DB0CDB04D9
:10BE140013614EE03B695A017B69134403F51063D7
:10BE24001B693A6951017A690A4402F51062DB0C14
:10BE3400DB0413613B695A017B69134403F5106306
:10BE44001B693A6951017A690A4402F5106223F0C8
:10BE5400FF5323F4C0131361BB689A69BB68DB68A2
:10BE64009A4203D9BB68DA68BB689A613B695A0194
:10BE74007B69134403F510631B693A6951017A69BC
:10BE84000A4402F5106243F4002313613B695A012A
:10BE94007B69134403F510631A69BB689B69C3F398
:10BEA4001203396948017969014401F510611343AA
:10BEB4000B61FB79012B1ED1BB685B69002B09D098
:10BEC4003B695A017B69134403F510631A46BB6846
:10BED4005B6953613B695A017B69134403F5106341
:10BEE4001B683A6951017A690A4402F5106243F009
:10BEF4000443136097E03B695A017B69134403F5DB
:10BF040010631B683A6951017A690A4402F51062A8
:10BF140043F004431360BB689B69002B00F08380EB
:10BF24007B6903F500635A6BBB681B7803F00F034E
:10BF3400012101FA03F3796901F5006113434B63AD
:10BF440071E03B695A017B69134403F530631B6953
:10BF54003A6951017A690A4402F53062DB0CDB0468
:10BF640013613B695A017B69134403F530631B6910
:10BF74003A6951017A690A4402F5306223F0FF53A9
:10BF840023F4C0131361BB689B69002B03D0BB6807
:10BF9400DA68BB689A61BB68DA68BB68DA613B69D6
:10BFA4005A017B69134403F530631B693A695101F3
:10BFB4007A690A4402F5306243F4002313613B6951
:10BFC4005A017B69134403F530631A69BB68DB6962
:10BFD400C3F31203396948017969014401F53061F9
:10BFE40013430B61FB79012B0DD1BB681B69002B3B
:10BFF40009D0BB6819693B695A017B69134403F58D
:10C0040030630A465A613B695A017B69134403F55C
:10C0140030631B683A6951017A690A4402F5306257
:10C0240043F004431360002318461C37BD465DF8F3
:10C03400047B704780B487B000AF78603960002318
:10C04400FB600023FB757B683B613B685B78012BDD
:10C054004AD13B681B785A013B69134403F51063CA
:10C064001B6803F00043B3F1004F40F086803B6847
:10C074001B785A013B69134403F510631B683A6843
:10C08400127851013A690A4402F5106243F00063E0
:10C0940013603B681B785A013B69134403F5106332
:10C0A4001B683A68127851013A690A4402F5106231
:10C0B40043F080431360FB680133FB60FB6842F28A
:10C0C4001072934202D90123FB7556E03B681B783A
:10C0D4005A013B69134403F510631B6803F00043E2
:10C0E400B3F1004FE7D048E03B681B785A013B6945
:10C0F400134403F530631B6803F00043B3F1004FAE
:10C104003BD13B681B785A013B69134403F5306308
:10C114001B683A68127851013A690A4402F53062A0
:10C1240043F0006313603B681B785A013B69134476
:10C1340003F530631B683A68127851013A690A447E
:10C1440002F5306243F080431360FB680133FB6007
:10C15400FB6842F21072934202D90123FB750CE092
:10C164003B681B785A013B69134403F530631B6831
:10C1740003F00043B3F1004FE7D0FB7D18461C37B2
:10C18400BD465DF8047B704780B489B000AFF860A9
:10C19400B96011461A460B46FB711346BB80FB6817
:10C1A4007B61BB68FB6197F82830002B23D1BB88E7
:10C1B40003339B083B610023BB6118E0FB791A033E
:10C1C4007B69134403F580531A46FB691B681360AB
:10C1D400FB690133FB61FB690133FB61FB690133DB
:10C1E400FB61FB690133FB61BB690133BB61BA6964
:10C1F4003B699A42E2D3002318462437BD465DF8D2
:10C20400047B704780B48BB000AFF860B96013460C
:10C21400FB80FB68BB61BB687B62FB889B089BB2AD
:10C224007B61FB8803F00303FB8300233B6214E080
:10C23400BB6903F580531A687B6A1A607B6A013311
:10C244007B627B6A01337B627B6A01337B627B6A3C
:10C2540001337B623B6A01333B623A6A7B699A42EF
:10C26400E6D3FB8B002B1ED000233B62BB6903F596
:10C2740080531A4607F1100312681A603A693B6A40
:10C28400DBB2DB0022FA03F3DAB27B6A1A703B6A90
:10C2940001333B627B6A01337B62FB8B013BFB8393
:10C2A400FB8B002BEAD17B6A18462C37BD465DF820
:10C2B400047B704780B485B000AF786039607B68D8
:10C2C400FB603B681B78BB603B685B78012B2CD11F
:10C2D400BB685A01FB68134403F510631B68002B09
:10C2E40012DBBB68002B0FD0BB685A01FB681344F8
:10C2F40003F510631B68BA685101FA680A4402F531
:10C30400106223F080431360BB685A01FB68134436
:10C3140003F510631B68BA685101FA680A4402F510
:10C32400106243F4001313602BE0BB685A01FB68EE
:10C33400134403F530631B68002B12DBBB68002B2E
:10C344000FD0BB685A01FB68134403F530631B68C4
:10C35400BA685101FA680A4402F5306223F0804356
:10C364001360BB685A01FB68134403F530631B6810
:10C37400BA685101FA680A4402F5306243F40013C2
:10C384001360002318461437BD465DF8047B7047DC
:10C3940080B485B000AF786039607B68FB603B682F
:10C3A4001B78BB603B685B78012B28D1BB685A01C2
:10C3B400FB68134403F510631B68BA685101FA68FB
:10C3C4000A4402F5106223F4001313603B681B79DE
:10C3D400032B03D03B681B79022B38D1BB685A016D
:10C3E400FB68134403F510631B68BA685101FA68CB
:10C3F4000A4402F5106243F08053136027E0BB68DF
:10C404005A01FB68134403F530631B68BA68510191
:10C41400FA680A4402F5306223F4001313603B689F
:10C424001B79032B03D03B681B79022B0FD1BB680C
:10C434005A01FB68134403F530631B68BA68510161
:10C44400FA680A4402F5306243F080531360002313
:10C4540018461437BD465DF8047B704780B485B038
:10C4640000AF78600B46FB707B68FB60FB6803F5EC
:10C4740000631B68FA6802F5006223F4FE6313602C
:10C48400FB6803F500631A68FB781B0103F4FE6381
:10C49400F96801F5006113430B6000231846143753
:10C4A400BD465DF8047B704780B485B000AF78600A
:10C4B4007B68FB60FB6803F560631B68FA6802F540
:10C4C400606223F003031360FB6803F500635B6899
:10C4D400FA6802F5006223F0020353600023184651
:10C4E4001437BD465DF8047B704780B485B000AF57
:10C4F40078607B68FB60FB6803F560631B68FA681F
:10C5040002F5606223F003031360FB6803F5006324
:10C514005B68FA6802F5006243F00203536000238B
:10C5240018461437BD465DF8047B704780B485B067
:10C5340000AF78607B685B69FB607B689B69FA6825
:10C544001340FB60FB6818461437BD465DF8047B56
:10C55400704780B485B000AF78607B68FB60FB688F
:10C5640003F500639B69BB60FB6803F50063DB694B
:10C57400BA681340BB60BB681B0C18461437BD4631
:10C584005DF8047B704780B485B000AF78607B6849
:10C59400FB60FB6803F500639B69BB60FB6803F504
:10C5A4000063DB69BA681340BB60BB689BB2184682
:10C5B4001437BD465DF8047B704780B485B000AF86
:10C5C40078600B46FB707B68FB60FB785A01FB6864
:10C5D400134403F530639B68BB60FB6803F5006399
:10C5E4005B69BA681340BB60BB6818461437BD4624
:10C5F4005DF8047B704780B487B000AF78600B4669
:10C60400FB707B687B617B6903F500631B693B619D
:10C614007B6903F500635B6BFB60FB7803F00F033E
:10C62400FA6822FA03F3DB01DBB23A6913433B6194
:10C63400FB785A017B69134403F510639B683A69DC
:10C644001340BB60BB6818461C37BD465DF8047BCD
:10C65400704780B483B000AF78607B685B6903F097
:10C66400010318460C37BD465DF8047B704780B45F
:10C6740085B000AF78607B68FB60FB6803F51063EE
:10C684001B68FA6802F5106223F4FF6323F00703C2
:10C694001360FB6803F500635B68FA6802F50062E7
:10C6A40043F480735360002318461437BD465DF885
:10C6B400047B704780B487B000AFF8600B467A60A3
:10C6C400FB72FB687B61FB683C3304331B683B6192
:10C6D4003B69264A93420AD97B6903F530631B6898
:10C6E40003F00043B3F1004F01D1002337E07B692D
:10C6F40003F530631A46002313617B6903F5306345
:10C704001B697A6902F5306243F4002313617B6983
:10C7140003F530631B697A6902F5306243F018034C
:10C7240013617B6903F530631B697A6902F5306232
:10C7340043F0C0431361FB7A012B0FD17B6903F5EE
:10C7440030631A467B6853617B6903F530631B6869
:10C754007A6902F5306243F080231360002318469F
:10C764001C37BD465DF8047B704700BF0A30544F48
:10C7740080B485B000AF78600023FB60FB680133B0
:10C78400FB60FB68134A934201D903231BE07B68D7
:10C794001B69002BF2DA0023FB607B681B6943F002
:10C7A40001027B681A61FB680133FB60FB68094A7C
:10C7B400934201D9032306E07B681B6903F001035C
:10C7C400012BF0D0002318461437BD465DF8047BD6
:10C7D400704700BF400D030080B584B000AF78609F
:10C7E4000B46FB704FF4077002F0EAFCF860FB683C
:10C7F400002B09D17B68D3F8D4227B68B0320021A6
:10C8040043F822100223D4E04FF407720021F868A1
:10C8140002F03EFD7B68D3F8D4227B68B032F9681D
:10C8240043F822107B68D3F8D4227B68B03253F8E3
:10C8340022207B68C3F8BC227B681B7C002B38D188
:10C844005E4B19784FF400730222786802F047FBBC
:10C854005A4B1B7803F00F02796813469B0013446C
:10C864009B000B44243301221A80554B19784FF452
:10C8740000730222786802F032FB514B1B7803F0FC
:10C884000F02796813469B0013449B000B4403F585
:10C89400B27301221A804B4B1B7803F00F027968A4
:10C8A40013469B0013449B000B44263310221A802A
:10C8B40035E0424B197840230222786802F00FFBDE
:10C8C4003E4B1B7803F00F02796813469B00134418
:10C8D4009B000B44243301221A80394B19784023DE
:10C8E4000222786802F0FBFA354B1B7803F00F0242
:10C8F400796813469B0013449B000B4403F5B27301
:10C9040001221A802F4B1B7803F00F02796813461B
:10C914009B0013449B000B44263310221A80294B9E
:10C92400197808230322786802F0D9FA254B1B787A
:10C9340003F00F02796813469B0013449B000B44D9
:10C94400243301221A80FB680022C3F804227B6886
:10C95400D3F8D4327A68B0339B0013445B681B6805
:10C964009847FB680022C3F81422FB680022C3F82E
:10C974001822FB68D3F80432002B01D1022318E0FB
:10C984007B681B7C002B0AD10D4B1978FB68D3F80C
:10C9940004224FF40073786802F090FB08E0084B1F
:10C9A4001978FB68D3F804224023786802F086FBE8
:10C9B400002318461037BD4680BD00BF9F000020ED
:10C9C400A0000020A100002080B582B000AF7860F4
:10C9D4000B46FB703A4B1B781946786802F0A5FAAF
:10C9E400374B1B7803F00F02796813469B001344FE
:10C9F4009B000B44243300221A80324B1B781946C7
:10CA0400786802F092FA2F4B1B7803F00F027968D2
:10CA140013469B0013449B000B4403F5B27300229E
:10CA24001A80294B1B781946786802F07EFA264B47
:10CA34001B7803F00F02796813469B0013449B0094
:10CA44000B44243300221A801F4B1B7803F00F027F
:10CA5400796813469B0013449B000B442633002241
:10CA64001A807B68D3F8D4227B68B03253F8223022
:10CA7400002B1FD07B68D3F8D4327A68B0339B0084
:10CA840013445B685B6898477B68D3F8D4227B685F
:10CA9400B03253F82230184602F0A0FB7B68D3F87A
:10CAA400D4227B68B032002143F822107B68002234
:10CAB400C3F8BC22002318460837BD4680BD00BF1A
:10CAC4009F000020A0000020A100002080B586B0B7
:10CAD40000AF786039607B68D3F8D4227B68B032C9
:10CAE40053F822303B6100237B7300237B810023B6
:10CAF400FB753B69002B01D10323BFE03B681B7826
:10CB040003F06003002B50D0202B40F0AF803B6833
:10CB1400DB88002B3AD03B681B785BB2002B1BDA16
:10CB24007B68D3F8D4327A68B0339B0013445B68D3
:10CB34009B683A68507839693A68D28898473B6864
:10CB4400DB88072B28BF0723FB813B69FA89194639
:10CB5400786801F06DFD90E03B685A783B6983F892
:10CB640000223B68DB883F2B03D83B68DB88DAB2C2
:10CB740000E040223B6983F8012239693B6993F85C
:10CB840001321A46786801F07FFD76E07B68D3F8BD
:10CB9400D4327A68B0339B0013445B689B683A686C
:10CBA400507800223968984767E03B685B780B2B24
:10CBB40051D801A252F823F0EDCB000869CC00084B
:10CBC4005BCC00085BCC00085BCC00085BCC0008A5
:10CBD4005BCC00085BCC00085BCC00085BCC000895
:10CBE40017CC000841CC00087B6893F89C32DBB278
:10CBF400032B07D107F10A0302221946786801F0D2
:10CC040017FD32E03968786801F0A1FC0323FB7555
:10CC14002BE07B6893F89C32DBB2032B07D107F13E
:10CC24000D0301221946786801F002FD1DE0396800
:10CC3400786801F08CFC0323FB7516E07B6893F89D
:10CC44009C32DBB2032B0FD03968786801F07FFC8B
:10CC54000323FB7508E03968786801F078FC032346
:10CC6400FB7502E000BF08E000BF06E039687868A1
:10CC740001F06DFC0323FB7500BFFB7D18461837DC
:10CC8400BD4680BD80B584B000AF78600B46FB70B4
:10CC94007B68D3F8C832FB607B68D3F8D4227B6806
:10CCA400B03253F82230002B01D1032365E07B68B6
:10CCB400D3F8D4227B68B03253F82230BB60FB78BF
:10CCC40003F00F02796813469B0013449B000B4446
:10CCD40018331B68002B2FD0FB7803F00F02796800
:10CCE40013469B0013449B000B4418331A68FB78CB
:10CCF40003F00F01F8680B46DB000B449B00034470
:10CD040048331B68B2FBF3F101FB03F3D31A002B86
:10CD140012D1FB7803F00F02796813469B00134489
:10CD24009B000B44183300221A60F9780023002278
:10CD3400786802F0A2F91FE0BB680022C3F814224D
:10CD44007B68D3F8D4327A68B0339B0013445B68B1
:10CD54001B69002B10D07B68D3F8D4327A68B033C7
:10CD64009B0013445B681B69BA68D2F80802BA686E
:10CD740002F50471FA789847002318461037BD4627
:10CD840080BD80B584B000AF78600B46FB707B68D3
:10CD9400D3F8D4227B68B03253F82230FB607B682E
:10CDA400D3F8D4227B68B03253F82230002B01D15F
:10CDB40003231AE0FB781946786802F0A0F90246CA
:10CDC400FB68C3F80C227B68D3F8D4327A68B0339A
:10CDD4009B0013445B68DB68FA68D2F80402FA68C3
:10CDE40002F5037211469847002318461037BD46D2
:10CDF40080BD80B584B000AF78607B68D3F8D4225E
:10CE04007B68B03253F82230FB60FB68002B01D101
:10CE1400032325E07B68D3F8D4327A68B0339B00CF
:10CE240013445B68002B1AD0FB6893F80032FF2B85
:10CE340015D07B68D3F8D4327A68B0339B0013449E
:10CE44005B689B68FA6892F80002F968FA6892F8DD
:10CE5400012292B29847FB68FF2283F80022002344
:10CE640018461037BD4680BD80B586B000AF7860E7
:10CE74008221184800F009FD78610121154800F06D
:10CE840004FD38618121134800F0FFFCF8607B69E0
:10CE9400002B02D07B6910229A713B69002B06D0CB
:10CEA4003B69002242F040021A7100225A71FB6869
:10CEB400002B06D0FB68002242F040021A710022C7
:10CEC4005A717B6843221A80024B18461837BD46B4
:10CED40080BD00BF5C00002080B586B000AF7860E4
:10CEE4008221184800F0D1FC78610121154800F036
:10CEF400CCFC38618121134800F0C7FCF8607B69E1
:10CF0400002B02D07B6910229A713B69002B06D05A
:10CF14003B6900221A71002242F002025A71FB6836
:10CF2400002B06D0FB6800221A71002242F0020294
:10CF34005A717B6843221A80024B18461837BD4643
:10CF440080BD00BF5C00002080B586B000AF786073
:10CF54008221184800F099FC78610121154800F0FD
:10CF640094FC38618121134800F08FFCF8607B69E0
:10CF7400002B02D07B6910229A713B69002B06D0EA
:10CF84003B69002242F040021A7100225A71FB6888
:10CF9400002B06D0FB68002242F040021A710022E6
:10CFA4005A717B6843221A80024B18461837BD46D3
:10CFB40080BD00BF5C00002080B483B000AF786007
:10CFC4007B680A221A80034B18460C37BD465DF86D
:10CFD400047B70471800002080B483B000AF7860F1
:10CFE40039603B68002B01D1032309E07B68D3F847
:10CFF400D4327A68B0339B0013443A685A600023F1
:10D0040018460C37BD465DF8047B704780B487B082
:10D0140000AFF860B9607A60FB68D3F8D422FB688B
:10D02400B03253F822307B617B69002B01D103239A
:10D0340008E07B69BA68C3F808227B697A68C3F898
:10D044001022002318461C37BD465DF8047B704748
:10D0540080B485B000AF786039607B68D3F8D4229F
:10D064007B68B03253F82230FB60FB68002B01D19F
:10D07400032304E0FB683A68C3F80422002318463B
:10D084001437BD465DF8047B7047000080B584B05A
:10D0940000AF78607B68D3F8D4227B68B03253F851
:10D0A4002230FB607B68D3F8D4227B68B03253F81B
:10D0B4002230002B01D1032318E07B681B7C002B5A
:10D0C4000AD10C4B1978FB68D3F804224FF400738F
:10D0D400786801F0F3FF08E0064B1978FB68D3F891
:10D0E40004224023786801F0E9FF00231846103732
:10D0F400BD4680BDA000002080B586B000AFF860BA
:10D10400B9601346FB71FB68002B01D103231FE0B8
:10D11400FB680022C3F8B822FB680022C3F8C422CB
:10D12400FB680022C3F8D022BB68002B03D0FB6845
:10D13400BA68C3F8B422FB68012283F89C22FB6816
:10D14400FA791A70F86801F063FE0346FB75FB7DFB
:10D1540018461837BD4680BD80B584B000AF7860EE
:10D1640039600023FB813B68002B01D1032325E0B8
:10D174007B683A68C3F8B8227B68D3F8D4227B680A
:10D18400AE3253F82230DB6A002B0FD07B68D3F821
:10D19400D4227B68AE3253F82230DB6A07F10E02E8
:10D1A4001046984702467B68C3F8D0227B68D3F8C0
:10D1B400D8325A1C7B68C3F8D8220023184610378B
:10D1C400BD4680BD80B582B000AF7860786801F05C
:10D1D4006BFE034618460837BD4680BD80B483B055
:10D1E40000AF7860002318460C37BD465DF8047B19
:10D1F400704780B584B000AF78600B46FB700023A5
:10D20400FB737B68D3F8B832002B09D07B68D3F862
:10D21400B8321B68FA781146786898470346FB735E
:10D22400FB7B18461037BD4680BD80B584B000AF87
:10D2340078600B46FB700023FB737B68D3F8B8322D
:10D244005B68FA781146786898470346002B01D04A
:10D254000323FB73FB7B18461037BD4680BD80B5A6
:10D2640084B000AF786039607B6803F2AA23396820
:10D27400184601F032F97B680122C3F894227B68D6
:10D28400B3F8B0321A467B68C3F898227B6893F8E7
:10D29400AA3203F01F03022B1AD0022B22D8002B30
:10D2A40002D0012B0AD01DE07B6803F2AA231946A1
:10D2B400786800F05FFB0346FB7320E07B6803F2B1
:10D2C400AA231946786800F0C7FB0346FB7316E0EF
:10D2D4007B6803F2AA231946786800F029FC034608
:10D2E400FB730CE07B6893F8AA3223F07F03DBB274
:10D2F4001946786801F038FE0346FB7300BFFB7BD8
:10D3040018461037BD4680BD80B586B000AFF860C2
:10D314000B467A60FB720023FB75FB7A002B6ED1FF
:10D32400FB6803F5AA733B61FB68D3F89432032BC3
:10D3340040F098803B699A683B69DB689A4213D94C
:10D344003B699A683B69DB68D21A3B699A603B691E
:10D35400DA683B699B68934228BF13461A4679688A
:10D36400F86801F0AEF97DE0FB6893F8AA3203F0A7
:10D374001F03022B14D0022B1DD8002B02D0012B2B
:10D3840003D018E00023BB7518E0FB68B3F8AE3295
:10D39400DBB21946F86800F05EFA0346BB750DE08F
:10D3A400FB68B3F8AE32DBB21946F86800F060FAF5
:10D3B4000346BB7502E00023BB7500BFBB7D002B99
:10D3C40019D1FB6893F89C32DBB2032B13D1BA7DDD
:10D3D400FB68AE3253F822301B69002B0BD0BA7DA8
:10D3E400FB68C3F8D422BA7DFB68AE3253F822300E
:10D3F4001B69F8689847F86801F074F932E0FB7A21
:10D4040003F07F03DBB21946F86800F031FA0346F3
:10D41400BB75BB7DFF2B25D0BB7D002B22D1FB68C8
:10D4240093F89C32DBB2032B17D1BA7DFB68AE3282
:10D4340053F822309B69002B0FD0BA7DFB68C3F8E8
:10D44400D422BA7DFB68AE3253F822309B69FA7A53
:10D454001146F86898470346FB75FB7D002B01D005
:10D46400FB7D00E0002318461837BD4680BD80B51B
:10D4740086B000AFF8600B467A60FB72FB7A002B33
:10D484006FD1FB6814333B61FB68D3F89432022BF1
:10D494005AD13B699A683B69DB689A4214D93B6963
:10D4A4009A683B69DB68D21A3B699A603B699B685E
:10D4B4001A467968F86801F0D6F8002300220021A2
:10D4C400F86801F0FBFD3FE03B69DA683B699B6863
:10D4D4009A421CD13B695A683B69DB689A4216D36D
:10D4E4003B695A68FB68D3F898329A420FD20022FB
:10D4F4000021F86801F0B7F8FB680022C3F898220D
:10D50400002300220021F86801F0D8FD1CE0FB682C
:10D5140093F89C32DBB2032B0FD1FB68D3F8B832FB
:10D52400DB68002B09D0FB680022C3F8D422FB6817
:10D53400D3F8B832DB68F86898478021F86801F0BE
:10D5440013FDF86801F0E1F8FB6893F8A032002BB2
:10D554003AD0F868FFF742FEFB68002283F8A02265
:10D5640032E0FB7A63F07F03DBB21946F86800F01F
:10D574007FF90346FB75FB7DFF2B25D0FB7D002B3C
:10D5840022D1FB6893F89C32DBB2032B1CD1FA7DC9
:10D59400FB68AE3253F822305B69002B14D0FA7D5D
:10D5A400FB68C3F8D422FA7DFB68AE3253F822300C
:10D5B4005B69FA7A1146F86898470346BB75BB7DE8
:10D5C400002B01D0BB7D00E0002318461837BD4670
:10D5D40080BD80B584B000AF78600023FB737B68A6
:10D5E400012283F89C227B680022C3F894227B6882
:10D5F40000225A607B680022C3F8A4227B680022C0
:10D6040083F8A0227B68D3F8B832002B14D07B684F
:10D61400D3F8B8325B68002B0ED07B68D3F8B832ED
:10D624005B687A685268D2B21146786898470346B4
:10D63400002B01D00323FB734023002200217868D0
:10D6440001F04DFC7B680122A3F864217B68402231
:10D65400C3F86021402300228021786801F03FFC58
:10D664007B6801229A847B6840221A62FB7B1846FD
:10D674001037BD4680BD80B483B000AF78600B46E0
:10D68400FB707B68FA781A74002318460C37BD4681
:10D694005DF8047B704780B483B000AF78607B682A
:10D6A40093F89C32DAB27B6883F89D227B6804226B
:10D6B40083F89C22002318460C37BD465DF8047B92
:10D6C400704780B483B000AF78607B6893F89C3275
:10D6D400DBB2042B06D17B6893F89D32DAB27B6807
:10D6E40083F89C22002318460C37BD465DF8047B62
:10D6F400704780B582B000AF78607B6893F89C3245
:10D70400DBB2032B10D17B68D3F8B832002B0BD0DB
:10D714007B68D3F8B832DB69002B05D07B68D3F87B
:10D72400B832DB6978689847002318460837BD4645
:10D7340080BD80B582B000AF78600B46FB707B681B
:10D74400D3F8D4227B68AE3253F82230002B01D1B7
:10D7540003231CE07B6893F89C32DBB2032B15D1C6
:10D764007B68D3F8D4227B68AE3253F822301B6A2C
:10D77400002B0BD07B68D3F8D4227B68AE3253F8ED
:10D7840022301B6AFA7811467868984700231846B5
:10D794000837BD4680BD80B582B000AF78600B46C7
:10D7A400FB707B68D3F8D4227B68AE3253F8223006
:10D7B400002B01D103231CE07B6893F89C32DBB27D
:10D7C400032B15D17B68D3F8D4227B68AE3253F88F
:10D7D40022305B6A002B0BD07B68D3F8D4227B68A1
:10D7E400AE3253F822305B6AFA781146786898476B
:10D7F400002318460837BD4680BD80B483B000AF0F
:10D804007860002318460C37BD465DF8047B7047EA
:10D8140080B584B000AF78600023FB737B6801227D
:10D8240083F89C227B68D3F8B832002B0ED07B6837
:10D83400D3F8B8325B687A685268D2B21146786815
:10D8440098470346002B01D00323FB73FB7B184648
:10D854001037BD4680BD80B483B000AF78600B46FE
:10D86400FB70002318460C37BD465DF8047B7047F7
:10D8740080B483B000AF78600B46FB700023184679
:10D884000C37BD465DF8047B704780B586B000AFA9
:10D8940078600B46FB707B687B617B68FB600023D0
:10D8A4003B61FB685B889AB2FB681B789BB29A4227
:10D8B40020D9FB681B789BB27B8113E007F10A0334
:10D8C4001946786900F01BF878617B695B78052B51
:10D8D40008D17B693B613B699B78FA789A4208D00E
:10D8E40000233B61FB685B889AB27B899A42E5D846
:10D8F40000E000BF3B6918461837BD4680BD80B4C0
:10D9040085B000AF786039607B68FB603B681A883B
:10D91400FB681B789BB213449AB23B681A80FB687D
:10D924001B781A467B681344FB60FB68184614375F
:10D93400BD465DF8047B704780B487B000AF786063
:10D944007B687B617B691B787B827B6901337B61AC
:10D954007B691B783B823B8A1B021AB2B7F91230EF
:10D9640013431BB2FB81FB8918461C37BD465DF887
:10D97400047B704780B584B000AF786039600023C1
:10D98400FB733B681B7803F06003402B05D0402BEE
:10D9940057D8002B0FD0202B53D17B68D3F8D42237
:10D9A4007B68AE3253F822309B68396878689847B0
:10D9B4000346FB734AE03B685B78092B3BD801A222
:10D9C40052F823F01DDA000831DA00083BDA0008C7
:10D9D40027DA00083BDA0008FBD90008F1D900086F
:10D9E4003BDA000813DA000805DA000839687868B9
:10D9F40000F03CFA24E03968786800F0CBFB1FE0C3
:10DA04003968786800F00AFC0346FB7318E039684B
:10DA1400786800F0ADFC13E03968786800F0DEFC4B
:10DA24000EE03968786800F00DFD09E0396878681F
:10DA340000F031FD04E03968786800F088FD00BF2B
:10DA440004E03968786800F082FD00BFFB7B18466B
:10DA54001037BD4680BD00BF80B584B000AF78608C
:10DA640039600023FB733B681B7803F06003402B91
:10DA740005D0402B52D8002B01D0202B4ED17B68EF
:10DA840093F89C32DBB2013B022B40D83B689B8865
:10DA9400DBB2012B36D83B689B88DBB21946786829
:10DAA400FFF7D9FE0346BB73BB7BFF2B1DD0BB7BAB
:10DAB400002B1AD1BA7B7B68AE3253F822309B68B4
:10DAC400002B0FD0BA7B7B68C3F8D422BA7B7B6867
:10DAD400AE3253F822309B68396878689847034619
:10DAE400FB7304E00323FB7301E00323FB733B6834
:10DAF400DB88002B10D1FB7B002B0DD1786800F064
:10DB0400F1FD09E03968786800F021FD04E0396826
:10DB1400786800F01CFD00E000BF04E03968786814
:10DB240000F015FD00BFFB7B18461037BD4680BDD5
:10DB340080B584B000AF786039600023FB733B6824
:10DB44009B88BB733B681B7803F06003402B07D0B2
:10DB5400402B00F27F81002B2AD0202B40F07A81C9
:10DB6400BB7B19467868FFF783FE03467B737B7B98
:10DB7400FF2B00F074817B7B002B40F070817A7B5B
:10DB84007B68C3F8D4227A7B7B68AE3253F82230A8
:10DB94009B68002B00F063817A7B7B68AE3253F87C
:10DBA40022309B683968786898470346FB7356E1CE
:10DBB4003B685B78032B08D0032B00F34581002BD3
:10DBC40000F09B80012B3CD03EE17B6893F89C32B3
:10DBD400DBB2022B02D0032B16D02CE0BB7B002B34
:10DBE4000DD0BB7B802B0AD0BB7B1946786801F033
:10DBF400BBF98021786801F0B7F900BF20E03968EB
:10DC0400786800F0A4FC1BE03B685B88002B0ED115
:10DC1400BB7B002B0BD0BB7B802B08D03B68DB8805
:10DC2400002B04D1BB7B1946786801F09DF9786814
:10DC340000F058FD04E03968786800F088FC00BF03
:10DC440007E17B6893F89C32DBB2022B02D0032BF2
:10DC540016D04BE0BB7B002B0DD0BB7B802B0AD0B6
:10DC6400BB7B1946786801F07FF98021786801F060
:10DC74007BF900BF40E03968786800F068FC3BE05D
:10DC84003B685B88002B36D1BB7B03F07F03002B02
:10DC940004D0BB7B1946786801F085F9786800F0F8
:10DCA40021FDBB7B19467868FFF7E2FD03467B73D1
:10DCB4007B7BFF2B1FD07B7B002B1CD17A7B7B686B
:10DCC400C3F8D4227A7B7B68AE3253F822309B6847
:10DCD400002B10D07A7B7B68AE3253F822309B68DD
:10DCE4003968786898470346FB7304E039687868B4
:10DCF40000F02DFC00E000BFABE07B6893F89C32A1
:10DD0400DBB2022B02D0032B32D097E0BB7B002B7B
:10DD140007D0BB7B802B04D03968786800F017FCEF
:10DD240091E097F90E30002B0BDABB7B03F07F02F6
:10DD340013469B0013449B0010337A681344043346
:10DD44000BE0BB7B03F07F0213469B0013449B0054
:10DD540003F5A8737A6813440433BB60BB680022DC
:10DD64001A60BB6802221946786800F061FC6AE018
:10DD740097F90E30002B11DABB7B03F00F027968A0
:10DD840013469B0013449B000B4424331B88002B35
:10DD940017D13968786800F0DAFB54E0BB7B03F0F4
:10DDA4000F02796813469B0013449B000B4403F550
:10DDB400B2731B88002B04D13968786800F0C7FB64
:10DDC40041E097F90E30002B0BDABB7B03F07F02A6
:10DDD40013469B0013449B0010337A6813440433A6
:10DDE4000BE0BB7B03F07F0213469B0013449B00B4
:10DDF40003F5A8737A6813440433BB60BB7B002B20
:10DE040002D0BB7B802B03D1BB6800221A600EE0DA
:10DE1400BB7B1946786801F0E5F80346002B03D074
:10DE2400BB6801221A6002E0BB6800221A60BB686A
:10DE340002221946786800F0FBFB04E03968786830
:10DE440000F085FB00BF04E03968786800F07FFBD0
:10DE540000BF05E03968786800F079FB00E000BF96
:10DE6400FB7B18461037BD4680BD000080B584B0EA
:10DE740000AF7860396000233B810023FB600023FE
:10DE8400FB723B685B881B0A9BB2013B0E2B00F2C2
:10DE9400528101A252F823F00DDF000825DF0008AB
:10DEA40065DF00083BE100083BE10008DBE0000817
:10DEB40007E100083BE100083BE100083BE1000802
:10DEC4003BE100083BE100083BE100083BE10008BE
:10DED400D9DE00087B68D3F8B432DB69002B0BD0A1
:10DEE4007B68D3F8B432DB697A68127C07F10801E5
:10DEF40010469847F86026E13968786800F027FBF7
:10DF0400FB7A0133FB721EE17B68D3F8B4321B68E1
:10DF14007A68127C07F1080110469847F86012E10C
:10DF24007B681B7C002B0DD17B68D3F8B8329B6ACD
:10DF340007F1080210469847F860FB680133022293
:10DF44001A7000E17B68D3F8B832DB6A07F1080283
:10DF540010469847F860FB68013302221A70F2E019
:10DF64003B685B88DBB2052B00F2AC8001A252F85F
:10DF740023F000BF91DF0008C5DF0008F9DF0008C7
:10DF84002DE0000861E0000895E000087B68D3F804
:10DF9400B4325B68002B0BD07B68D3F8B4325B6877
:10DFA4007A68127C07F1080110469847F86091E0FE
:10DFB4003968786800F0CBFAFB7A0133FB7289E0A8
:10DFC4007B68D3F8B4329B68002B0BD07B68D3F802
:10DFD400B4329B687A68127C07F1080110469847AE
:10DFE400F86077E03968786800F0B1FAFB7A0133B9
:10DFF400FB726FE07B68D3F8B432DB68002B0BD084
:10E004007B68D3F8B432DB687A68127C07F10801C4
:10E0140010469847F8605DE03968786800F097FA30
:10E02400FB7A0133FB7255E07B68D3F8B4321B6989
:10E03400002B0BD07B68D3F8B4321B697A68127C4E
:10E0440007F1080110469847F86043E0396878689A
:10E0540000F07DFAFB7A0133FB723BE07B68D3F876
:10E06400B4325B69002B0BD07B68D3F8B4325B69A4
:10E074007A68127C07F1080110469847F86029E095
:10E084003968786800F063FAFB7A0133FB7221E0A7
:10E094007B68D3F8B4329B69002B0BD07B68D3F830
:10E0A400B4329B697A68127C07F1080110469847DC
:10E0B400F8600FE03968786800F049FAFB7A0133B8
:10E0C400FB7207E03968786800F041FAFB7A0133A3
:10E0D400FB7200BF37E07B681B7C002B09D17B6897
:10E0E400D3F8B8325B6B07F1080210469847F86022
:10E0F40029E03968786800F02AFAFB7A0133FB7268
:10E1040021E07B681B7C002B0DD17B68D3F8B832EF
:10E114001B6B07F1080210469847F860FB6801334F
:10E1240007221A700FE03968786800F010FAFB7A59
:10E134000133FB7207E03968786800F008FAFB7A6B
:10E144000133FB7200BFFB7A002B1ED13B68DB88D6
:10E15400002B16D03B89002B0ED03B68DA883B8914
:10E16400934228BF13469BB23B813B891A46F96808
:10E17400786800F05DFA09E03968786800F0E7F93A
:10E1840004E0786800F0AEFA00E000BF1037BD4646
:10E1940080BD00BF80B584B000AF786039603B6853
:10E1A4009B88002B31D13B68DB88002B2DD13B6849
:10E1B4005B887F2B29D83B685B88DBB203F07F0345
:10E1C400FB737B6893F89C32DBB2032B04D1396870
:10E1D400786800F0BCF91DE07B68FA7B83F89E2226
:10E1E400FB7B1946786800F029FF786800F07AFA1A
:10E1F400FB7B002B04D07B68022283F89C2209E07D
:10E204007B68012283F89C2204E03968786800F076
:10E214009EF900BF00BF1037BD4680BD80B584B0F5
:10E2240000AF786039600023FB733B685B88DAB227
:10E234004E4B1A704D4B1B78012B05D93968786801
:10E2440000F085F903238CE07B6893F89C32DBB201
:10E25400022B02D0032B29D075E0444B1B78002BF2
:10E2640020D0424B1B781A467B685A603F4B1B7880
:10E2740019467868FEF7BDFF0346FB73FB7B002B52
:10E2840008D03968786800F062F97B68022283F864
:10E294009C2265E0786800F025FA7B68032283F805
:10E2A4009C225DE0786800F01DFA59E02F4B1B7842
:10E2B400002B12D17B68022283F89C222B4B1B7803
:10E2C4001A467B685A60294B1B7819467868FEF712
:10E2D400ACFF786800F006FA42E0244B1B781A463B
:10E2E4007B685B689A422AD07B685B68DBB219461C
:10E2F4007868FEF79AFF1D4B1B781A467B685A60B4
:10E304001A4B1B7819467868FEF773FF0346FB73B4
:10E31400FB7B002B0FD03968786800F018F97B6814
:10E324005B68DBB219467868FEF77FFF7B680222E0
:10E3340083F89C2214E0786800F0D4F910E078683F
:10E3440000F0D0F90CE03968786800F000F9074B68
:10E354001B7819467868FEF768FF0323FB7300BF38
:10E36400FB7B18461037BD4680BD00BFA0060020C9
:10E3740080B582B000AF786039603B68DB88012BE0
:10E3840004D03968786800F0E2F823E07B6893F8F9
:10E394009C32DBB2022B02DC002B03DC15E0032BE6
:10E3A4000BD012E07B6800229A607B68083301225C
:10E3B4001946786800F03CF90CE07B6804330122CC
:10E3C4001946786800F034F904E03968786800F098
:10E3D400BEF800BF00BF0837BD4680BD80B582B01F
:10E3E40000AF786039607B6893F89C32DBB2013B04
:10E3F400022B1ED83B68DB88022B04D0396878686E
:10E4040000F0A5F81AE07B680122DA607B68D3F893
:10E41400A432002B05D07B68DB6843F002027B68E2
:10E42400DA607B680C3302221946786800F000F940
:10E4340004E03968786800F08AF800BF00BF083744
:10E44400BD4680BD80B582B000AF786039603B685E
:10E454005B88012B07D17B680122C3F8A42278686A
:10E4640000F040F913E03B685B88022B0BD13B685A
:10E474009B881B0A9BB2DAB27B6883F8A022786877
:10E4840000F030F903E03968786800F060F800BF04
:10E494000837BD4680BD80B582B000AF7860396072
:10E4A4007B6893F89C32DBB2013B022B0BD83B68B0
:10E4B4005B88012B0CD17B680022C3F8A422786806
:10E4C40000F010F904E03968786800F040F800E0E2
:10E4D40000BF00BF0837BD4680BD80B584B000AF23
:10E4E400786039603B68FB60FB681A787B681A7057
:10E4F400FB680133FB60FB681A787B685A70FB6821
:10E504000133FB60F868FFF717FA03461A467B6885
:10E514005A80FB680133FB60FB680133FB60F868D9
:10E52400FFF70AFA03461A467B689A80FB680133B0
:10E53400FB60FB680133FB60F868FFF7FDF90346F5
:10E544001A467B68DA8000BF1037BD4680BD80B5AF
:10E5540082B000AF786039608021786800F004FDF3
:10E564000021786800F000FD00BF0837BD4680BD7B
:10E5740080B586B000AFF860B9607A600023FB759F
:10E58400FB68002B36D0FB683B61386900F036F835
:10E59400034601339BB25B009AB27B681A80FB7D11
:10E5A400BA6813447A6812781A70FB7D0133FB75DC
:10E5B400FB7DBA68134403221A70FB7D0133FB759B
:10E5C40013E0FB7DBA6813443A6912781A703B6908
:10E5D40001333B61FB7D0133FB75FB7DBA6813445A
:10E5E40000221A70FB7D0133FB753B691B78002BFD
:10E5F400E7D100E000BF1837BD4680BD80B485B0C8
:10E6040000AF78600023FB737B68BB6005E0FB7B95
:10E614000133FB73BB680133BB60BB681B78002B01
:10E62400F5D1FB7B18461437BD465DF8047B704773
:10E6340080B584B000AFF860B9607A60FB680222EC
:10E64400C3F89422FB687A689A61FB687A68DA6195
:10E654007B68BA680021F86800F00FFD00231846B3
:10E664001037BD4680BD80B584B000AFF860B96096
:10E674007A607B68BA680021F86800F0FEFC002329
:10E6840018461037BD4680BD80B584B000AFF86031
:10E69400B9607A60FB680322C3F89422FB687A6845
:10E6A400C3F85821FB687A68C3F85C217B68BA68B0
:10E6B4000021F86800F002FD002318461037BD461B
:10E6C40080BD80B584B000AFF860B9607A607B68C3
:10E6D400BA680021F86800F0F1FC002318461037EE
:10E6E400BD4680BD80B582B000AF78607B680422EF
:10E6F400C3F89422002300220021786800F0BDFCB6
:10E70400002318460837BD4680BD80B582B000AFEF
:10E7140078607B680522C3F894220023002200213C
:10E72400786800F0CBFC002318460837BD4680BD4E
:10E7340080B500AF002212491248FEF7DDFC034603
:10E74400002B01D0F2F7F6FF0F490E48FEF704FD47
:10E754000346002B01D0F2F7EDFF0C490948FEF700
:10E764003BFC0346002B01D0F2F7E4FF0548FEF71B
:10E7740029FD0346002B01D0F2F7DCFF00BF80BD6A
:10E78400B8000020A406002024000020A4000020DB
:10E7940080B500AF002205490548FEF737FC05495E
:10E7A4000348FEF755FC0023184680BD8011002065
:10E7B400A40600208009002080B400AF002318467E
:10E7C400BD465DF8047B704780B483B000AF034658
:10E7D4003960FB711346BB80FB79232B4AD801A215
:10E7E40052F823F079E8000879E8000879E800088D
:10E7F40079E8000879E8000879E8000879E8000871
:10E8040079E8000879E8000879E8000879E8000860
:10E8140079E8000879E8000879E8000879E8000850
:10E8240079E8000879E8000879E8000879E8000840
:10E8340079E8000879E8000879E8000879E8000830
:10E8440079E8000879E8000879E8000879E8000820
:10E8540079E8000879E8000879E8000879E8000810
:10E8640079E8000879E8000879E8000879E8000800
:10E8740079E8000800BF002318460C37BD465DF850
:10E88400047B704790B585B000AF78603960164A54
:10E8940007F1080392E80300186004331980134851
:10E8A400FEF7F4FB07F108031946786800F0F8FC5A
:10E8B4000346002B0DD07868F1F7A2FC044607F15B
:10E8C40008031846F1F79CFC03469C4201D1F2F779
:10E8D400CBFB4FF400620021786800F0D9FC0023E0
:10E8E40018461437BD4690BD1CF30008A40600204A
:10E8F40080B487B000AFF860B9601346FB710023A1
:10E90400FB7597F9173018461C37BD465DF8047B34
:10E914007047000080B483B000AF03463960FB71D8
:10E924003B6812221A80034B18460C37BD465DF82B
:10E93400047B7047D800002080B483B000AF034646
:10E944003960FB713B6804221A80034B18460C376C
:10E95400BD465DF8047B7047F800002080B582B0A6
:10E9640000AF03463960FB71FB79002B05D13A688F
:10E9740007490848FFF7FCFD04E03A6804490548E4
:10E98400FFF7F6FD024B18460837BD4680BD00BFB1
:10E994008019002024F3000880B582B000AF03463C
:10E9A4003960FB713A6804490448FFF7E1FD024B02
:10E9B40018460837BD4680BD801900203CF3000886
:10E9C40080B582B000AF03463960FB713B681A2200
:10E9D4001A8000F055F8024B18460837BD4680BD32
:10E9E400FC00002080B582B000AF03463960FB71A3
:10E9F400FB79002B05D13A6807490848FFF7B8FDB1
:10EA040004E03A6804490548FFF7B2FD024B184692
:10EA14000837BD4680BD00BF8019002050F30008B0
:10EA240080B582B000AF03463960FB71FB79002BDF
:10EA340005D13A6807490848FFF79AFD04E03A68A7
:10EA440004490548FFF794FD024B18460837BD46B4
:10EA540080BD00BF801900205CF3000880B483B03F
:10EA640000AF03463960FB713B680C221A80034BEC
:10EA740018460C37BD465DF8047B7047EC00002057
:10EA840080B584B000AF0F4B1B68FB600E4B1B6856
:10EA9400BB600E4B1B687B60FA687B681344FB60A9
:10EAA400FB68002B09D008220949F86800F014F823
:10EAB40004220849B86800F00FF800BF1037BD46BB
:10EAC40080BD00BF107AFF1F147AFF1F187AFF1F42
:10EAD400FE0000200E01002080B487B000AFF86073
:10EAE400B9601346FB710023FB750023FB7527E017
:10EAF400FB681B0F092B0BD8FB681B0FDAB2FB7DDD
:10EB04005B001946BB680B443032D2B21A700AE07B
:10EB1400FB681B0FDAB2FB7D5B001946BB680B4434
:10EB24003732D2B21A70FB681B01FB60FB7D5B00BD
:10EB34000133BA68134400221A70FB7D0133FB755C
:10EB4400FA7DFB799A42D3D300BF00BF1C37BD4680
:10EB54005DF8047B7047000080B5A0B000AF78601A
:10EB640007F16C0300221A605A609A60DA601A6135
:10EB740007F110035C220021184600F089FB7B6832
:10EB84001B68B3F1A04F49D14FF480733B6100235C
:10EB94007B6607F110031846F8F752FA0346002B78
:10EBA40001D0F2F7C7FD0023FB601E4B1B6B1D4A0F
:10EBB40043F0010313631B4B1B6B03F00103FB6066
:10EBC400FB684FF4C053FB6602233B6700237B675B
:10EBD4000323BB670A23FB6707F16C03194612483A
:10EBE400F5F762FC0F4B5B6B0E4A43F080035363F3
:10EBF4000023BB600B4B5B6C0A4A43F480435364B1
:10EC0400084B5B6C03F48043BB60BB6800220021AB
:10EC14004320F5F718F84320F5F731F800BF8037A3
:10EC2400BD4680BD003802400000024080B582B07D
:10EC340000AF78607B68D3F808257B6803F2C4438F
:10EC440019461046FEF70BFB00BF0837BD4680BDD2
:10EC540080B582B000AF78600B46FB707B68D3F858
:10EC64000805FA7879681346DB0013449B000B44CB
:10EC740003F523731A68FB781946FEF745FB00BFBA
:10EC84000837BD4680BD80B582B000AF78600B46C2
:10EC9400FB707B68D3F80805FA7879681346DB00C3
:10ECA40013449B000B444C331A68FB781946FEF757
:10ECB400DEFB00BF0837BD4680BD80B582B000AF23
:10ECC40078607B68D3F808351846FEF712FD00BF5C
:10ECD4000837BD4680BD80B584B000AF786001239D
:10ECE400FB737B68DB68002B02D10023FB7308E015
:10ECF4007B68DB68022B02D10123FB7301E0F2F78E
:10ED040019FD7B68D3F80835FA7B11461846FEF7DF
:10ED1400B2FC7B68D3F808351846FEF75AFC00BFEE
:10ED24001037BD4680BD000080B582B000AF78606A
:10ED34007B68D3F808351846FEF7ADFC7B681B6882
:10ED440003F560631B687A68126802F5606243F039
:10ED5400010313607B681B6A002B05D0044B1B69FD
:10ED6400034A43F00603136100BF0837BD4680BD64
:10ED740000ED00E080B582B000AF78607B68D3F826
:10ED840008351846FEF79DFC00BF0837BD4680BD18
:10ED940080B582B000AF78600B46FB707B68D3F817
:10EDA4000835FA7811461846FEF7F5FC00BF083717
:10EDB400BD4680BD80B582B000AF78600B46FB7065
:10EDC4007B68D3F80835FA7811461846FEF7B1FC8B
:10EDD40000BF0837BD4680BD80B582B000AF786003
:10EDE4007B68D3F808351846FEF707FD00BF0837DF
:10EDF400BD4680BD80B582B000AF78607B68D3F833
:10EE040008351846FEF704FD00BF0837BD4680BD2F
:10EE140080B582B000AF78607B681B78002B3CD152
:10EE2400204A7B68C2F808357B681E4AC3F8C822AA
:10EE34001C4B4FF0A0421A601A4B06225A60194B21
:10EE44000222DA60174B00221A61164B02229A61E1
:10EE5400144B0022DA61134B00221A62114B002278
:10EE64005A62104B0022DA620E4B00221A630D48DC
:10EE7400F6F7D1FC0346002B01D0F2F75BFC8021AE
:10EE84000848F7F75CFF402200210648F7F710FF17
:10EE9400802201210348F7F70BFF002318460837A7
:10EEA400BD4680BD801B002080B584B000AF786073
:10EEB4000023FB730023BB737B68D3F8C832184666
:10EEC400F6F7CDFD0346FB73FB7B184600F090F983
:10EED4000346BB73BB7B18461037BD4680BD80B567
:10EEE40084B000AF7860084611461A460346FB70AA
:10EEF4000B46BB7013463B800023FB730023BB739C
:10EF04007B68D3F8C802BB783A88F978F7F7CBFA6C
:10EF14000346FB73FB7B184600F06AF90346BB7398
:10EF2400BB7B18461037BD4680BD80B584B000AFAA
:10EF340078600B46FB700023FB730023BB737B6874
:10EF4400D3F8C832FA7811461846F7F714FB03468B
:10EF5400FB73FB7B184600F04BF90346BB73BB7B8A
:10EF640018461037BD4680BD80B584B000AF7860C8
:10EF74000B46FB700023FB730023BB737B68D3F841
:10EF8400C832FA7811461846F7F7ECFB0346FB73D0
:10EF9400FB7B184600F02CF90346BB73BB7B184679
:10EFA4001037BD4680BD80B584B000AF78600B4695
:10EFB400FB700023FB730023BB737B68D3F8C83258
:10EFC400FA7811461846F7F731FC0346FB73FB7BCE
:10EFD400184600F00DF90346BB73BB7B1846103787
:10EFE400BD4680BD80B485B000AF78600B46FB7031
:10EFF4007B68D3F8C832FB6097F90330002B0BDA37
:10F00400FB7803F07F02F9681346DB0013449B008E
:10F014000B443E331B780BE0FB7803F07F02F96866
:10F024001346DB0013449B000B4403F27E231B783E
:10F0340018461437BD465DF8047B704780B584B02C
:10F0440000AF78600B46FB700023FB730023BB7397
:10F054007B68D3F8C832FA7811461846F7F7FEF9F8
:10F064000346FB73FB7B184600F0C2F80346BB73F0
:10F07400BB7B18461037BD4680BD80B586B000AF57
:10F08400F8607A603B600B46FB720023FB7500233B
:10F09400BB75FB68D3F8C802F97A3B687A68F7F75E
:10F0A40017FB0346FB75FB7D184600F0A1F80346E9
:10F0B400BB75BB7D18461837BD4680BD80B586B08C
:10F0C40000AFF8607A603B600B46FB720023FB756F
:10F0D4000023BB75FB68D3F8C802F97A3B687A68E9
:10F0E400F7F793FA0346FB75FB7D184600F080F8AA
:10F0F4000346BB75BB7D18461837BD4680BD80B539
:10F1040082B000AF78600B46FB707B68D3F8C832DE
:10F11400FA7811461846F7F7C3FA03461846083733
:10F12400BD4680BD80B582B000AF78600B46FB70F1
:10F13400FB78002B02D0012B1FD03BE07B681B6ABD
:10F14400002B07D0F2F728FA1C4B1B691B4A23F04B
:10F15400060313617B681B6803F560631B687A68A8
:10F16400126802F5606223F0010313607B68D3F830
:10F1740008351846FEF7A5FA1CE07B681B6803F502
:10F1840060631B687A68126802F5606243F00103E9
:10F1940013607B68D3F808351846FEF77CFA7B6861
:10F1A4001B6A002B05D0054B1B69044A43F0060378
:10F1B400136100BF00BF0837BD4680BD00ED00E00D
:10F1C40080B483B000AF7860034B18460C37BD465B
:10F1D4005DF8047B704700BF8C20002080B483B0AE
:10F1E40000AF786000BF0C37BD465DF8047B704704
:10F1F40080B485B000AF0346FB710023FB73FB7939
:10F20400032B17D801A252F823F000BF21F2000803
:10F2140027F200082DF2000833F200080023FB73E4
:10F224000BE00323FB7308E00123FB7305E00323D6
:10F23400FB7302E00323FB7300BFFB7B1846143708
:10F24400BD465DF8047B704770B50D4D0D4C641BD5
:10F25400A4100026A64209D10B4D0C4C00F036F840
:10F26400641BA4100026A64205D170BD55F8043BCA
:10F2740098470136EEE755F8043B98470136F2E724
:10F2840094F3000894F3000894F3000898F300083A
:10F2940002440346934200D1704703F8011BF9E787
:10F2A4000A7870B56AB970BD9A4209D10C46054610
:10F2B40014F8013F002BF6D015F8016F9E42F7D0E9
:10F2C40001300378002BEFD11846ECE7F8B500BF06
:10F2D400F8BC08BC9E467047F8B500BFF8BC08BC33
:04F2E4009E4670478B
:10F2E8000102030405060708090A0000EC000100F2
:10F2F800C30000009000060101000000910000001A
:10F308000A000000800000000400000093000001D3
:10F31800F40000004D3939393900000053544D3399
:10F3280032205669727475616C20436F6D506F722C
:10F338007400000053544D6963726F656C656374A3
:10F34800726F6E696373000043444320436F6E66B7
:10F358006967000043444320496E746572666163BF
:10F368006500000000000000000000000102030426
:10F378000607080900000000010203040006101631
:04F388000006101655
:08F38C00B80EFF7F0100000034
:04F39400E901000883
:04F39800C5010008A3
:10F39C000102030405060101010000000024F40031
:10F3AC0010000000010000000A06000200000040EE
:10F3BC0001000000DDC70008CDC90008D1CA000853
:10F3CC0000000000F7CD000889CC000887CD0008AC
:10F3DC00000000000000000000000000DDCE00086E
:10F3EC006DCE00084DCF0008BDCF000809024300C8
:10F3FC00020100C0320904000001020201000524D0
:10F40C000010010524010001042402020524060059
:10F41C00010705820308001009040100020A00001C
:10F42C000007050102400000070581024000008131
:10F43C000182000095E70008BDE70008CDE7000851
:10F44C0089E80008F5E8000819E900083DE900081A
:10F45C009DE9000861E90008C5E90008E9E9000830
:10F46C0025EA000861EA00081201010202020040CC
:10F47C00830440570002010203010000050F0C0039
:10F48C000107100202000000040309041A03000023
:10F49C000000000000000000000000000000000060
:08F4AC00000000000000000058
:0400000508002E6160
:00000001FF
